:0420000051EF10F09C
:062008005B82BEEFA5F0B3
:102018005B80D8CFEDF2E8CFEEF2E0CFEFF2FACF67
:10202800F0F2FBCFF1F2E1CFF2F2E2CFF3F2D9CF47
:10203800F4F2DACFF5F2F3CFF6F2F4CFF7F2F6CF07
:10204800F8F2F7CFF9F2F8CFFAF2F5CFFBF29DB23A
:102058009EA203D033EC46F09E92FBC2F5FFFAC273
:10206800F8FFF9C2F7FFF8C2F6FFF7C2F4FFF6C2AD
:10207800F3FFF5C2DAFFF4C2D9FFF3C2E2FFF2C2FE
:10208800E1FFF1C2FBFFF0C2FAFFEFC2E0FFEEC2D0
:10209800E8FFEDC2D8FF5B901000F4EFBFF000013D
:1020A800000A006400E80310270100100000010086
:1020B800107E2138210421C12009024300020100B9
:1020C800C0320904000001020201000524001001C9
:1020D8000424020205240600010524010001070565
:1020E800810308000209040100020A000000070534
:1020F800020240000007058202400000340343004A
:10210800440043002000520053002D0032003300E9
:102118003200200045006D0075006C0061007400FD
:1021280069006F006E002000440065006D006F00BC
:1021380034034D006900630072006F00630068009B
:1021480069007000200054006500630068006E009C
:102158006F006C006F0067007900200049006E0076
:1021680063002E001201000202000008D8040A00D1
:102178000001010200010403090446697265205A3E
:102188006F6E65202575206661756C7420726573A5
:10219800746F72652E506172746974696F6E203144
:1021A8002E0D0A0046697265205A6F6E65202575E6
:1021B800206661756C7420726573746F72652E5039
:1021C8006172746974696F6E20322E0D0A00503284
:1021D8002E456E7472792064656C6179206578701B
:1021E800697265642E44656C6179207A6F6E65202A
:1021F800616C61726D0D0A00535441592044495372
:1022080041524D494E472E20557365722020257541
:102218002E506172746974696F6E20312E0D0A0038
:10222800535441592044495341524D494E472E2059
:1022380055736572202025752E5061727469746912
:102248006F6E20322E0D0A004D6F646520503120CC
:102258002D206B6579706164732073757065727673
:1022680069736F72792072657365742E0D0A004D5B
:102278006F6465205032202D206B6579706164731E
:102288002073757065727669736F727920726573E1
:1022980065742E0D0A004D6F6465205031202D2085
:1022A80072657475726E20746F2073656C656374E3
:1022B800696E67206D6F64652E0D0A004D6F646549
:1022C800205032202D2072657475726E20746F2034
:1022D80073656C656374696E67206D6F64652E0D38
:1022E8000A00535441592041524D494E472E20551A
:1022F800736572202025752E506172746974696F38
:102308006E20312E0D0A00535441592041524D4937
:102318004E472E2055736572202025752E50617208
:10232800746974696F6E20322E0D0A0046697265F1
:10233800205A6F6E6520257520726573746F7265FB
:102348002E506172746974696F6E20312E0D0A0007
:1023580046697265205A6F6E65202575207265730F
:10236800746F72652E506172746974696F6E203271
:102378002E0D0A004D6F6465205031202D207265A6
:102388007475726E20746F2067656E6572616C205B
:102398006D6F64652E0D0A004D6F64652050322004
:1023A8002D2072657475726E20746F2067656E6576
:1023B80072616C206D6F64652E0D0A0041434620E2
:1023C8007A6F6E6520257520726573746F72652E3D
:1023D800506172746974696F6E20312E0D0A004164
:1023E8004346207A6F6E6520257520726573746F79
:1023F80072652E506172746974696F6E20322E0D89
:102408000A0046697265205A6F6E6520257520613D
:102418006C61726D2E506172746974696F6E2031CF
:102428002E0D0A0046697265205A6F6E6520257563
:10243800206661756C742E506172746974696F6E70
:1024480020312E0D0A0046697265205A6F6E65208C
:10245800257520616C61726D2E50617274697469A2
:102468006F6E20322E0D0A0046697265205A6F6E13
:1024780065202575206661756C742E5061727469CB
:1024880074696F6E20322E0D0A005375706572766E
:1024980069736F727920726573746F72652E204B41
:1024A80065797061642025752E0D0A004143462028
:1024B8007A6F6E6520257520616C61726D2E506192
:1024C80072746974696F6E20312E0D0A004143469B
:1024D800207A6F6E6520257520616C61726D2E50B3
:1024E8006172746974696F6E20322E0D0A00466F2E
:1024F8007263656420657869742066726F6D2074F4
:1025080072616E736D697373696F6E2E0D0A003E8A
:102518004576656E742E436F64652066726F6D2014
:102528004573707269742E25752C25752E0D0A0059
:102538005F4B65797061645F44656C657465416C77
:102548006C5573657273436F64657328293B0D0A74
:102558000053757065727669736F727920616C616A
:10256800726D2E204B65797061642025752E0D0AD9
:10257800005F44616C6C61735F44656C65746541B0
:102588006C6C55736572734B65797328293B0D0A1A
:10259800003E4576656E743A2575202025632563CF
:1025A80025632025632563202563256325630D0A9C
:1025B800004D6F6465205031202D206B6579706166
:1025C800642070726F6772616D6D696E672E0D0A97
:1025D800004D6F6465205032202D206B6579706145
:1025E800642070726F6772616D6D696E672E0D0A77
:1025F800004C4152532062797465733A2025582C57
:102608002025582C2025582C202558200D0A00500C
:10261800616E656C206D6F64652070617274697499
:10262800696F6E2031203D20302E0D0A0050616EFA
:10263800656C206D6F646520706172746974696F70
:102648006E2032203D20302E0D0A003E4368616E18
:102658006765207365637572697479206D6F646549
:1026680020746F20302E0D0A003E4368616E676546
:10267800207365637572697479206D6F6465207461
:102688006F20312E0D0A004576656E742E436F64F7
:10269800652066726F6D20445343202825582558BD
:1026A800292E0D0A004D6F6465205031202D2063BE
:1026B8006F64652070726F6772616D6D696E672EE9
:1026C8000D0A004D6F6465205032202D20636F6421
:1026D800652070726F6772616D6D696E672E0D0A85
:1026E800004C6F6164696E672064656661756C741F
:1026F8002070726F66696C652E2E2E0D0A005A6F57
:102708006E6520312E205377696E67657220736875
:102718007574646F776E2E0D0A005A6F6E652032DD
:102728002E205377696E6765722073687574646FBD
:10273800776E2E0D0A005A6F6E6520332E20537760
:10274800696E6765722073687574646F776E2E0D95
:102758000A005A6F6E6520342E205377696E6765BC
:10276800722073687574646F776E2E0D0A005A6F45
:102778006E6520352E205377696E67657220736801
:102788007574646F776E2E0D0A005A6F6E65203669
:102798002E205377696E6765722073687574646F4D
:1027A800776E2E0D0A005F4B65797061645F446532
:1027B8006C657465416C6C436F64657328293B0DC7
:1027C8000A005F44616C6C61735F44656C65746595
:1027D800416C6C4B65797328293B0D0A004E6F20BC
:1027E800616E737765722066726F6D206D6F6475A8
:1027F8006C652025750D0A005A6F6E652064756D2D
:10280800703A204B312D25582C204B322D25582E2F
:102818000D0A0044656661756C742070726F666994
:102828006C65206C6F616465642E0D0A003E53650B
:1028380063757269747920636F6465206368616E7B
:102848006765642E0D0A00536176696E67206E65B0
:1028580077204D4153544552204B45592E0D0A00BF
:10286800496E637265617365206F6620505350200E
:1028780044656C61792E0D0A00436F6465202564F8
:102888002E506172746974696F6E2025642E0D0A6A
:10289800004E6577206775617264206B65792073D7
:1028A8006176696E672E0D0A004D6173746572203A
:1028B800636F64652E204D6F64652025752E0D0AA3
:1028C80000434F525445582053656E64696E672023
:1028D800746573742E2E0D0A005A6F6E6520256478
:1028E80020636F756E7465722072657365740D0A66
:1028F800004E65772075736572206B65792073616A
:1029080076696E672E0D0A003E4576656E742E4315
:102918006F64652066726F6D2053422E0D0A004465
:10292800656661756C742E20556E706C75672055E0
:1029380053422E0A0D004D6F646520503120726598
:102948007475726E20746F20302E0D0A004D6F64FE
:10295800652050322072657475726E20746F203055
:102968002E0D0A004C4152532053656E64696E6700
:1029780020746573742E2E0D0A004F726967696E94
:10298800616C205053502044656C61792E0D0A000B
:102998004B6579706164203120656E726F6C6C696B
:1029A8006E672E0D0A004B657970616420322065D0
:1029B8006E726F6C6C696E672E0D0A004576656ED7
:1029C800742E204D6173746572204F5554210D0A81
:1029D80000204E6F2054726D2E4576656E7420204F
:1029E8002575200D0A004D65737361676520667251
:1029F8006F6D20414241532E0D0A003E4C6F6164B9
:102A08002063666720726571756573742E0D0A0000
:102A180053757065727669736F7279207265736524
:102A2800742E0D0A004576656E742E204D61737400
:102A3800657220494E210D0A005A6F6E65203220BA
:102A4800697320636C6F7365212E0D0A003E536510
:102A58007269616C20427573206D6F64652E0D0A72
:102A6800003E555342206366672072657175657331
:102A7800742E0D0A0023343A303230303030303280
:102A88003030303046430D0A004D6F64756C652058
:102A980025752072656D6F7665640D0A0025582CC2
:102AA80025582C25582C25582C25582C25580D0AE6
:102AB800004E657720636F646520736176696E6781
:102AC8002E0D0A00506F696E74657220636C656123
:102AD8007265642E0D0A0042617474657279207201
:102AE8006573746F72652E0D0A005A6F6E6520311A
:102AF80020697320636C6F73652E0D0A005A6F6E20
:102B080065203220697320636C6F73652E0D0A008F
:102B18005A6F6E65203320697320636C6F73652E5E
:102B28000D0A005A6F6E65203420697320636C6F3C
:102B380073652E0D0A005A6F6E6520352069732063
:102B4800636C6F73652E0D0A005A6F6E6520362010
:102B5800697320636C6F73652E0D0A00434F5254DE
:102B680045582070726F746F636F6C2E0D0A005594
:102B780053422072656C6F61642E432F25752E0DAC
:102B88000A004D6F64756C65206973207265616415
:102B9800792E0D0A00506F696E74657220636C653A
:102BA800617265642E0A0D0044656C617920657850
:102BB800706972656420320D0A0023343A3030306F
:102BC800303030303146460D0A0D0A004C6F672010
:102BD800636C656172696E672E2E2E0D0A004B6557
:102BE80079737769746368206D6F64652E0D0A00C8
:102BF8003E4D6167656C6C616E206D6F64652E0D6E
:102C08000A0044534320697320726573746F7265B8
:102C18002E0D0A004C415253312070726F746F634D
:102C28006F6C2E0D0A005A6F6E6520312069732073
:102C38006F70656E2E0D0A005A6F6E65203220691E
:102C480073206F70656E2E0D0A005A6F6E65203303
:102C5800206973206F70656E2E0D0A005A6F6E65BD
:102C68002034206973206F70656E2E0D0A005A6F2C
:102C78006E652035206973206F70656E2E0D0A0011
:102C88005A6F6E652036206973206F70656E2E0D41
:102C98000A004D6F64756C65202575206164646554
:102CA800640D0A005031206B65795F636F6465209D
:102CB8002558200D0A005032206B65795F636F64D8
:102CC80065202558200D0A00303132333435363727
:102CD8003839414243444546004B657973776974F6
:102CE8006368206F6666210D0A0043494420202549
:102CF80058202558202558200D0A003E4D6F646540
:102D080020756E6B6E6F776E210D0A0057616974BE
:102D180020666F72206865782E2E0D0A004E5820A6
:102D2800697320726573746F72652E0D0A004C41C9
:102D380052532070726F746F636F6C2E0D0A0052BD
:102D48006567206D6F646520657869742E0D0A00CB
:102D58003E4D6F646520726571756573742E0D0A3A
:102D68000055534220736F66742072657365740D45
:102D78000A004576656E742066726F6D204E582E77
:102D88000D0A004B657970616473207265696E691C
:102D98002E0D0A004B6579737769746368206F6E2E
:102DA800210D0A004C4152535F646174612025581B
:102DB800200D0A003E457370726974206D6F64655A
:102DC8002E0D0A003E4C6F6720726571756573742D
:102DD8002E0D0A004E65656420656E747279203286
:102DE8000D0A0055736572206B65792025642E0DD8
:102DF8000A004C4F4720636C65617265642E0D0AAA
:102E0800004B6579706164206D6F64652E0D0A0052
:102E18003E50616E656C206D6F64652E0D0A00442E
:102E2800616C6C6173206D6F64652E0D0A004453EC
:102E380043206973206C6F73742E0D0A004261740D
:102E480074657279206C6F772E0D0A0052656720C1
:102E58006D6F646520312E0D0A00204576656E740D
:102E680020202575200D0A0053746174696F6E2047
:102E78002575200D0A00536C656570696E672E2EE6
:102E88002E0D0A003E41425553206D6F64652E0D8C
:102E98000A004C415253207461626C652E0D0A0081
:102EA8004E58206973206C6F73742E0D0A00436F9F
:102EB8006465206572726F720D0A0057616B696EE6
:102EC80067207570210D0A003E445343206D6F64DE
:102ED800652E0D0A00762E25645F6D6F6465300DD2
:102EE8000A005A3120636C6F73652E0D0A005A323E
:102EF80020636C6F73652E0D0A005A3320636C6F64
:102F080073652E0D0A005A3420636C6F73652E0D9D
:102F18000A005A3520636C6F73652E0D0A005A3605
:102F280020636C6F73652E0D0A005A3720636C6F2F
:102F380073652E0D0A005A3820636C6F73652E0D69
:102F48000A00556E6C6F636B6564210D0A00546549
:102F58007374204F46462E0D0A003E4E58206D6F62
:102F680064652E0D0A004353206572726F722E0D30
:102F78000A00556E6C6F636B6564210A0D00546519
:102F88007374204F46462E0A0D005A31206F706523
:102F98006E2E0D0A005A32206F70656E2E0D0A00D3
:102FA8005A33206F70656E2E0D0A005A34206F70E8
:102FB800656E2E0D0A005A35206F70656E2E0D0A4B
:102FC800005A36206F70656E2E0D0A005A37206F32
:102FD80070656E2E0D0A005A38206F70656E2E0DC2
:102FE8000A00434F4445204552520A0D00496E7469
:102FF8006572696F722000545832202575200D0AB9
:1030080000545833202575200D0A0054726D202570
:1030180075200D0A00434F4445204F4B0A0D002AE6
:10302800236C6F636B5F6530005374617274210D9C
:103038000A00746573745F6F6666004B65792025B6
:10304800580D0A002A2370636C72660050313A20CA
:10305800230D0A0050323A20230D0A0050313A203D
:103068002A0D0A0050323A202A0D0A0050313A201F
:10307800300D0A0050323A20300D0A0050313A2003
:10308800310D0A0050323A20310D0A0050313A20F1
:10309800320D0A0050323A20320D0A0050313A20DF
:1030A800330D0A0050323A20330D0A0050313A20CD
:1030B800340D0A0050323A20340D0A0050313A20BB
:1030C800350D0A0050323A20350D0A0050313A20A9
:1030D800360D0A0050323A20360D0A0050313A2097
:1030E800370D0A0050323A20370D0A0050313A2085
:1030F800380D0A0050323A20380D0A0050313A2073
:10310800390D0A0050323A20390D0A0044656C61C5
:103118007920004E414B210D0A0041434B210D0AF5
:10312800004D61672B0D0A004D61672D0D0A0031B6
:10313800306D2E0D0A00432F25640D0A003A6D6F7D
:10314800646530003A6D6F646531003A6E636F6490
:1031580065006C6F67636C7200356D2E0D0A002375
:10316800343A3130006D6F64653F0072656465669E
:10317800003A6C636667003A73636667003A6C6C82
:0F3188006F6700255820003A3030005445000092
:10319800A30ED66E0001E12B050E0201641903E1AE
:1031A800550E01012F6F270E0201641903E1750EF8
:1031B80001012F6FB10E0201641903E1A50E01018F
:1031C8002F6F640E0201641903E1350E01012F6FA0
:1031D800750E0201641903E1350E01012F6F7F0E90
:1031E8000201641903E1350E01012F6F690E020116
:1031F800641903E1350E01012F6F7A0E020164197B
:1032080003E1350E01012F6F820E0201641903E1FB
:10321800350E01012F6F5D0E0201641903E1750E71
:1032280001012F6F930E0201641903E1950E01014C
:103238002F6F0A0E0201641903E1950E01012F6F29
:103248004C0E0201641903E1A50E01012F6FD50E82
:103258000201641903E1950E01012F6F160E020198
:10326800641903E1550E01012F6F110E0201641953
:1032780003E1890E01012F6F5D0E0201641903E15C
:10328800750E01012F6F630E0201641903E1750EBB
:1032980001012F6FA50E0201641903E1830E0101DC
:1032A8002F6F01012F510001E15D01E327D263BDBA
:1032B80004D0786A7684A496A3868A9220D10201E3
:1032C80064BF11D28A820FD2020164BD0CD2FAD730
:1032D800020164BB08D2F6D7020164B904D2F2D75E
:1032E800020164B700D2EED7020164B5FCD1EAD777
:1032F800020164B3F8D1E6D7020164B1F4D1E2D790
:103308008A82E36BE26B0301986B976BECD1020145
:1033180063BFE9D1D7D7020163BDE5D1D3D7020195
:1033280063BBE1D1CFD7020163B9DDD1CBD70201AD
:1033380063B7D9D1C7D7020163B5D5D1C3D70201C5
:1033480063B3D1D1BFD7020163B1CDD1BBD70201DD
:1033580062BFC9D1B7D7020162BDC5D1B3D70201D7
:1033680062BBC1D1AFD7020162B9BDD1ABD70201EF
:1033780062B7B9D1A7D7020162B5B5D1A3D7020107
:1033880062B3B1D19FD7020162B1ADD19BD702011F
:1033980061BFA9D197D7020161BDA5D193D7020119
:1033A80061BBA1D18FD7020161B99DD18BD7020131
:1033B80061B799D187D7020161B595D183D7020149
:1033C80061B391D17FD7020161B18DD17BD7020161
:1033D80060BF89D177D7020160BD85D173D702015B
:1033E80060BB81D16FD7020160B97DD16BD7020173
:1033F80060B779D167D7020160B575D163D702018B
:1034080060B371D15FD7020160B16DD15BD7E8BFFE
:103418006AD158D7E8BD67D155D7E8BB64D152D730
:10342800E8B961D14FD7E8B75ED14CD7E8B55BD1E1
:1034380049D7E8B358D146D7E8B155D143D7E7BF04
:1034480052D140D7E7BD4FD13DD7E7BB4CD13AD792
:10345800E7B949D137D7E7B746D134D7E7B543D12C
:1034680031D7E7B340D12ED7E7B13DD12BD7E6BF4F
:103478003AD128D7E6BD37D125D7E6BB34D122D7F4
:10348800E6B931D11FD7E6B72ED11CD7E6B52BD177
:1034980019D7E6B328D116D7E6B125D113D7E5BF9A
:1034A80022D110D7E5BD1FD10DD7E5BB1CD10AD756
:1034B800E5B919D107D7E5B716D104D7E5B513D1C2
:1034C80001D7E5B310D1FED6E5B10DD1FBD6E4BFE7
:1034D8000AD1F8D6E4BD07D1F5D6E4BB04D1F2D6BB
:1034E800E4B901D1EFD6E4B7FED0ECD6E4B5FBD011
:1034F800E9D6E4B3F8D0E6D6E4B1F5D0E3D6E151A5
:10350800020A01E1DCD6060A01E1DED6020A01E17F
:10351800DFD60E0A01E1E0D6020A01E1E1D6060A89
:1035280001E1E2D6020A01E1E3D61E0A01E1E4D68E
:10353800020A01E1E5D6060A01E1E9D6020A01E13B
:10354800EAD60E0A01E1EBD6020A01E1ECD6060A38
:1035580001E1EDD6020A01E1EED63E0A01E1EFD61D
:10356800020A01E1F0D6060A01E1F1D6020A01E1F8
:10357800F2D60E0A01E1F3D6020A01E1F4D6060AF0
:1035880001E1F5D6020A01E1F6D61E0A01E1F7D6F5
:10359800020A01E1F8D6060A01E1F9D6020A01E1B8
:1035A800FAD60E0A01E1FBD6020A01E1FCD6060AA8
:1035B80001E1FDD6020A01E1FED67E0A01E1FFD64D
:1035C800020A01E100D7060A01E101D7020A01E176
:1035D80002D70E0A01E103D7020A01E104D7060A5D
:1035E80001E105D7020A01E106D71E0A01E107D762
:1035F800020A01E108D7060A01E109D7020A01E136
:1036080009D70E0A01E109D7020A01E109D7060A1A
:1036180001E109D7020A01E109D73E0A01E109D708
:10362800020A01E109D7060A01E109D7020A01E104
:1036380009D70E0A01E109D7020A01E109D7060AEA
:1036480001E109D7020A01E109D71E0A01E109D7F8
:10365800020A01E109D7060A01E109D7020A01E1D4
:1036680009D70E0A01E109D7020A01E109D7060ABA
:1036780001E109D7020A01E109D7FE0A01E109D7E8
:10368800020A01E109D7060A01E109D7020A01E1A4
:1036980009D70E0A01E109D7020A01E109D7060A8A
:1036A80001E109D7020A01E109D71E0A01E109D798
:1036B800020A01E109D7060A01E109D7020A01E174
:1036C80009D70E0A01E109D7020A01E109D7060A5A
:1036D80001E109D7020A01E109D73E0A01E109D748
:1036E800020A01E109D701012F050001716F71512B
:1036F800E11901E18A828A76637D120001012F5166
:103708000001E11901E18A9201012F51090F00011D
:10371800716F7151E15D02E28A96639D7151E11901
:10372800D8A41200E16B0201975101E097073C0E03
:10373800971902E13AECCBF0460E97190EE1000119
:1037480067B109D0020E016E010EA1EC9FF0020EC6
:10375800016EA1EC9FF0000167915F0E02019719BD
:1037680001E07FD00001706B0201652B65510A0DE5
:10377800400EF324D96E040EF420DA6EB10EDF6E1B
:1037880065510A0D410EF324D96E040EF420DA6E49
:103798005BC2DFFF65510A0D420EF324D96E040E99
:1037A800F420DA6EDF6A65510A0D430EF324D96EF0
:1037B800040EF420DA6EDF6A65510A0D440EF32414
:1037C800D96E040EF420DA6EDF6A65510A0D450ED3
:1037D800F324D96E040EF420DA6E5AC2DFFF655165
:1037E8000A0D460EF324D96E040EF420DA6EDF6A51
:1037F80065510A0D470EF324D96E040EF420DA6ED3
:10380800DF6A65510A0D480EF324D96E040EF420C0
:10381800DA6EDF6A0001726B080E726501D016D08D
:10382800020165510A0D400E4D6E040E4E6EF350A6
:103838004D26F4504E22000172514D24D96E000ECF
:103848004E20DA6EDF507027722BE6D702016551E1
:103858000A0D490EF324D96E040EF420DA6E70C0F6
:10386800DFFF5A0E971960E1652B65510A0D400E6E
:10387800F324D96E040EF420DA6E160EDF6E65514D
:103888000A0D410EF324D96E040EF420DA6E0E0EE2
:10389800DF6E65510A0D420EF324D96E040EF42032
:1038A800DA6E230EDF6E65510A0D430EF324D96ECE
:1038B800040EF420DA6EF20EDF6E65510A0D440E26
:1038C800F324D96E040EF420DA6E390EDF6E6551DA
:1038D8000A0D450EF324D96E040EF420DA6EDF6863
:1038E80065510A0D460EF324D96E040EF420DA6EE3
:1038F800DF6865510A0D470EF324D96E040EF420D3
:10390800DA6EDF6865510A0D480EF324D96E040E8D
:10391800F420DA6EDF6865510A0D490EF324D96E7A
:10392800040EF420DA6EDF68550E97195CE1652BFA
:1039380065510A0D400EF324D96E040EF420DA6E98
:10394800110EDF6E65510A0D410EF324D96E040E77
:10395800F420DA6EDF6865510A0D420EF324D96E41
:10396800040EF420DA6EDF6865510A0D430EF32465
:10397800D96E040EF420DA6EDF6865510A0D440E24
:10398800F324D96E040EF420DA6EDF6865510A0D4F
:10399800450EF324D96E040EF420DA6EDF68655103
:1039A8000A0D460EF324D96E040EF420DA6EDF6891
:1039B80065510A0D470EF324D96E040EF420DA6E11
:1039C800DF6865510A0D480EF324D96E040EF42001
:1039D800DA6EDF6865510A0D490EF324D96E040EBC
:1039E800F420DA6EDF68110E641901E0C1D0E3C07B
:1039F8004DF0C00E4D1603E10001648302D00001B2
:103A08006493E3C04DF0300E4D1602E1638F01D090
:103A1800639F0201975144E077C24DF0030E4D16A3
:103A280014E1776B000164A302D0020177810001E1
:103A380063AF02D002017783170E0C6E040E0B6E73
:103A480077C20DF00DECCAF01DD0000164B30BD0A5
:103A5800020177A108D00B0E396E010E3A6EBCEC4C
:103A680058F000016A89000163BF0CD0020177A3F6
:103A780009D00B0E396E020E3A6E010EBCEC58F0EE
:103A880000016A87000164A302D0648502D00001A6
:103A9800649563AF02D064816BD00001649168D0F3
:103AA800000164A564A325D0020177B115D0778100
:103AB800170E0C6E040E0B6E77C20DF00DECCAF0EB
:103AC800980E1E6E290E1F6ED1ECD0F0640E020106
:103AD800976F000167810DD00C0E396E010E3A6E9A
:103AE800BCEC58F08B0E1E6E2D0E1F6ED1ECD0F074
:103AF800EDD764A163AF26D0020177B315D07783E1
:103B0800170E0C6E040E0B6E77C20DF00DECCAF09A
:103B1800AE0E1E6E290E1F6ED1ECD0F0640E02019F
:103B2800976F000167810ED00C0E396E020E3A6E47
:103B3800010EBCEC58F08B0E1E6E2D0E1F6ED1ECD4
:103B4800D0F0ECD764B564B308D00B0E396E010E13
:103B58003A6EBCEC58F000016A8964B163BF92D731
:103B68000B0E396E020E3A6E010EBCEC58F088D777
:103B7800030198B15DD00201652B65510A0D400E15
:103B8800F324D96E040EF420DA6E4C0EDF6E655104
:103B98000A0D410EF324D96E040EF420DA6EDF68A4
:103BA80065510A0D420EF324D96E040EF420DA6E24
:103BB800DF6865510A0D430EF324D96E040EF42014
:103BC800DA6EDF6865510A0D440EF324D96E040ECF
:103BD800F420DA6EDF6865510A0D450EF324D96EBC
:103BE800040EF420DA6EDF6865510A0D460EF324E0
:103BF800D96E040EF420DA6EDF6865510A0D470E9F
:103C0800F324D96E040EF420DA6EDF6865510A0DCC
:103C1800480EF324D96E040EF420DA6EDF6865517D
:103C28000A0D490EF324D96E040EF420DA6EDF680B
:103C3800030197B55DD00201652B65510A0D400E51
:103C4800F324D96E040EF420DA6ED50EDF6E6551BA
:103C58000A0D410EF324D96E040EF420DA6EDF68E3
:103C680065510A0D420EF324D96E040EF420DA6E63
:103C7800DF6865510A0D430EF324D96E040EF42053
:103C8800DA6EDF6865510A0D440EF324D96E040E0E
:103C9800F420DA6EDF6865510A0D450EF324D96EFB
:103CA800040EF420DA6EDF6865510A0D460EF3241F
:103CB800D96E040EF420DA6EDF6865510A0D470EDE
:103CC800F324D96E040EF420DA6EDF6865510A0D0C
:103CD800480EF324D96E040EF420DA6EDF686551BD
:103CE8000A0D490EF324D96E040EF420DA6EDF684B
:103CF800D50E020164192CE1E3C031F1E2C030F1C4
:103D0800000E1E6E280E1F6E31C120F0216A30C1D0
:103D180022F0236AD1ECD0F0010131290BE03139CE
:103D28000F0B316F030E311903E000016A8902D0CD
:103D380000016A99010130290BE030390F0B306F0F
:103D4800030E301903E000016A8702D000016A9768
:103D5800050E0201641902E047EF23F00001E25169
:103D680007E17C0E1E6E300E1F6ED1ECD0F07BD0BA
:103D7800050EE21907E18C0E1E6E300E1F6ED1EC97
:103D8800D0F071D00A0EE21907E19C0E1E6E300EBB
:103D98001F6ED1ECD0F067D00F0EE21907E1AC0E20
:103DA8001E6E300E1F6ED1ECD0F05DD0110EE219F0
:103DB80007E1BC0E1E6E300E1F6ED1ECD0F053D052
:103DC800160EE21907E1CC0E1E6E300E1F6ED1ECF6
:103DD800D0F049D01B0EE21907E1DC0E1E6E300E42
:103DE8001F6ED1ECD0F03FD01C0EE21907E1EC0EAB
:103DF8001E6E300E1F6ED1ECD0F035D0220EE219B7
:103E080007E1FC0E1E6E300E1F6ED1ECD0F02BD0E9
:103E1800270EE21907E10C0E1E6E310E1F6ED1EC53
:103E2800D0F021D02D0EE21907E15C0E1E6E300E87
:103E38001F6ED1ECD0F017D0280EE21907E16C0EF6
:103E48001E6E300E1F6ED1ECD0F00DD0E2290BE0C3
:103E5800BE0E1E6E2C0E1F6EE2C020F0216AD1EC41
:103E6800D0F00001E2690001E35107E1740E1E6E13
:103E7800300E1F6ED1ECD0F034D2050EE31907E1F5
:103E8800840E1E6E300E1F6ED1ECD0F02AD20A0EB0
:103E9800E31907E1940E1E6E300E1F6ED1ECD0F0C0
:103EA80020D20F0EE31907E1A40E1E6E300E1F6E0E
:103EB800D1ECD0F016D2110EE31907E1B40E1E6E44
:103EC800300E1F6ED1ECD0F00CD2160EE31907E1BC
:103ED800C40E1E6E300E1F6ED1ECD0F002D21B0E37
:103EE800E31907E1D40E1E6E300E1F6ED1ECD0F030
:103EF800F8D11C0EE31907E1E40E1E6E300E1F6E9A
:103F0800D1ECD0F0EED1220EE31907E1F40E1E6ECB
:103F1800300E1F6ED1ECD0F0E4D1270EE31907E183
:103F2800040E1E6E310E1F6ED1ECD0F0DAD12D0EBC
:103F3800E31907E1540E1E6E300E1F6ED1ECD0F05F
:103F4800D0D1280EE31907E1640E1E6E300E1F6EE5
:103F5800D1ECD0F0C6D1E32901E1C3D1AC0E1E6E7D
:103F68002C0E1F6EE3C020F0216AD1ECD0F00001C6
:103F7800E369B7D10001E32901E176D30A0E010113
:103F8800476FDD0E4525D96EDA6A030EDA22000185
:103F9800E351D6ECC7F0DF6E0101452B2D0E000171
:103FA800E31910E10101456B55B40AD0000167B56A
:103FB80007D0016A026A010E2FECB7F00201796B93
:103FC8003AECCBF0040E0101451901E04DD3000194
:103FD8006D8138EC7DF00101456B46D30001E32982
:103FE80001E142D31E0E0101476F2D0E0001E319B6
:103FF80021E10101456B49073E0E1E6E290E1F6E19
:10400800D1ECD0F00E0E396E3A6A010EBCEC58F0C5
:10401800010E02015F6F800E5E6F016A026A010E77
:104028002FECB7F0010E02015D6F800E5C6F3AEC69
:10403800CBF01AD3050EE31916E1020E0101496F00
:10404800AD0E1E6E260E1F6ED1ECD0F00101456B31
:10405800A70E02015F6F5D6F200E016E010E026EEA
:104068002FECB7F001D30A0EE31918E1030E010192
:10407800496FB90E1E6E250E1F6ED1ECD0F00101EE
:10408800456B200E016E020E026E010E2FECB7F08A
:10409800E50E02015F6F810E5E6FE6D20F0EE31927
:1040A80014E1040E0101496F500E1E6E220E1F6EA0
:1040B800D1ECD0F00101456B200E016E040E026EAA
:1040C800010E2FECB7F0A70EE4D7010E016EA1EC9C
:1040D8009FF0CAD20001E32901E1C6D21E0E0101F8
:1040E800476FDD0E4525D96EDA6A030EDA22000124
:1040F800E351D6ECC7F0DF6E0101452B2D0E000110
:10410800E31919E10101456B49079E0E1E6E220E47
:104118001F6ED1ECD0F0A60E02015F6F820E5E6FAB
:10412800200E016E026A010E2FECB7F0A60E0201F6
:104138005D6F800E5C6F020E0101451916E10301E7
:10414800DD510A0DF350DE2500016E6F100E6E6111
:1041580006D00B0E016E010EA1EC9FF006D0010EE9
:10416800016EA1EC9FF00101456B030E0101451999
:1041780010E1030E0301DF6106D00C0E016E010E83
:10418800A1EC9FF006D0010E016EA1EC9FF0010199
:104198004507070E0101451901E066D200016D814E
:1041A80038EC7DF00A0E016E010EA1EC9FF013D7DA
:1041B8000001E32901E158D21E0E0101476F452B8A
:1041C8002D0E0001E3191FE10101456B496B7C0EBF
:1041D8001E6E230E1F6ED1ECD0F00E0E396E3A6AA9
:1041E800010EBCEC58F0010E02015F6F810E5E6F8C
:1041F800016A026A010E2FECB7F0010E02015D6F31
:10420800810E5C6F31D2020E0101451901E02CD2FA
:10421800456B496B7C0E1E6E230E1F6ED1ECD0F0E1
:104228000E0E396E3A6A010EBCEC58F0010E02010E
:104238005F6F810E5E6F016A026A010E2FECB7F0A4
:10424800010E02015D6F810E5C6F0A0E016E010E98
:10425800A1EC9FF009D20001E32901E105D21E0E6D
:104268000101476F2D0E0001E31918E10101456BAB
:10427800496B7C0E1E6E230E1F6ED1ECD0F0010E22
:1042880002015F6F810E5E6F016A026A010E2FECF8
:10429800B7F0010E02015D6F810E5C6F280E000100
:1042A800E31901E0E1D10101456B496B180E1E6E5F
:1042B8002A0E1F6ED1ECD0F0170E0C6E040E0B6E8A
:1042C8000D6A0DECCAF00201776B640E976F010E50
:1042D8005F6F810E5E6F016A026A010E2FECB7F004
:1042E8008CD70101495101E145D6010A01E176D691
:1042F800030A01E1EFD6010A01E15AD7070AABE048
:10430800B3D10001E22901E1BED10A0E0101466FD5
:10431800D40E4425D96EDA6A030EDA220001E2517E
:10432800D6ECC7F0DF6E0101442B2D0E0001E21917
:1043380010E10101446B55B20AD0000167B307D000
:10434800016A026A020E2FECB7F00201786B3AECB0
:10435800CBF0040E0101441901E095D100016C8FE6
:1043680038EC7DF00101446B8ED10001E22901E1B6
:104378008AD11E0E0101466F2D0E0001E21921E1BE
:104388000101446B4807550E1E6E290E1F6ED1ECB5
:10439800D0F00E0E396E3A6A010EBCEC58F0010EE0
:1043A80002015F6F800E5E6F016A026A020E2FECD7
:1043B800B7F0010E02015D6F800E5C6F3AECCBF036
:1043C80062D1050EE21917E1020E0101486FCB0E0A
:1043D8001E6E260E1F6ED1ECD0F00101446BA70EA5
:1043E80002015F6F5D6F200E016E010E026E020EFC
:1043F8002FECB7F048D10A0EE21917E1030E0101BC
:10440800486FD90E1E6E250E1F6ED1ECD0F001013B
:10441800446B200E016E020E026E2FECB7F0E50E13
:1044280002015D6F810E5C6F2ED10F0EE21914E14F
:10443800040E0101486F770E1E6E220E1F6ED1EC1E
:10444800D0F00101446B200E016E040E026E020EC4
:104458002FECB7F0A70EE4D7010E016E020EA1EC07
:104468009FF011D10001E22901E10DD11E0E0101D9
:10447800466FD40E4425D96EDA6A030EDA2200019B
:10448800E251D6ECC7F0DF6E0101442B2D0E00017E
:10449800E21919E10101446B4807C40E1E6E220E91
:1044A8001F6ED1ECD0F0A60E02015F6F800E5E6F1A
:1044B800200E016E026A020E2FECB7F0A60E020162
:1044C8005D6F820E5C6F020E0101441917E1030152
:1044D800D4510A0DF350D52500016F6F100E6F618E
:1044E80006D00B0E016E020EA1EC9FF007D0010E54
:1044F800016E020EA1EC9FF00101446B030E010155
:10450800441911E1030E0301D66106D00C0E016EA9
:10451800020EA1EC9FF007D0010E016E020EA1EC75
:104528009FF001014407070E0101441901E0ABD0D7
:1045380000016C8F38EC7DF00A0E016E020EA1ECC2
:104548009FF010D70001E22901E19DD01E0E010164
:10455800466F442B2D0E0001E2191BE10101446B4B
:10456800486BA00E1E6E230E1F6ED1ECD0F00E0EFF
:10457800396E3A6A010EBCEC58F0010E02015F6F09
:10458800810E5E6F016A026A020E2FECB7F0010E0F
:1045980047D7020E0101441976E1446B486BA00E1F
:1045A8001E6E230E1F6ED1ECD0F00E0E396E3A6AD5
:1045B800010EBCEC58F0010E02015F6F810E5E6FB8
:1045C800016A026A010E2FECB7F0010E02015D6F5D
:1045D800810E5C6F0A0E016E020EA1EC9FF053D0A3
:1045E8000001E22950E01E0E0101466F2D0E000168
:1045F800E21918E10101446B486BA00E1E6E230EF0
:104608001F6ED1ECD0F0010E02015F6F810E5E6F5C
:10461800016A026A020E2FECB7F0010E02015D6F0B
:10462800810E5C6F280E0001E2192DE10101446B37
:10463800486B180E1E6E2A0E1F6ED1ECD0F0170EA6
:104648000C6E040E0B6E0D6A0DECCAF00201776B4E
:10465800640E976F010E5F6F810E5E6F016A026ACA
:10466800020E2FECB7F093D70101485101E149D66A
:10467800010A01E17AD6030A01E1F4D6010A01E14F
:1046880061D7070AADE0020165510AE1050E646FC2
:104698005EC263F25FC262F25CC261F25DC260F246
:1046A8006551D8B412004AC464F24BC463F24CC4D6
:1046B80062F24DC461F24EC460F24FC4E8F050C4D7
:1046C800E7F051C4E6F052C4E5F053C4E4F06507DE
:1046D8006551D8B412000001736B32D0746B090EA7
:1046E800746501D02CD073510A0D400E4D6E040E26
:1046F8004E6E140E4D26000E4E22F3504D26F450E9
:104708004E2274514D24D96E000E4E20DA6E73512C
:104718000A0D400E4F6E040E506E0A0E4F26000E04
:104728005022F3504F26F450502274514F24E16E1A
:10473800000E5020E26EDFCFE7FF742BD0D7732B2B
:10474800020165510001735DC9E312000C6A0D6A2C
:10475800010135510C26000E0D220C500B6E0A6A11
:104768000C6A0B500D6E34510C26000E0D220201FE
:10477800A16BA06B9F6B0D5003E1090E0C5C0FE35E
:104788000D500DE1290E0C5C0AE2360EACEC2AF055
:1047980034EC2BF0F80EF1EC2AF087ECD2F00D5047
:1047A80003E1290E0C5C0FE30D500DE1490E0C5C82
:1047B8000AE2370EACEC2AF034EC2BF0D80EF1EC10
:1047C8002AF087ECD2F0490E0C180D1007E1360ECE
:1047D800ACEC2AF0E9EC2AF03FEC2BF04A0E0C186E
:1047E8000D1006E1360E94EC2AF0360E3FEC2BF055
:1047F8004B0E0C180D1009E1370E0101A7EC2AF039
:10480800350EA06F390E3FEC2BF04E0E0C180D1024
:1048180007E1360EACEC2AF0A06F300E1EEC2BF040
:104828004F0E0C180D1006E1360EACEC2AF0300EC7
:1048380005EC2BF0500E0C180D1007E1360EACEC01
:104848002AF03CEC2BF01EEC2BF0510E0C180D103E
:1048580006E1B7EC2AF0A2EC2AF09B6F9A6F520E91
:104868000C180D1007E1370EACEC2AF0A06F300ED3
:104878001EEC2BF0530E0C180D1006E1370EACECA5
:104888002AF0300E05EC2BF0540E0C180D1007E131
:10489800370EACEC2AF03CEC2BF01EEC2BF0550E4E
:1048A8000C180D1006E1BBEC2AF0A2EC2AF09B6F65
:1048B8009A6F0D5003E1560E0C5C0FE30D500DE19D
:1048C800760E0C5C0AE2360E8EEC2AF0F7EC2AF033
:1048D800AB0EF1EC2AF087ECD2F00D5003E1760E26
:1048E8000C5C0FE30D500DE1960E0C5C0AE2370EDE
:1048F8008EEC2AF0F7EC2AF08B0EF1EC2AF087EC1C
:10490800D2F0980E0C180D1008E1360E0101A7EC34
:104918002AF0E9EC2AF0BFEC2AF00D5003E1990ED9
:104928000C5C0FE30D500DE1BB0E0C5C0AE2370E78
:1049380094EC2AF0310E9F6F680EF1EC2AF087ECA8
:10494800D2F0BB0E0C180D1006E1370E94EC2AF0CD
:10495800320E48EC2BF0BC0E0C180D1008E1370E87
:1049680094EC2AF0310E9F6F340E62EC2BF0BD0EE2
:104978000C180D1007E1370E94EC2AF066EC2BF0BA
:1049880044EC2BF0BE0E0C180D1009E1370E010196
:10499800A7EC2AF0350EA06F360EBFEC2AF0BF0E3A
:1049A8000C180D1005E1370E94EC2AF01EEC2BF0D4
:1049B8000D5003E1C00E0C5C0FE30D500DE1E20E4B
:1049C8000C5C0AE2360E94EC2AF0310E9F6F410E11
:1049D800F1EC2AF087ECD2F0E20E0C180D1006E18B
:1049E800360E94EC2AF0320E48EC2BF0E30E0C183D
:1049F8000D1007E1360E94EC2AF066EC2BF062EC11
:104A08002BF0E40E0C180D1008E1360E94EC2AF089
:104A1800310E9F6F340E44EC2BF0E50E0C180D1080
:104A280006E1360E94EC2AF0350EBFEC2AF0E60EBD
:104A38000C180D1005E1360E94EC2AF01EEC2BF044
:104A4800E70E0C180D1008E1360E8EEC2AF0300E29
:104A5800A06F320EBFEC2AF0E80E0C180D1008E11A
:104A6800360E8EEC2AF0300EA06F310EBFEC2AF015
:104A7800E90E0C180D1007E1360E8EEC2AF0E9EC61
:104A88002AF0BFEC2AF0EA0E0C180D1007E1360EDA
:104A98008EEC2AF0DAEC2AF0BFEC2AF0EC0E0C18B7
:104AA8000D1007E1360E8EEC2AF031EC2BF0BFEC3E
:104AB8002AF0EF0E0C180D1008E1370E8EEC2AF0D4
:104AC800300EA06F320EBFEC2AF0F00E0C180D104D
:104AD80008E1370E8EEC2AF0300EA06F310EBFECD5
:104AE8002AF0F10E0C180D1007E1370E8EEC2AF0A3
:104AF800E9EC2AF0BFEC2AF0F20E0C180D1007E1D1
:104B0800370E8EEC2AF0DAEC2AF0BFEC2AF0F40E1D
:104B18000C180D1007E1370E8EEC2AF031EC2BF053
:104B2800BFEC2AF0F70E0C180D1007E1360E8EECCC
:104B38002AF039EC2BF0BFEC2AF0FE0E0C180D1001
:104B480007E114EC2BF0B2EC2AF0320EBFEC2AF09D
:104B58000C280D1007E114EC2BF0B2EC2AF0310E02
:104B6800BFEC2AF0030E0C180AE10D0408E1360E1A
:104B7800ACEC2AF0330EA06F390EBFEC2AF02C0EE5
:104B88000C5C010E0D580DE373EC2BF00AE2370EA6
:104B98008EEC2AF07DEC2BF0D50EFCEC2AF087EC9D
:104BA800D2F073EC2BF00DE36EEC2BF00AE2370E2B
:104BB8008EEC2AF07DEC2BF0B50EFCEC2AF087EC9D
:104BC800D2F06EEC2BF00DE369EC2BF00AE2360E16
:104BD8008EEC2AF0F7EC2AF0950EFCEC2AF087EC24
:104BE800D2F069EC2BF00FE3AC0E0C5C010E0D5803
:104BF8000AE2360E8EEC2AF0F7EC2AF0750EFCEC81
:104C08002AF087ECD2F0AD0E0C1809E10D0407E18B
:104C180014EC2BF0E4EC2AF0370EBFEC2AF0AC0EC3
:104C28000C1809E10D0407E114EC2BF0E4EC2AF070
:104C3800380EBFEC2AF0B00E0C5C010E0D580EE3D6
:104C4800D00E0C5C010E0D5809E210EC2BF0C4ECF0
:104C58002AF0510EFCEC2AF087ECD2F0630E0C1807
:104C68000AE1020E0D1807E1370EACEC2AF02EEC23
:104C78002BF0BFEC2AF0640E0C180AE1020E0D1896
:104C880007E1360EACEC2AF02EEC2BF0BFEC2AF044
:104C98006A0E0C180AE1020E0D1807E1370E8EECA9
:104CA8002AF039EC2BF0BFEC2AF0980E0C1809E129
:104CB800020E0D1806E1370E94EC2AF0380EBFEC00
:104CC8002AF09A0E0C1808E1020E0D1805E1370EAD
:104CD80094EC2AF01EEC2BF0E90E0C180AE1020EF7
:104CE8000D1807E1370E8EEC2AF0D5EC2AF0310EBC
:104CF8009A6FEA0E0C180AE1020E0D1807E1370E3A
:104D08008EEC2AF0D5EC2AF0320E9A6FF30E0C18BE
:104D180009E1020E0D1806E1370EFCDBD5EC2AF08E
:104D2800330E9A6FEC0E0C1809E1020E0D1806E10D
:104D3800370EF0DBD5EC2AF0340E9A6FED0E0C1816
:104D480009E1020E0D1806E1370EE4DBD5EC2AF076
:104D5800350E9A6FEE0E0C1809E1020E0D1806E1D9
:104D6800370ED8DBD5EC2AF0360E9A6FEF0E0C18FA
:104D780009E1020E0D1806E1370ECCDBD5EC2AF05E
:104D8800370E9A6FF00E0C1809E1020E0D1806E1A5
:104D9800370EC0DBD5EC2AF0380E9A6FF10E0C18DE
:104DA80008E1020E0D1805E1360EB4DBFADB310E10
:104DB8009A6FF20E0C1808E1020E0D1805E1360E76
:104DC800A9DBEFDB320E9A6FF30E0C1808E1020E26
:104DD8000D1805E1360E9EDBE4DB330E9A6FF40EF8
:104DE8000C1808E1020E0D1805E1360E93DBD9DB2D
:104DF800340E9A6FF50E0C1808E1020E0D1805E135
:104E0800360E88DBCEDB350E9A6FF60E0C1808E1ED
:104E1800020E0D1805E1360E7DDBC3DB360E9A6FE8
:104E2800F70E0C1808E1020E0D1805E1360E72DBBC
:104E3800B8DB370E9A6FF80E0C1808E1020E0D1841
:104E480005E1360E67DBADDB380E9A6FF90E0C18EC
:104E580008E1020E0D1805E1370E5CDBA2DB390E06
:104E68009A6FFA0E0C1808E1020E0D1805E1370EBC
:104E780051DB92DB300E9A6FFB0E0C1807E1020E25
:104E88000D1804E1370E46DB87DB9A6FFC0E0C1811
:104E980008E1020E0D1805E1370E3CDB7DDB320E12
:104EA8009A6FFD0E0C1808E1020E0D1805E1370E79
:104EB80031DB72DB330E9A6FFE0E0C1808E1020E1E
:104EC8000D1805E1370E26DB67DB340E9A6F0C28C8
:104ED80008E1020E0D1805E1360E1CDB62DB390E07
:104EE8009A6F030E0D180C1005E1360E13DB54DB18
:104EF800300E9A6F0C0407E1030E0D1804E1360E0C
:104F080009DB4ADB9A6F020E0C1808E1030E0D1834
:104F180005E1360EFFDA40DB320E9A6F030E0C18ED
:104F280008E1030E0D1805E1360EF4DA35DB330E11
:104F38009A6F040E0C1808E1030E0D1805E1360EE1
:104F4800E9DA2ADB340E9A6F050E0C1808E1030E15
:104F58000D1805E1370EDEDA1FDB370E9A6F060EE5
:104F68000C1808E1030E0D1805E1360ED3DA14DB30
:104F7800370E9A6F070E0C1808E1030E0D1805E19D
:104F8800370EC8DA09DB380E9A6F080E0C1808E1DC
:104F9800030E0D1805E1360EBDDAFEDA380E9A6FEB
:104FA800090E0C1808E1030E0D1805E1370EB2DAE8
:104FB800F3DA390E9A6F0A0E0C1808E1030E0D1871
:104FC80005E1360EA7DAE8DA390E9A6F0B0E0C18DF
:104FD80008E1030E0D1805E1370E9CDAD8DA300E19
:104FE8009A6F0C0E0C1808E1030E0D1805E1360E29
:104FF80091DACDDA300E9A6F0D0E0C1808E1030E17
:105008000D1805E1370E86DAC2DA310E9A6F0E0EE8
:105018000C1808E1030E0D1805E1360E7BDAB7DA35
:10502800310E9A6F0F0E0C1807E1030E0D1804E1EC
:10503800370E70DAACDA9A6F100E0C1807E1030E0F
:105048000D1804E1360E66DAA2DA9A6F110E0C1802
:1050580008E1030E0D1805E1370E5CDA98DA330E15
:105068009A6F110E0C1808E1030E0D1805E1360EA3
:1050780051DA8DDA330E9A6F130E0C1808E1030E0D
:105088000D1805E1370E46DA82DA340E9A6F140EDF
:105098000C1808E1030E0D1805E1360E3BDA77DA35
:1050A800340E9A6F150E0C1808E1030E0D1805E161
:1050B800370E30DA71DA350E9A6F160E0C1808E1D1
:1050C800030E0D1805E1360E25DA66DA350E9A6FED
:1050D800170E0C1808E1030E0D1805E1370E1ADA41
:1050E8005BDA360E9A6F180E0C1808E1030E0D18CD
:1050F80005E1360E0FDA50DA360E9A6F190E0C18D3
:1051080008E1030E0D1805E1370E04DA40DA350E12
:105118009A6F1A0E0C1808E1030E0D1805E1360EE9
:10512800F9D935DA350E9A6F1B0E0C1808E1030E03
:105138000D1805E1370EEED92ADA360E9A6F1F0ED2
:105148000C1808E1030E0D1805E1360EE3D91FDA35
:10515800360E9A6F1C0E0C1808E1030E0D1805E1A7
:10516800370ED8D914DA370E9A6F200E0C1808E1CA
:10517800030E0D1805E1360ECDD909DA370E9A6FF0
:105188001D0E0C1808E1030E0D1805E1370EC2D9E3
:10519800FED9380E9A6F210E0C1808E1030E0D186F
:1051A80005E1360EB7D9F3D9380E9A6F1E0E0C18D2
:1051B80008E1030E0D1805E1370EACD9E8D9390E10
:1051C8009A6F220E0C1808E1030E0D1805E1360E31
:1051D800A1D9DDD9390E9A6F350E0C5C030E0D5826
:1051E8000CE367DA0AE2370EB3D9340EA06F350E36
:1051F8009F6FD40E19DA87ECD2F05BDA0FE3410E19
:105208000C5C030E0D580AE2360EA2D9340EA06FBC
:10521800350E9F6FCE0E08DA87ECD2F0410E0C18CF
:1052280008E1030E0D1805E1370E92D9C2D9370EE1
:105238009A6F420E0C1808E1030E0D1805E1360EA0
:1052480087D9B7D9370E9A6F430E0C1808E1030EA9
:105258000D1805E1370E7CD9ACD9380E9A6F440E7B
:105268000C1808E1030E0D1805E1360E71D9A1D905
:10527800380E9A6F450E0C1808E1030E0D1805E15B
:10528800370E66D996D9390E9A6F460E0C1808E172
:10529800030E0D1805E1360E5BD98BD9390E9A6FBE
:1052A800510E0C1808E1030E0D1805E1370E50D900
:1052B80080D9360E9A6F520E0C1808E1030E0D189D
:1052C80005E1360E45D975D9360E9A6FB50E0C180C
:1052D80007E1030E0D1804E1370E1CD9300E91D9E1
:1052E800B60E0C1807E1030E0D1804E1360E12D99C
:1052F800300E87D9040E0D5C09E3D6D907E233D9FD
:10530800020116D9210E90D987ECD2F0CDD90CE341
:10531800EBD90AE22CD902010BD90C28086EFC0E35
:105328000D20096E87ECD2F0DFD909E3B3D907E283
:10533800360EF0D858D9E10E87D987ECD2F0AAD921
:105348000CE3800E0C5C040E0D5807E2370EE2D811
:105358004AD9C10E79D987ECD2F0050E0D180C1078
:1053680005E1370EDDD834D9350E9A6F0C0408E103
:10537800050E0D1805E1370ED3D82AD9360E9A6FC7
:10538800020E0C1808E1050E0D1805E1370EC8D8F5
:105398001FD9370E9A6F030E0C1808E1050E0D1869
:1053A80005E1370EBDD814D9380E9A6F040E0C18C3
:1053B80008E1050E0D1805E1370EB2D809D9390EE6
:1053C8009A6F050E0C5C050E0D580DE33A0E0C5C39
:1053D800050E0D5808E2370EA3D8310E9F6F260E22
:1053E80033D987ECD2F03A0E0C1808E1050E0D18E7
:1053F80005E1360E95D8ECD8350E9A6F3B0E0C1891
:1054080008E1050E0D1805E1360E8AD8E1D8360EEA
:105418009A6F3C0E0C1808E1050E0D1805E1360EC2
:105428007FD8D6D8370E9A6F3D0E0C1808E1050EB6
:105438000D1805E1360E74D8CBD8380E9A6F3E0E8B
:105448000C1808E1050E0D1805E1360E69D8C0D80C
:10545800390E9A6F3F0E0C5C050E0D5811E3740E51
:105468000C5C050E0D580CE2360E5AD8310E9F6FA3
:10547800EC0E0C24086EFA0E0D20096E87ECD2F0A3
:10548800400E0C5C140E0D5809E309D907E2370EDB
:1054980041D8A9D8E10ED2D887ECD2F000D909E3D7
:1054A8002DD907E2360E36D89ED8C10EC7D887EC5C
:1054B800D2F024D90BE3A00E0C5C140E0D5806E2B2
:1054C800ABD85ED8A10EBAD887ECD2F0F10E0C1882
:1054D80009E11B0E0D1806E1370E1CD8300EA06F1F
:1054E800350E49D8770E0C1808E1770E0D1805E12E
:1054F800360E84D802EC9EF089D8780E0C1809E193
:10550800770E0D18D8A41200370E78D802EC9EF04A
:105518007DD812000101586F330E0201A16F330CC0
:105528000101586F340E0201A16F300EA06F300CCC
:10553800A16F330EA06F300E9F6F300C0201A16F68
:10554800A06F9F6F300C586F340E0201A16F340C9E
:105558000101586F310E0201A16F310C0201A16FD8
:10556800300EA06F300C360E0101586F310C370E1B
:105578000101586F310C9F6F300E9B6F9A6F300C82
:105588000201A16F370EA06F300E9F6F300CA06F15
:105598009F6F320E9B6F320CA06F9F6F310E9B6F07
:1055A800310CA06F9F6F300E9B6F300C370EA06FC1
:1055B800330C340EA06F350E9F6F310E9B6F310C7C
:1055C8000201A16F320EA06F320C320EA06F310CA7
:1055D800310E9F6F330E9B6F330C0C24086EFF0E39
:1055E8000D20096E1200380EA06F330E9F6F330C1A
:1055F8000C24086EFE0E0D20096E12000101586F72
:10560800380CA06F9F6F9B6F9A6F12009F6F320EBE
:105618009B6F300E9A6F300C360E0101586F350CA7
:10562800360E0101586F360C0C24086EFC0E0D2046
:10563800096E12009F6F9B6F9A6F12000C24086E00
:10564800EB0E0D20096E12000C24086EFB0E0D20C7
:10565800096E1200340EA06F330C350EA06F310C9A
:10566800330EA06F300E9F6F300C350EA06F340CC8
:10567800320EA06F300C9F6F300E9B6F9A6F300CFC
:105688009B6F320E9A6F320C9F6F340E9B6F300EE9
:105698009A6F300C600E0C5C040E0D581200600EF0
:1056A8000C5C140E0D581200200E0C5C040E0D58E4
:1056B80012003B0E0C5C030E0D5812009B6F310E4E
:1056C8009A6F310C310E9F6F340C8C0E0C5C010EEE
:1056D8000D5812006C0E0C5C010E0D5812004C0E89
:1056E8000C5C010E0D581200400E0C5C040E0D5897
:1056F8001200380EA06F340E9F6F340C800E0C5CB5
:10570800140E0D5812000501FB6F02017D1D0501E5
:10571800FC6FFB0501E08AD302018C51010B0501E6
:10572800FD6FFDA162D0FD51FC1539E055B455A2BD
:105738005CD054B403D0000169AF17D002018505CD
:1057480006E0020E851903E0030E85194EE1010EED
:105758000501F96FFA6FADEC32F0010E0501F96F32
:10576800FA6F020EADEC32F040D00201850509E077
:10577800020E851906E0030E851903E0040E85194B
:1057880034E1010E0501F96FFA6FADEC32F0010E4C
:105798000501F96FFA6F020EADEC32F026D0FD511B
:1057A80002015B1522E054A40FD0850506E0020E25
:1057B800851903E0030E851918E1010E0501F96F3B
:1057C800FA6FADEC32F011D0850509E0020E8519AB
:1057D80006E0030E851903E0040E851906E1010EA3
:1057E8000501F96FFA6FADEC32F002018C51020B32
:1057F8000501FD6FFDA368D0FD51FC153DE055B4D2
:1058080055A262D054B403D0000169AF19D0020187
:10581800840506E0020E841903E0030E841954E19E
:10582800010E0501F96F020EFA6F010EADEC32F0B0
:10583800010E0501F96F020EFA6FADEC32F044D09B
:105848000201840509E0020E841906E0030E84199A
:1058580003E0040E841938E1010E0501F96F020E08
:10586800FA6F010EADEC32F0010E0501F96F020E70
:10587800FA6FADEC32F028D0FD5102015B1524E03F
:1058880054A40FD0840506E0020E841903E0030E29
:1058980084191AE1010E0501F96FFA6FADEC32F0C7
:1058A80013D0840509E0020E841906E0030E84195A
:1058B80003E0040E841908E1010E0501F96F020ED8
:1058C800FA6F010EADEC32F002018C51040B0501A8
:1058D800FD6FFDA56CD0FD51FC153FE055B455A2F8
:1058E80066D054B403D0000169AF1AD00201830511
:1058F80006E0020E831903E0030E831958E1010E36
:105908000501F96F030EFA6F010EADEC32F0010ECE
:105918000501F96F030EFA6F020EADEC32F047D0B5
:105928000201830509E0020E831906E0030E8319BC
:1059380003E0040E83193BE1010E0501F96F030E24
:10594800FA6F010EADEC32F0010E0501F96F030E8E
:10595800FA6F020EADEC32F02AD0FD5102015B1550
:1059680026E054A411D0830506E0020E831903E053
:10597800030E83191CE1010E0501F96F030EFA6F7E
:10598800010EADEC32F013D0830509E0020E831945
:1059980006E0030E831903E0040E831908E1010EE3
:1059A8000501F96F030EFA6F010EADEC32F002013A
:1059B8008C51080B0501FD6FFDA76CD0FD51FC153E
:1059C8003FE055B455A266D054B403D0000169AF86
:1059D8001AD00201820506E0020E821903E0030EC6
:1059E800821958E1010E0501F96F040EFA6F010ED4
:1059F800ADEC32F0010E0501F96F040EFA6F020EDC
:105A0800ADEC32F047D00201820509E0020E82199E
:105A180006E0030E821903E0040E82193BE1010E31
:105A28000501F96F040EFA6F010EADEC32F0010EAC
:105A38000501F96F040EFA6F020EADEC32F02AD0B0
:105A4800FD5102015B1526E054A411D0820506E041
:105A5800020E821903E0030E82191CE1010E0501F2
:105A6800F96F040EFA6F010EADEC32F013D0820517
:105A780009E0020E821906E0030E821903E0040E03
:105A8800821908E1010E0501F96F040EFA6F010E83
:105A9800ADEC32F002018C51100B0501FD6FFDA930
:105AA8006CD0FD51FC153FE055B455A266D054B4F6
:105AB80003D0000169AF1AD00201810506E0020E89
:105AC800811903E0030E811958E1010E0501F96FF0
:105AD800050EFA6F010EADEC32F0010E0501F96FFB
:105AE800050EFA6F020EADEC32F047D002018105C7
:105AF80009E0020E811906E0030E811903E0040E85
:105B080081193BE1010E0501F96F050EFA6F010ECF
:105B1800ADEC32F0010E0501F96F050EFA6F020EB9
:105B2800ADEC32F02AD0FD5102015B1526E054A4F9
:105B380011D0810506E0020E811903E0030E8119D8
:105B48001CE1010E0501F96F050EFA6F010EADECAF
:105B580032F013D0810509E0020E811906E0030E28
:105B6800811903E0040E811908E1010E0501F96F9E
:105B7800050EFA6F010EADEC32F002018C51200BCC
:105B88000501FD6FFDAB6CD0FD51FC153FE055B430
:105B980055A266D054B403D0000169AF1AD00201EF
:105BA800800506E0020E801903E0030E801958E113
:105BB800010E0501F96F060EFA6F010EADEC32F019
:105BC800010E0501F96F060EFA6F020EADEC32F008
:105BD80047D00201800509E0020E801906E0030E95
:105BE800801903E0040E80193BE1010E0501F96FED
:105BF800060EFA6F010EADEC32F0010E0501F96FD9
:105C0800060EFA6F020EADEC32F02AD0FD510201F9
:105C18005B1526E054A411D0800506E0020E801919
:105C280003E0030E80191CE1010E0501F96F060E51
:105C3800FA6F010EADEC32F013D0800509E0020EC8
:105C4800801906E0030E801903E0040E801908E1AC
:105C5800010E0501F96F060EFA6F010EADEC32F078
:105C680002018C51400B0501FD6FFDAD6CD0FD515B
:105C7800FC153FE055B455A266D054B403D00001DA
:105C880069AF1AD002017F0506E0020E7F1903E012
:105C9800030E7F1958E1010E0501F96F070EFA6F1F
:105CA800010EADEC32F0010E0501F96F070EFA6F27
:105CB800020EADEC32F047D002017F0509E0020E7A
:105CC8007F1906E0030E7F1903E0040E7F193BE1FC
:105CD800010E0501F96F070EFA6F010EADEC32F0F7
:105CE800010E0501F96F070EFA6F020EADEC32F0E6
:105CF8002AD0FD5102015B1526E054A411D07F057E
:105D080006E0020E7F1903E0030E7F191CE1010E65
:105D18000501F96F070EFA6F010EADEC32F013D0E2
:105D28007F0509E0020E7F1906E0030E7F1903E0E4
:105D3800040E7F1908E1010E0501F96F070EFA6FCD
:105D4800010EADEC32F002018C51800B0501FD6FA4
:105D5800FDAF6CD0FD51FC153FE055B455A266D09F
:105D680054B403D0000169AF1AD002017E0506E0E1
:105D7800020E7E1903E0030E7E1958E1010E05019B
:105D8800F96F080EFA6F010EADEC32F0010E050145
:105D9800F96F080EFA6F020EADEC32F047D002012F
:105DA8007E0509E0020E7E1906E0030E7E1903E067
:105DB800040E7E193BE1010E0501F96F080EFA6F1A
:105DC800010EADEC32F0010E0501F96F080EFA6F05
:105DD800020EADEC32F02AD0FD5102015B1526E02F
:105DE80054A411D07E0506E0020E7E1903E0030ECE
:105DF8007E191CE1010E0501F96F080EFA6F010EFC
:105E0800ADEC32F013D07E0509E0020E7E1906E0F3
:105E1800030E7E1903E0040E7E1908E1010E050148
:105E2800F96F080EFA6F010EADEC32F0020E0501A3
:105E3800FB19D8A4120002018C51010B0501FD6F5A
:105E4800FDA167D0FD51FC1539E055B455A261D0CC
:105E580054B403D0000169AF17D00201850506E0EC
:105E6800020E851903E0030E851953E1010E0501A1
:105E7800F96FFA6FADEC32F0010E0501F96FFA6FA8
:105E8800020EADEC32F045D00201850509E0020EA4
:105E9800851906E0030E851903E0040E851939E11A
:105EA800010E0501F96FFA6FADEC32F0010E050134
:105EB800F96FFA6F020EADEC32F02BD0FD510201F2
:105EC8005A1527E0000169AF11D00201850506E0E7
:105ED800020E851903E0030E85191BE1010E050169
:105EE800F96FFA6F020EADEC32F013D0020185059E
:105EF80009E0020E851906E0030E851903E0040E79
:105F0800851907E1010E0501F96FFA6F020EADEC74
:105F180032F002018C51020B0501FD6FFDA36BD01D
:105F2800FD51FC153DE055B455A265D054B403D0DD
:105F3800000169AF19D00201840506E0020E841938
:105F480003E0030E841957E1010E0501F96F020EF3
:105F5800FA6F010EADEC32F0010E0501F96F020E79
:105F6800FA6FADEC32F047D00201840509E0020E69
:105F7800841906E0030E841903E0040E84193BE13A
:105F8800010E0501F96F020EFA6F010EADEC32F049
:105F9800010E0501F96F020EFA6FADEC32F02BD04D
:105FA800FD5102015A1527E0000169AF11D0020125
:105FB800840506E0020E841903E0030E84191BE130
:105FC800010E0501F96FFA6F020EADEC32F013D035
:105FD8000201840509E0020E841906E0030E841903
:105FE80003E0040E841907E1010E0501F96F020EA2
:105FF800FA6FADEC32F002018C51040B0501FD6F14
:10600800FDA56FD0FD51FC153FE055B455A269D0F0
:1060180054B403D0000169AF1AD00201830506E029
:10602800020E831903E0030E83195BE1010E0501DB
:10603800F96F030EFA6F010EADEC32F0010E050197
:10604800F96F030EFA6F020EADEC32F04AD002017E
:10605800830509E0020E831906E0030E831903E0A5
:10606800040E83193EE1010E0501F96F030EFA6F64
:10607800010EADEC32F0010E0501F96F030EFA6F57
:10608800020EADEC32F02DD0FD5102015A1529E077
:10609800000169AF12D00201830506E0020E8319E0
:1060A80003E0030E83191DE1010E0501F96F030ECC
:1060B800FA6F020EADEC32F014D00201830509E04C
:1060C800020E831906E0030E831903E0040E8319F8
:1060D80008E1010E0501F96F030EFA6F020EADEC2F
:1060E80032F002018C51080B0501FD6FFDA76FD03E
:1060F800FD51FC153FE055B455A269D054B403D006
:10610800000169AF1AD00201820506E0020E821969
:1061180003E0030E82195BE1010E0501F96F040E1D
:10612800FA6F010EADEC32F0010E0501F96F040EA5
:10613800FA6F020EADEC32F04AD00201820509E096
:10614800020E821906E0030E821903E0040E82197A
:106158003EE1010E0501F96F040EFA6F010EADEC78
:1061680032F0010E0501F96F040EFA6F020EADEC64
:1061780032F02DD0FD5102015A1529E0000169AF16
:1061880012D00201820506E0020E821903E0030E16
:1061980082191DE1010E0501F96F040EFA6F020E56
:1061A800ADEC32F014D00201820509E0020E82192A
:1061B80006E0030E821903E0040E821908E1010EBD
:1061C8000501F96F040EFA6F020EADEC32F0020110
:1061D8008C51100B0501FD6FFDA96FD0FD51FC1509
:1061E8003FE055B455A269D054B403D0000169AF5B
:1061F8001AD00201810506E0020E811903E0030EA0
:1062080081195BE1010E0501F96F050EFA6F010EA8
:10621800ADEC32F0010E0501F96F050EFA6F020EB2
:10622800ADEC32F04AD00201810509E0020E811975
:1062380006E0030E811903E0040E81193EE1010E08
:106248000501F96F050EFA6F010EADEC32F0010E83
:106258000501F96F050EFA6F020EADEC32F02DD084
:10626800FD5102015A1529E0000169AF12D002015F
:10627800810506E0020E811903E0030E81191DE174
:10628800010E0501F96F050EFA6F020EADEC32F042
:1062980014D00201810509E0020E811906E0030EFF
:1062A800811903E0040E811908E1010E0501F96F57
:1062B800050EFA6F020EADEC32F002018C51200B84
:1062C8000501FD6FFDAB6FD0FD51FC153FE055B4E6
:1062D80055A269D054B403D0000169AF1AD00201A5
:1062E800800506E0020E801903E0030E80195BE1C9
:1062F800010E0501F96F060EFA6F010EADEC32F0D2
:10630800010E0501F96F060EFA6F020EADEC32F0C0
:106318004AD00201800509E0020E801906E0030E4A
:10632800801903E0040E80193EE1010E0501F96FA2
:10633800060EFA6F010EADEC32F0010E0501F96F91
:10634800060EFA6F020EADEC32F02DD0FD510201AF
:106358005A1529E0000169AF12D00201800506E054
:10636800020E801903E0030E80191DE1010E0501DC
:10637800F96F060EFA6F020EADEC32F014D002017E
:10638800800509E0020E801906E0030E801903E07B
:10639800040E801908E1010E0501F96F060EFA6F67
:1063A800020EADEC32F002018C51400B0501FD6F7D
:1063B800FDAD6FD0FD51FC153FE055B455A269D035
:1063C80054B403D0000169AF1AD002017F0506E07A
:1063D800020E7F1903E0030E7F195BE1010E050130
:1063E800F96F070EFA6F010EADEC32F0010E0501E0
:1063F800F96F070EFA6F020EADEC32F04AD00201C7
:106408007F0509E0020E7F1906E0030E7F1903E0FD
:10641800040E7F193EE1010E0501F96F070EFA6FB0
:10642800010EADEC32F0010E0501F96F070EFA6F9F
:10643800020EADEC32F02DD0FD5102015A1529E0C3
:10644800000169AF12D002017F0506E0020E7F1934
:1064580003E0030E7F191DE1010E0501F96F070E18
:10646800FA6F020EADEC32F014D002017F0509E09C
:10647800020E7F1906E0030E7F1903E0040E7F1950
:1064880008E1010E0501F96F070EFA6F020EADEC77
:1064980032F002018C51800B0501FD6FFDAF120037
:1064A800FD51FC1531E055B455A2120054B403D087
:1064B800000169AF13D002017E0507E0020E7E19C4
:1064C80004E0030E7E19D8A41200010E0501F96F2D
:1064D800080EFA6F010EADEC32F033D002017E05E2
:1064E8000AE0020E7E1907E0030E7E1904E0040E8E
:1064F8007E19D8A41200010E0501F96F080EFA6F73
:10650800010EADEC32F01DD0FD5102015A15D8B480
:106518001200000169AF08D002017E0512E0020EE8
:106528007E190FE0030E0AD002017E050AE0020E72
:106538007E1907E0030E7E1904E0040E7E19D8A424
:106548001200010E0501F96F080EFA6F020EADEF89
:1065580032F00601486F480501E19AD3C2D30F0E05
:10656800E86F240EE96FFAC5EAF5EB6B1DECD0F085
:10657800538E53BC8A8C020186513C0DF3CF6FF3C6
:10658800F4CF70F300016785310E0201A16F330E5D
:10659800A06F300E9F6F9E6F310E9D6F300E9C6FF7
:1065A8009B6F0501FA51300F02019A6F060E050123
:1065B800D66F000E19ECABF018D00201798127D004
:1065C8000201798324D00201798521D002017987DB
:1065D8001ED0020179891BD00201798B18D00201E3
:1065E800798D15D00201798F12D00501FA51010A6F
:1065F800E4E0030AE5E0010AE6E0070AE7E0010A49
:10660800E8E0030AE9E0010AEAE00F0AEBE0110E0C
:1066180002015F6F0401426F0301F76B79C2F8F35F
:10662800010ECCECBBF05DD3390EE86F230EE96F99
:10663800FAC5EAF5EB6B1DECD0F0310E0201A16F43
:10664800330EA06F300E9F6F9E6F310E9D6F300E10
:106658009C6F9B6F0501FA51300F02019A6F070E6C
:106668000501D66F000E19ECABF03BD3000166AF05
:1066780003D00501FA0531E0000166AD04D0020E31
:106688000501FA192AE0000166AB04D0030E0501E2
:10669800FA1923E0000166A904D0040E0501FA19CD
:1066A8001CE0000166A704D0050E0501FA1915E0E3
:1066B800000166A504D0060E0501FA190EE00001D6
:1066C80066A304D0070E0501FA1907E0000166A1C8
:1066D80028D0080E0501FA1924E1330E0201A16F32
:1066E800370EA06F330E9F6F300E9E6F310E9D6F69
:1066F800300E9C6F9B6F0501FA51300F02019A6FA3
:10670800060E0501D66F000E19ECABF02C0E050134
:10671800E86F240EE96FFAC5EAF5EB6B1DECD0F0D3
:10672800E0D2310E0201A16FA06F300E9F6F9E6FF5
:10673800310E9D6F300E9C6F9B6F0501FA51300F23
:1067480002019A6F060E0501D66F000E19ECABF028
:10675800538E53BC8A8C020186513C0DF3CF6FF3E4
:10676800F4CF70F30001678518D00201798127D032
:106778000201798324D00201798521D00201798729
:106788001ED0020179891BD00201798B18D0020131
:10679800798D15D00201798F12D00501FA51010ABD
:1067A800E4E0030AE5E0010AE6E0070AE7E0010A97
:1067B800E8E0030AE9E0010AEAE00F0AEBE0110E5B
:1067C80002015F6F0401426F0301F76B79C2F8F3AE
:1067D800010ECCECBBF00A0E0501E86F240EE96F40
:1067E800FAC5EAF5EB6B1DECD0F07BD2000166AF81
:1067F80003D00501FA0531E0000166AD04D0020EB0
:106808000501FA192AE0000166AB04D0030E050160
:10681800FA1923E0000166A904D0040E0501FA194B
:106828001CE0000166A704D0050E0501FA1915E061
:10683800000166A504D0060E0501FA190EE0000154
:1068480066A304D0070E0501FA1907E0000166A146
:1068580039D0080E0501FA1935E1000166BF669FB7
:1068680066BD669D66BB669B66B9669966B76697A0
:1068780066B5669566B3669366B16691330E020196
:10688800A16F370EA06F330E9F6F300E9E6F310EC3
:106898009D6F300E9C6F9B6F0501FA51300F0201FE
:1068A8009A6F070E0501D66F000E19ECABF0820E39
:1068B8000501E86F210EE96FFAC5EAF5EB6B1DECEF
:1068C800D0F00FD2310E0201A16FA06F300E9F6F72
:1068D8009E6F310E9D6F300E9C6F9B6F0501FA51B4
:1068E800300F02019A6F070E0501D66F000E19ECE2
:1068F800ABF0340E0501E86F230EE96FFAC5EAF52F
:10690800EB6B1DECD0F0EDD1330E0201A16F300E10
:10691800A06F310E9F6F300E9E6F9D6F9C6F9B6FA7
:106928009A6F060E0501D66F000E19ECABF0B40E87
:106938000501E86F240EE96FFAC5EAF5EB6B1DEC6B
:10694800D0F0CFD1330E0201A16F300EA06F310EFF
:106958009F6F300E9E6F9D6F9C6F9B6F9A6F070E97
:106968000501D66F000E19ECABF0C40E0501E86FF7
:10697800230EE96FFAC5EAF5EB6B1DECD0F0B1D147
:10698800EF0EE86F220EE96FFAC5EAF5EB6B1DEC26
:10699800D0F002015E91170E0301FB6F030EFA6F30
:1069A80033ECC3F001090601406F170E0401FA6FBA
:1069B800030EF96F40C6FBF40BECC7F00A0E030197
:1069C800F76F0501FA51B1ECCFF002019B6F9B51B3
:1069D800F60DF3500501FA2502019A6F300E9A2739
:1069E8009B27340EA16F300EA06F310E9F6F300EB3
:1069F8009E6F310E9D6F300E9C6F070E0501D66F8E
:106A0800000E19ECABF06DD1EA0EE86F220EE96FBB
:106A1800FAC5EAF5EB6B1DECD0F002015E915E87DA
:106A28005EC241F4170E0301FB6F030EFA6F33ECDD
:106A3800C3F002090601416F170E0401FA6F030E35
:106A4800F96F41C6FBF40BECC7F00A0E0301F76FB0
:106A58000501FA51B1ECCFF002019B6F9B51F60D85
:106A6800F3500501FA2502019A6F300E9A279B27E9
:106A7800340EA16FA06F310E9F6F300E9E6F310ED6
:106A88009D6F300E9C6F070E0501D66F000E19EC36
:106A9800ABF027D1050EE86F220EE96FFAC5EAF5CB
:106AA800EB6B1DECD0F002015E93170E0301FB6F38
:106AB800030EFA6F33ECC3F0FC0B0601426F170E9E
:106AC8000401FA6F030EF96F42C6FBF40BECC7F032
:106AD8000A0E0301F76F0501FA51B1ECCFF002017C
:106AE8009B6F9B51F60DF3500501FA2502019A6F31
:106AF800300E9A279B27340EA16F300EA06F310EEF
:106B08009F6F300E9E6F310E9D6F300E9C6F060E7C
:106B18000501D66F000E19ECABF0E3D0000EE86F5C
:106B2800220EE96FFAC5EAF5EB6B1DECD0F0F50E15
:106B380002015E17170E0301FB6F030EFA6F33ECA9
:106B4800C3F0FC0B0601436F170E0401FA6F030E26
:106B5800F96F43C6FBF40BECC7F00A0E0301F76F9D
:106B68000501FA51B1ECCFF002019B6F9B51F60D74
:106B7800F3500501FA2502019A6F300E9A279B27D8
:106B8800340EA16FA06F310E9F6F300E9E6F310EC5
:106B98009D6F300E9C6F060E0501D66F000E19EC26
:106BA800ABF09FD0330E0201A16FA06F9F6F300E24
:106BB8009E6F9D6F9C6F9B6F0501FA51300F02010C
:106BC8009A6F060E0501D66F000E19ECABF0590E40
:106BD8000501E86F250EE96FFAC5EAF5EB6B1DECC8
:106BE800D0F07FD0330E0201A16FA06F9F6F300EDF
:106BF8009E6F9D6F9C6F9B6F0501FA51300F0201CC
:106C08009A6F070E0501D66F000E19ECABF0920EC5
:106C18000501E86F240EE96FFAC5EAF5EB6B1DEC88
:106C2800D0F05FD0360E0201A16F320EA06F370E82
:106C38009F6F300E9E6F9D6F9C6F9B6F9A6F060EB5
:106C48000501D66F000E19ECABF02D0E0501E86FAB
:106C58002A0EE96F1DECD0F044D0360E0201A16F68
:106C6800320EA06F380E9F6F300E9E6F9D6F9C6F17
:106C78009B6F9A6F060E0501D66F000E19ECABF0EC
:106C8800C40E0501E86F290EE96F1DECD0F029D07C
:106C98000501F951010A01E162D4030A01E1C4D4F2
:106CA800010A01E16DD6070A01E1F4D6010A01E102
:106CB800DDD4030A01E19AD5010A01E125D60F0ABC
:106CC80001E140D6010A01E19FD6030A01E126D776
:106CD800010A01E167D7070A85E0010AA3E0030A70
:106CE800BCE0020E0601481901E1EFD21200530E72
:106CF800E86F240EE96FFAC5EAF5EB6B1DECD0F0EE
:106D0800538E0001678353BC8A8C020186513C0D67
:106D1800F3CF6FF3F4CF70F3310EA16F330EA06F82
:106D2800300E9F6F9E6F320E9D6F300E9C6F9B6F63
:106D38000501FA51300F02019A6F060E0501D66F50
:106D4800000E19ECABF018D00201788127D00201AF
:106D5800788324D00201788521D0020178871ED05B
:106D6800020178891BD00201788B18D00201788D36
:106D780015D00201788F12D00501FA51010AE4E01A
:106D8800030AE5E0010AE6E0070AE7E0010AE8E0AD
:106D9800030AE9E0010AEAE00F0AEBE0110E02013A
:106DA8005D6F0301F76B78C2F8F3020ECCEFBBF00E
:106DB8005D0EE86F230EE96FFAC5EAF5EB6B1DEC83
:106DC800D0F0310E0201A16F330EA06F300E9F6F0D
:106DD8009E6F320E9D6F300E9C6F9B6F0501FA51AE
:106DE800300F02019A6FE9D1000165AF03D00501A8
:106DF800FA0531E0000165AD04D0020E0501FA196B
:106E08002AE0000165AB04D0030E0501FA1923E05E
:106E1800000165A904D0040E0501FA191CE000015F
:106E280065A704D0050E0501FA1915E0000165A54E
:106E380004D0060E0501FA190EE0000165A304D07E
:106E4800070E0501FA1907E0000165A122D0080E16
:106E58000501FA191EE1330E0201A16F370EA06F6A
:106E6800330E9F6F300E9E6F320E9D6F300E9C6FEB
:106E78009B6F0501FA51300F02019A6F060E05014A
:106E8800D66F000E19ECABF0700E0501E86F240EFA
:106E98000ED1310E0201A16FA06F300E9F6F9E6F51
:106EA800320E9D6F300E9C6F9B6F0501FA51300FAB
:106EB80002019A6F060E0501D66F000E19ECABF0B1
:106EC800538E53BC8A8C020186513C0DF3CF6FF36D
:106ED800F4CF70F30001678318D00201788127D0BE
:106EE8000201788324D00201788521D002017887B5
:106EF8001ED0020178891BD00201788B18D00201BC
:106F0800788D15D00201788F12D00501FA51010A47
:106F1800E4E0030AE5E0010AE6E0070AE7E0010A1F
:106F2800E8E0030AE9E0010AEAE00F0AEBE0110EE3
:106F380002015D6F0301F76B78C2F8F3020ECCEC27
:106F4800BBF04E0E0501E86F240EB1D0000165AF0D
:106F580003D00501FA0531E0000165AD04D0020E49
:106F68000501FA192AE0000165AB04D0030E0501FA
:106F7800FA1923E0000165A904D0040E0501FA19E5
:106F88001CE0000165A704D0050E0501FA1915E0FB
:106F9800000165A504D0060E0501FA190EE00001EE
:106FA80065A304D0070E0501FA1907E0000165A1E1
:106FB80033D0080E0501FA192FE1000165BF659F5E
:106FC80065BD659D65BB659B65B9659965B7659741
:106FD80065B5659565B3659365B16591330E020135
:106FE800A16F370EA06F330E9F6F300E9E6F320E5B
:106FF8009D6F300E9C6F9B6F0501FA51300F020197
:107008009A6F070E0501D66F000E19ECABF0AC0EA7
:107018000501E86F210E4BD0310E0201A16FA06F60
:10702800300E9F6F9E6F320E9D6F300E9C6F9B6F60
:107038000501FA51300F02019A6F070E0501D66F4C
:10704800000E19ECABF0580E0501E86F230E2FD097
:10705800330E0201A16F300EA06F310E9F6F300EFC
:107068009E6F9D6F9C6F9B6F9A6F060E0501D66F82
:10707800000E19ECABF0D50E0501E86F240E17D001
:10708800330E0201A16F300EA06F310E9F6F300ECC
:107098009E6F9D6F9C6F9B6F9A6F070E0501D66F51
:1070A800000E19ECABF0E70E0501E86F230EE96F4F
:1070B800FAC5EAF5EB6B1DEFD0F0140EE86F230E5E
:1070C800E96FFAC5EAF5EB6B1DECD0F002015C91B3
:1070D8000A0E0301F76F0501FA51B1ECCFF0020176
:1070E8009B6F9B51F60DF3500501FA2502019A6F2B
:1070F800300E9A279B27340EA16F300EA06F310EE9
:107108009F6F300E9E6F320E9D6F300E9C6F070E74
:107118000501D66F000E19ECABF0170E0301FB6FDB
:10712800030EFA6F33ECC3F004090601446F170E1F
:107138000401FA6F030EF96F44C6FBF40BEFC7F0B6
:107148000F0EE86F230EE96FFAC5EAF5EB6B1DEC3D
:10715800D0F002015C915C87170E0301FB6F030EF0
:10716800FA6F33ECC3F008090601456F170E0401E6
:10717800FA6F030EF96F45C6FBF40BECC7F00A0E65
:107188000301F76F0501FA51B1ECCFF002019B6FD3
:107198009B51F60DF3500501FA2502019A6F300E46
:1071A8009A279B27340EA16FA06F310E9F6F300E68
:1071B8009E6F320E9D6F300E9C6F070E81D02D0E84
:1071C800E86F220EE96FFAC5EAF5EB6B1DECD0F01B
:1071D80002015C930A0E0301F76F0501FA51B1EC45
:1071E800CFF002019B6F9B51F60DF3500501FA2574
:1071F80002019A6F300E9A279B27340EA16F300E2A
:10720800A06F310E9F6F300E9E6F320E9D6F300E45
:107218009C6F060E0501D66F000E19ECABF0170E29
:107228000301FB6F030EFA6F33ECC3F0F30B060197
:10723800466F170E0401FA6F030EF96F46C6FBF48A
:107248000BEFC7F0280EE86F220EE96FFAC5EAF5D2
:10725800EB6B1DECD0F0F50E02015C17170E030165
:10726800FB6F030EFA6F33ECC3F0F30B0601476FA5
:10727800170E0401FA6F030EF96F47C6FBF40BEC07
:10728800C7F00A0E0301F76F0501FA51B1ECCFF010
:1072980002019B6F9B51F60DF3500501FA2502017F
:1072A8009A6F300E9A279B27340EA16FA06F310E6C
:1072B8009F6F300E9E6F320E9D6F300E9C6F060EC4
:1072C8000501D66F000E19EFABF00501F951010A5F
:1072D80001E10DD5030A01E16BD5010A01E1EDD603
:1072E800070A01E16CD7010A01E17ED5030A01E131
:1072F8002DD6010A01E1ACD60F0A01E1C1D6010A77
:1073080001E11ED7030A9EE01200446E02017D1DB2
:10731800456E440401E049D38C51010B466E46A0EA
:107328005BD04650451435E055B455A255D054B4F9
:1073380003D0000169AF15D00201850506E0020EF1
:10734800851903E0030E851947E1010E396E3A6E7F
:10735800BCEC58F0010E396E3A6E020EBCEC58F0D7
:107368003BD00201850509E0020E851906E0030EEF
:10737800851903E0040E85192FE1010E396E3A6E66
:10738800BCEC58F0010E396E3A6E020EBCEC58F0A7
:1073980023D046505B1520E054A40ED0850506E0A6
:1073A800020E851903E0030E851916E1010E396EE8
:1073B8003A6EBCEC58F010D0850509E0020E85192C
:1073C80006E0030E851903E0040E851905E1010E98
:1073D800396E3A6EBCEC58F002018C51020B466EC5
:1073E80046A261D04650451439E055B455A25BD049
:1073F80054B403D0000169AF17D00201840506E038
:10740800020E841903E0030E84194DE1010E396E52
:10741800020E3A6E010EBCEC58F0010E396E020EE7
:107428003A6EBCEC58F03FD00201840509E0020E28
:10743800841906E0030E841903E0040E841933E16D
:10744800010E396E020E3A6E010EBCEC58F0010EB8
:10745800396E020E3A6EBCEC58F025D046505B15DA
:1074680022E054A40ED0840506E0020E841903E03D
:10747800030E841918E1010E396E3A6EBCEC58F00F
:1074880012D0840509E0020E841906E0030E84195F
:1074980003E0040E841907E1010E396E020E3A6EFC
:1074A800010EBCEC58F002018C51040B466E46A448
:1074B80065D0465045143BE055B455A25FD054B44E
:1074C80003D0000169AF18D00201830506E0020E5F
:1074D800831903E0030E831951E1010E396E030E7F
:1074E8003A6E010EBCEC58F0010E396E030E3A6E7E
:1074F800020EBCEC58F042D00201830509E0020EEE
:10750800831906E0030E831903E0040E831936E19C
:10751800010E396E030E3A6E010EBCEC58F0010EE6
:10752800396E030E3A6E020EBCEC58F027D0465066
:107538005B1524E054A410D0830506E0020E8319DD
:1075480003E0030E83191AE1010E396E030E3A6E39
:10755800010EBCEC58F012D0830509E0020E831925
:1075680006E0030E831903E0040E831907E1010EF8
:10757800396E030E3A6E010EBCEC58F002018C51C4
:10758800080B466E46A665D0465045143BE055B4F8
:1075980055A25FD054B403D0000169AF18D00201DE
:1075A800820506E0020E821903E0030E821951E1FA
:1075B800010E396E040E3A6E010EBCEC58F0010E45
:1075C800396E040E3A6E020EBCEC58F042D002013D
:1075D800820509E0020E821906E0030E821903E013
:1075E800040E821936E1010E396E040E3A6E010E50
:1075F800BCEC58F0010E396E040E3A6E020EBCEC6B
:1076080058F027D046505B1524E054A410D08205CA
:1076180006E0020E821903E0030E82191AE1010E38
:10762800396E040E3A6E010EBCEC58F012D0820589
:1076380009E0020E821906E0030E821903E0040E27
:10764800821907E1010E396E040E3A6E010EBCEC88
:1076580058F002018C51100B466E46A865D0465072
:1076680045143BE055B455A25FD054B403D0000193
:1076780069AF18D00201810506E0020E811903E006
:10768800030E811951E1010E396E050E3A6E010E95
:10769800BCEC58F0010E396E050E3A6E020EBCECC9
:1076A80058F042D00201810509E0020E811906E076
:1076B800030E811903E0040E811936E1010E396EBB
:1076C800050E3A6E010EBCEC58F0010E396E050E2F
:1076D8003A6E020EBCEC58F027D046505B1524E0F9
:1076E80054A410D0810506E0020E811903E0030EB0
:1076F80081191AE1010E396E050E3A6E010EBCECC5
:1077080058F012D0810509E0020E811906E0030E37
:10771800811903E0040E811907E1010E396E050E87
:107728003A6E010EBCEC58F002018C51200B466EEB
:1077380046AA65D0465045143BE055B455A25FD0E3
:1077480054B403D0000169AF18D00201800506E0E7
:10775800020E801903E0030E801951E1010E396E03
:10776800060E3A6E010EBCEC58F0010E396E060E8C
:107778003A6E020EBCEC58F042D00201800509E0D6
:10778800020E801906E0030E801903E0040E80192A
:1077980036E1010E396E060E3A6E010EBCEC58F059
:1077A800010E396E060E3A6E020EBCEC58F027D068
:1077B80046505B1524E054A410D0800506E0020E64
:1077C800801903E0030E80191AE1010E396E060EC6
:1077D8003A6E010EBCEC58F012D0800509E0020E9A
:1077E800801906E0030E801903E0040E801907E1F2
:1077F800010E396E060E3A6E010EBCEC58F002010D
:107808008C51400B466E46AC65D0465045143BE063
:1078180055B455A25FD054B403D0000169AF18D055
:1078280002017F0506E0020E7F1903E0030E7F19AF
:1078380051E1010E396E070E3A6E010EBCEC58F09C
:10784800010E396E070E3A6E020EBCEC58F042D0AB
:1078580002017F0509E0020E7F1906E0030E7F1979
:1078680003E0040E7F1936E1010E396E070E3A6EF9
:10787800010EBCEC58F0010E396E070E3A6E020E7E
:10788800BCEC58F027D046505B1524E054A410D027
:107898007F0506E0020E7F1903E0030E7F191AE147
:1078A800010E396E070E3A6E010EBCEC58F012D07C
:1078B8007F0509E0020E7F1906E0030E7F1903E039
:1078C800040E7F1907E1010E396E070E3A6E010E9C
:1078D800BCEC58F002018C51800B466E46AE65D068
:1078E800465045143BE055B455A25FD054B403D07C
:1078F800000169AF18D002017E0506E0020E7E196C
:1079080003E0030E7E1951E1010E396E080E3A6E3E
:10791800010EBCEC58F0010E396E080E3A6E020EDC
:10792800BCEC58F042D002017E0509E0020E7E1937
:1079380006E0030E7E1903E0040E7E1936E1010EFF
:10794800396E080E3A6E010EBCEC58F0010E396E15
:10795800080E3A6E020EBCEC58F027D046505B1564
:1079680024E054A410D07E0506E0020E7E1903E040
:10797800030E7E191AE1010E396E080E3A6E010ED9
:10798800BCEC58F012D07E0509E0020E7E1906E024
:10799800030E7E1903E0040E7E1907E1010E396E0D
:1079A800080E3A6E010EBCEC58F0020E4418D8A42A
:1079B800120002018C51010B466E46A060D0465061
:1079C800451435E055B455A25AD054B403D000013B
:1079D80069AF15D00201850506E0020E851903E09E
:1079E800030E85194CE1010E396E3A6EBCEC58F065
:1079F800010E396E3A6E020EBCEC58F040D002010E
:107A0800850509E0020E851906E0030E851903E0D5
:107A1800040E851934E1010E396E3A6EBCEC58F04B
:107A2800010E396E3A6E020EBCEC58F028D0465062
:107A38005A1525E0000169AF10D00201850506E05E
:107A4800020E851903E0030E851919E1010E396E3E
:107A58003A6E020EBCEC58F012D00201850509E01E
:107A6800020E851906E0030E851903E0040E851938
:107A780006E1010E396E3A6E020EBCEC58F00201B6
:107A88008C51020B466E46A264D04650451439E02C
:107A980055B455A25ED054B403D0000169AF17D0D5
:107AA8000201840506E0020E841903E0030E84191E
:107AB80050E1010E396E020E3A6E010EBCEC58F020
:107AC800010E396E020E3A6EBCEC58F042D002013B
:107AD800840509E0020E841906E0030E841903E008
:107AE800040E841936E1010E396E020E3A6E010E4B
:107AF800BCEC58F0010E396E020E3A6EBCEC58F030
:107B080028D046505A1525E0000169AF10D002016F
:107B1800840506E0020E841903E0030E841919E1B6
:107B2800010E396E3A6E020EBCEC58F012D002010A
:107B3800840509E0020E841906E0030E841903E0A7
:107B4800040E841906E1010E396E020E3A6EBCEC81
:107B580058F002018C51040B466E46A468D046507A
:107B680045143BE055B455A262D054B403D000018B
:107B780069AF18D00201830506E0020E831903E0FD
:107B8800030E831954E1010E396E030E3A6E010E8D
:107B9800BCEC58F0010E396E030E3A6E020EBCECC6
:107BA80058F045D00201830509E0020E831906E06A
:107BB800030E831903E0040E831939E1010E396EAF
:107BC800030E3A6E010EBCEC58F0010E396E030E2E
:107BD8003A6E020EBCEC58F02AD046505A1527E0EF
:107BE800000169AF11D00201830506E0020E831976
:107BF80003E0030E83191BE1010E396E030E3A6E82
:107C0800020EBCEC58F013D00201830509E0020E05
:107C1800831906E0030E831903E0040E831907E1B4
:107C2800010E396E030E3A6E020EBCEC58F00201DA
:107C38008C51080B466E46A668D0465045143BE06A
:107C480055B455A262D054B403D0000169AF18D01E
:107C58000201820506E0020E821903E0030E821972
:107C680054E1010E396E040E3A6E010EBCEC58F068
:107C7800010E396E040E3A6E020EBCEC58F045D077
:107C88000201820509E0020E821906E0030E82193C
:107C980003E0040E821939E1010E396E040E3A6EC2
:107CA800010EBCEC58F0010E396E040E3A6E020E4D
:107CB800BCEC58F02AD046505A1527E0000169AFAD
:107CC80011D00201820506E0020E821903E0030EBC
:107CD80082191BE1010E396E040E3A6E020EBCECDD
:107CE80058F013D00201820509E0020E821906E05D
:107CF800030E821903E0040E821907E1010E396EA2
:107D0800040E3A6E020EBCEC58F002018C51100BB6
:107D1800466E46A868D0465045143BE055B455A277
:107D280062D054B403D0000169AF18D002018105B4
:107D380006E0020E811903E0030E811954E1010ED9
:107D4800396E050E3A6E010EBCEC58F0010E396E14
:107D5800050E3A6E020EBCEC58F045D002018105C2
:107D680009E0020E811906E0030E811903E0040EF2
:107D7800811939E1010E396E050E3A6E010EBCEC1F
:107D880058F0010E396E050E3A6E020EBCEC58F032
:107D98002AD046505A1527E0000169AF11D00201D8
:107DA800810506E0020E811903E0030E81191BE12B
:107DB800010E396E050E3A6E020EBCEC58F013D067
:107DC8000201810509E0020E811906E0030E8119FE
:107DD80003E0040E811907E1010E396E050E3A6EB3
:107DE800020EBCEC58F002018C51200B466E46AADC
:107DF80068D0465045143BE055B455A262D054B4FF
:107E080003D0000169AF18D00201800506E0020E18
:107E1800801903E0030E801954E1010E396E060E35
:107E28003A6E010EBCEC58F0010E396E060E3A6E31
:107E3800020EBCEC58F045D00201800509E0020EA4
:107E4800801906E0030E801903E0040E801939E159
:107E5800010E396E060E3A6E010EBCEC58F0010E9A
:107E6800396E060E3A6E020EBCEC58F02AD0465017
:107E78005A1527E0000169AF11D00201800506E01C
:107E8800020E801903E0030E80191BE1010E396E02
:107E9800060E3A6E020EBCEC58F013D002018005B3
:107EA80009E0020E801906E0030E801903E0040EB3
:107EB800801907E1010E396E060E3A6E020EBCEC0F
:107EC80058F002018C51400B466E46AC68D04650C3
:107ED80045143BE055B455A262D054B403D0000118
:107EE80069AF18D002017F0506E0020E7F1903E092
:107EF800030E7F1954E1010E396E070E3A6E010E1A
:107F0800BCEC58F0010E396E070E3A6E020EBCEC4E
:107F180058F045D002017F0509E0020E7F1906E0FE
:107F2800030E7F1903E0040E7F1939E1010E396E43
:107F3800070E3A6E010EBCEC58F0010E396E070EB2
:107F48003A6E020EBCEC58F02AD046505A1527E07B
:107F5800000169AF11D002017F0506E0020E7F190A
:107F680003E0030E7F191BE1010E396E070E3A6E0E
:107F7800020EBCEC58F013D002017F0509E0020E96
:107F88007F1906E0030E7F1903E0040E7F1907E14D
:107F9800010E396E070E3A6E020EBCEC58F0020163
:107FA8008C51800B466E46AE1200465045142FE0A9
:107FB80055B455A2120054B403D0000169AF12D0D1
:107FC80002017E0507E0020E7E1904E0030E7E1909
:107FD800D8A41200010E396E080E3A6E010EBCECE0
:107FE80058F031D002017E050AE0020E7E1907E042
:107FF800030E7E1904E0040E7E19D8A41200010EA7
:10800800396E080E3A6E010EBCEC58F01CD0465082
:108018005A15D8B41200000169AF08D002017E05D4
:1080280012E0020E7E190FE0030E0AD002017E054F
:108038000AE0020E7E1907E0030E7E1904E0040E22
:108048007E19D8A41200010E396E080E3A6E020E7F
:10805800BCEF58F0136A000163973DEF45F0B4ECAC
:1080680045F0DF5009E12CEC46F00A6F100E0B6F5B
:108078000C6B0D6BB2EF45F0B4EC45F0DE0405E196
:108088002CEC46F00A6F200EF2D7B4EC45F0020E45
:10809800DE1802E1060E08D0B4EC45F0030EDE1837
:1080A80002E0B2EF45F0070E0101076F380EDDD789
:1080B80052EC63F023EC46F0B2ECC9F0B4EC45F0B6
:1080C800DF507AECCFF08ED1070EC0EC45F010EC03
:1080D80046F0B2ECC9F0B4EC45F0DF507AECCFF0E2
:1080E80081D1B4EC45F0DF5009E1070EC0EC45F052
:1080F80011C001F0030EB2ECC9F0BBD7B4EC45F0E7
:10810800DE0405E0B4EC45F0020EDE1809E1070EC6
:108118000101076F450E05EC46F0B2ECC9F0A9D78E
:10812800B4EC45F0030EDE1807E152EC63F029ECDD
:1081380046F0B2ECC9F09DD7B4EC45F0040EDE1859
:1081480008E1070EC0EC45F023EC46F0B2ECC9F0AC
:1081580090D7B4EC45F0050EDE1808E1070EC0EC28
:1081680045F026EC46F0B2ECC9F083D7B4EC45F004
:10817800060EDE1802E0B2EF45F0070EC0EC45F03F
:1081880030EC46F0B2ECC9F074D7060EC0EC45F0FE
:1081980010EC46F0B2ECC9F0B4EC45F0DF507AECE4
:1081A800CFF020D1060EC0EC45F010EC46F0B2EC52
:1081B800C9F0B4EC45F0DF507AECCFF013D1060EDD
:1081C800C0EC45F029EC46F0B2ECC9F0B4EC45F04F
:1081D800DF507AECCFF006D1B4EC45F0DF5008E17F
:1081E800070EC0EC45F01DEC46F0B2ECC9F041D7E3
:1081F800B4EC45F0DE0405E0B4EC45F0020EDE1800
:1082080008E1060EC0EC45F026EC46F0B2ECC9F0E9
:1082180030D7B4EC45F0030EDE180AE0B4EC45F0B4
:10822800040EDE1805E0B4EC45F0070EDE1808E190
:10823800060EC0EC45F029EC46F0B2ECC9F019D7AF
:10824800B4EC45F0050EDE1808E1060EC0EC45F06A
:1082580030EC46F0B2ECC9F00CD7B4EC45F0060EA1
:10826800DE1802E0B2EF45F0060EC0EC45F030EC47
:1082780046F0B2ECC9F0FDD649EC63F0EFEC45F0FE
:10828800B2ECC9F0B4EC45F0DF507AECCFF0AAD0EC
:10829800060E3DEC63F016EC46F0B2ECC9F0B4EC17
:1082A80045F0DF507AECCFF09DD06BEC63F0EFEC4B
:1082B80045F0B2ECC9F0B4EC45F0DF507AECCFF001
:1082C80091D0070E3DEC63F016EC46F0B2ECC9F025
:1082D800B4EC45F0DF507AECCFF084D0070E010102
:1082E800076F110EEFEC45F0B2ECC9F0B4EC45F0B5
:1082F800DF507AECCFF076D0B4EC45F0DF5007E1F0
:1083080067EC63F0EFEC45F0B2ECC9F0B2D6B4EC30
:1083180045F0DE0407E119EC46F0EFEC45F0B2EC6D
:10832800C9F0A7D6B4EC45F0020EDE1808E16BECF4
:1083380063F00A6F1DEC46F0B2ECC9F09AD6B4ECC3
:1083480045F0030EDE1807E152EC63F030EC46F01E
:10835800B2ECC9F08ED6B4EC45F0040EDE1808E194
:10836800060E4DEC63F023EC46F0B2ECC9F081D672
:10837800F7DB050EDE1807E167EC63F0CDEC45F09E
:10838800B2ECC9F076D6ECDB060EDE1801E0E6D3D7
:10839800060E0101076F420EFCDBB2ECC9F069D68C
:1083A80049EC63F0EFEC45F0B2ECC9F0D9DBDF50F3
:1083B8007AECCFF017D0060E3DEC63F026EC46F0D1
:1083C800B2ECC9F0CDDBDF507AECCFF00BD0070E62
:1083D8003DEC63F026EC46F0B2ECC9F0C1DBDF50AF
:1083E8007AECCFF00101F7D1070EBFDB010EB2EC3A
:1083F800C9F03FD6070E0101076F300ECADBB2EC99
:10840800C9F037D6070E4DEC63F020EC46F0B2EC1D
:10841800C9F02FD6070E76EC63F0F3DBB2ECC9F0A7
:1084280028D6070EF2DBB5DBB2ECC9F022D6070E70
:10843800ECDBAFDBB2ECC9F01CD6070E0101076F0D
:10844800620E0A6F29EC46F0B2ECC9F012D6070E9C
:1084580079EC63F0CADBB2ECC9F00BD6070E85DB0A
:10846800010EB2ECC9F005D6070E7FDB020EB2ECA6
:10847800C9F0FFD5070E79DB040EB2ECC9F0010E86
:10848800AAD1070EA1DBB2ECC9F0F3D5070E9CDB2D
:10849800B2ECC9F0F4D7070E68DB000EB2ECC9F0F5
:1084A800E8D5ABDB76DBB2ECC9F0E9D7070E5DDBCC
:1084B800040EB2ECC9F0020E8ED1070E56DB040E84
:1084C800B2ECC9F0030E87D1070E4FDB000EB2ECF9
:1084D800C9F0D5D792DB5DDBB2ECC9F0ECD7070E5B
:1084E80044DB040EB2ECC9F0040E75D1070E3DDB77
:1084F800040EB2ECC9F0050E6ED132DBDF5001E19B
:1085080073D7010A01E176D7030A01E17BD7010A93
:1085180081E0070A86E0010A8AE0030A8EE0010A80
:1085280096E00F0A9BE0010A9FE0020AA3E0070A0F
:10853800A8E0010AABE0030AAEE0010AB2E01F0AB4
:10854800B5E0010ABAE0030ABFE0010AC3E0070A7E
:10855800C6E0010ACBE002D3060E0101076F300E18
:1085680018DBB2ECC9F085D5060E4DEC63F064DB80
:10857800B2ECC9F07ED5060E76EC63F042DBB2ECC5
:10858800C9F077D5060E41DB04DBB2ECC9F071D532
:10859800060E3BDBFEDAB2ECC9F06BD506DB060E45
:1085A800B2ECC9F066D5060E79EC63F01EDBB2ECCE
:1085B800C9F05FD5060ED9DA010EB2ECC9F059D56B
:1085C800060ED3DA020EB2ECC9F053D5060ECDDA98
:1085D800040EB2ECC9F053D7060EF6DAB2ECC9F0C5
:1085E80048D5060EF1DAB2ECC9F049D7060EBDDA65
:1085F800000EB2ECC9F03DD5FCDACBDAB2ECC9F02A
:108608003ED7060EB2DA040EB2ECC9F054D7060E05
:10861800ACDA040EB2ECC9F055D7060EA6DA000E95
:10862800B2ECC9F02CD7E5DAB4DAB2ECC9F043D72A
:10863800060E9BDA040EB2ECC9F056D7060E95DA90
:10864800040EB2ECC9F057D78BDADF50010A84E088
:10865800030A8AE0010A8FE0070A94E0010A98E019
:10866800030A9CE0010A9FE00F0AA4E0010AA8E0BF
:10867800020AACE0070AB0E0010AB3E0030AB6E078
:10868800010ABAE01F0ABDE0010AC1E0030AC5E019
:10869800010AC9E0070ACCE0010AD0E05FD2060E61
:1086A800BEDA77DAB2ECC9F0E4D4060E0101076F3E
:1086B800340E6FDAB2ECC9F0DCD4060E01018FDAA1
:1086C800B2ECC9F0D6D4060EAADAA2DAB2ECC9F036
:1086D800D0D446DADF50E3E0010AE7E0030AEDE030
:1086E800010AF1E03BD2070E9ADA53DAB2ECC9F08C
:1086F800C0D4070E0101076F340E4BDAB2ECC9F093
:10870800B8D4070E01016BDAB2ECC9F0B2D4070E87
:1087180086DA7EDAB2ECC9F0ACD422DADF50E3E0D4
:10872800010AE7E0030AEDE0010AF1E017D2060EBC
:108738004DEC63F07EDAB2ECC9F09BD472EC63F0D6
:1087480060DAB2ECC9F095D430DA070EB2ECC9F0B1
:1087580090D42BDA080EB2ECC9F08BD426DA070EC7
:10876800B2ECC9F086D421DA080EB2ECC9F081D493
:108778001CDA070EB2ECC9F07CD417DA080EB2EC9A
:10878800C9F077D4060E0101076F650E0A6F11C094
:1087980001F0040EB2ECC9F06CD4E2D9DF50C7E0A6
:1087A800010ACCE0030AD0E0010AD3E0070AD6E0C8
:1087B800010AD9E0030ADCE0010ADFE00F0AE2E07F
:1087C800CDD1060EFAD9040EB2ECC9F0C9D9DF50E2
:1087D8007AECCFF007D60D6FC1D1070EEED9040E93
:1087E800B2ECC9F0BDD9DF507AECCFF0FBD5060E5C
:1087F800E4D9000EB2ECC9F0B3D9DF507AECCFF06F
:10880800F1D5070EDAD9000EB2ECC9F0A9D9DF50BC
:108818007AECCFF0E7D5A4D9DF500DE0A1D9110E3D
:10882800DF6009D0AED9030EB2ECC9F099D9DF5098
:108838007AECCFF0D7D594D9110EDE1804E090D990
:10884800120EDE1809E19DD9030EB2ECC9F088D9E1
:10885800DF507AECCFF0C6D583D9120EDF640DD085
:108868007FD9170EDF6009D08CD9030EB2ECC9F09E
:1088780077D9DF507AECCFF0B5D572D91A0EDF640C
:108888006DD16ED91F0EDF6069D17BD9030EB2ECB2
:10889800C9F066D9DF507AECCFF0A4D561D9DF50A2
:1088A8000DE05ED9110EDF6009D077D9030EB2EC66
:1088B800C9F056D9DF507AECCFF094D551D9110EC2
:1088C800DE1804E04DD9120EDE1809E166D9030E50
:1088D800B2ECC9F045D9DF507AECCFF083D540D956
:1088E800120EDF640DD03CD9170EDF6009D055D9C0
:1088F800030EB2ECC9F034D9DF507AECCFF072D560
:108908002FD91A0EDF642AD12BD91F0EDF6026D18A
:1089180044D9030EB2ECC9F023D9DF507AECCFF07A
:1089280061D51ED9DF500DE01BD9110EDF6009D0CB
:1089380028D9050EB2ECC9F013D9DF507AECCFF084
:1089480051D50ED9110EDE1804E00AD9120EDE1820
:1089580009E117D9050EB2ECC9F002D9DF507AEC5B
:10896800CFF040D5FDD8120EDF640DD0F9D8170E20
:10897800DF6009D006D9050EB2ECC9F0F1D8DF5096
:108988007AECCFF02FD5ECD81A0EDF64E7D0E8D810
:108998001F0EDF60E3D0F5D8050EB2ECC9F0E0D8C1
:1089A800DF507AECCFF01ED5DBD8DF500DE0D8D8F9
:1089B800110EDF6009D0F1D8050EB2ECC9F0D0D89D
:1089C800DF507AECCFF00ED5CBD8110EDE1804E0CC
:1089D800C7D8120EDE1809E1E0D8050EB2ECC9F0CE
:1089E800BFD8DF507AECCFF0FDD4BAD8120EDF64CE
:1089F8000DD0B6D8170EDF6009D0CFD8050EB2EC6F
:108A0800C9F0AED8DF507AECCFF0ECD4A9D81A0E62
:108A1800DF64A4D0A5D81F0EDF60A0D0BED8050E95
:108A2800B2ECC9F09DD8DF507AECCFF0DBD4FDD89A
:108A3800D2D8B2ECC9F094D8DF507AECCFF0D2D4C7
:108A480049EC63F0C8D8B2ECC9F08AD8DF507AECA8
:108A5800CFF0C8D4070E0101076F570EBCD8B2EC8F
:108A6800C9F07ED8DF507AECCFF0BCD40D0E136E6F
:108A780075D01150D96EDA6ADF501B0A02E133EF64
:108A880040F0070A02E15CEF40F0010A02E168EFFA
:108A980040F0030A02E175EF40F0010A02E1C9EF74
:108AA80040F03F0A02E1D6EF40F0010A02E1E3EFAD
:108AB80040F0030A02E1F0EF40F0010A02E140EF62
:108AC80041F0070A02E14CEF41F0010A02E159EFD7
:108AD80041F0030A02E165EF41F0010A02E172EF99
:108AE80041F00F0A01E108D4010A01E159D4030A4F
:108AF80001E161D4010A01E16AD4070A01E1A4D5C0
:108B0800010A01E1FAD4030A01E1E3D5010A01E10E
:108B180004D61F0A01E141D6010A01E152D6030A2F
:108B280001E15BD6010A01E162D6070A01E169D6D3
:108B3800010A01E170D6030A01E1B0D6010A01E198
:108B4800F0D60F0A01E130D7010A01E170D7030A14
:108B580001E176D7010A01E17DD788D713501200C9
:108B68001150D96EDA6AD92A12000101076F350E41
:108B78000A6F11C001F0350C0101076F400E0A6F32
:108B8800400C060E0101076F140E0A6F11C001F0A8
:108B9800140C0A6F11C001F0010C070E0101076FD8
:108BA800140E0A6F11C001F0140C060E0101076FB4
:108BB800620E0A6F11C001F0620C0101076F380ED6
:108BC8000A6F11C001F0380C0101076F340E0A6FEB
:108BD80011C001F0040C0A6F11C001F0000C076FFE
:108BE800340E0A6F11C001F0020C0A6F11C001F0B7
:108BF800030C060E0101076F380C070E0101076F01
:108C0800380C0A6F11C001F0020C0101076F320C19
:108C18000A6F11C001F0080C11C001F0010C01012C
:108C2800076F330C11C001F0000C060E0101076F2D
:108C3800100C11C001F0050C11C001F0020C11C09C
:108C480001F0080C11C001F0070C11C001F0060C6E
:108C5800060E0101076F530C11C001F0090C030146
:108C6800922B654B662B0101562B0201532B0301F6
:108C7800912B0101104B112B03013F2B000E4023B8
:108C880041234223390E3F1907E1790E401904E1C7
:108C9800040E411942110AE0730E3F1947E1F20E22
:108CA800401944E1080E4119421140E1610E0201E8
:108CB800D06F310ED16F51ECD0F0000160A536D0E5
:108CC8000301614B622B8A51611962112FE1616BBB
:108CD800626BC90E0201D06F280ED16F51ECD0F033
:108CE8000001618743C21EF144C21FF158A80BD08E
:108CF800360E0201A16F300EA06F320E9F6F300E3C
:108D08009E6F9D6F0BD0360E0201A16F300EA06FC3
:108D1800320E9F6F390E9E6F9D6F300E9C6F9B6F4A
:108D28009A6F060EBE6F000EACECACF0730E03012A
:108D38003F194EE1F20E40194BE1080E411942115C
:108D480047E1370E0201D06F310ED16F51ECD0F0F0
:108D580003013F6B406B416B426B000160B902D06D
:108D680060A736D00301614B622B895161196211EA
:108D78002FE1616B626B6C0E0201D06F290ED16F0F
:108D880051ECD0F00001618743C21EF144C21FF1CB
:108D980058A80BD0360E0201A16F300EA06F320E0C
:108DA8009F6F300E9E6F9D6F0BD0360E0201A16F24
:108DB800300EA06F320E9F6F390E9E6F9D6F300E72
:108DC8009C6F9B6F9A6F060EBE6F000EACECACF0FA
:108DD8004B0E0301911903E1916B0001607FD00EE6
:108DE8000101101905E1070E111902E1106B116B51
:108DF80037ECC8F07C0E010156650BD0566B0E059A
:108E08000F1101E1568E0E510F1103E00E07D8A085
:108E18000F07210503E1216B52ECAFF0215102E16C
:108E280003017B6B0101215101E0210759A212D0F6
:108E3800275101E02707275102E1266B256B030123
:108E48005D515E1103E05D07D8A05E075D515E11BC
:108E580001E1948C01012A5101E02A072A0501E168
:108E68008D9458A808D0502B040E506504D0506B30
:108E7800548811ECCBF003016D07D8A06E076D5133
:108E88006E1102E157AC559E7151721108E07107DD
:108E9800D8A072077151721102E10101546B58A2F6
:108EA80002D08F9040D00201735104E0000160AFFE
:108EB8000DD00FD0000161B560A103D060AB06D022
:108EC80008D061B560B104D061B103D08D9402D0EF
:108ED80061A58D84000161AB12D060AF02D08F8094
:108EE80001D08F90000160AF02D08C8E01D08C9E93
:108EF800000160AF02D08A8C17D08A9C15D003017C
:108F08007751781103E07707D8A0780777057811AB
:108F180001E18F907551761103E07507D8A07607A7
:108F28007505761101E18C9E190E0301921901E075
:108F38008DD0926B0001010E61A3000E0201EA6F51
:108F48000001010E61A5000E0201EA1B5DE00001AF
:108F580061A528D0450E0201D06F2E0ED16F51ECBD
:108F6800D0F043C21EF144C21FF158A80AD0330EF4
:108F7800A16F300EA06F320E9F6F300E9E6F9D6FE7
:108F880009D0380EA16F320EA06F9F6F390E9E6FF9
:108F98009D6F300E9C6F9B6F9A6F060EBE6F100E02
:108FA800ACECACF0000161B528D0DF0E0201D06F47
:108FB8002A0ED16F51ECD0F043C21EF144C21FF10A
:108FC80058A80AD0330EA16F300EA06F320E9F6FD3
:108FD800300E9E6F9D6F09D0380EA16F320EA06FB4
:108FE8009F6F390E9E6F9D6F300E9C6F9B6F9A6FAF
:108FF800070EBE6F100EACECACF0000161A502D0FC
:10900800618302D0000161930101242908E0245101
:1090180001E02407245103E158BAEFEC9CF0020167
:10902800AB51C00BEB6FA8C2ABF2EB51AB1358A816
:1090380003D029ECA2F002D02DEC82F00201A86B3B
:10904800010E03017F6F000E1EECD5F0E80E030140
:10905800651903E1030E6619D8A412000001608D9A
:109068000301656B666B0201A72B3C0EA71902E191
:10907800A62BA76B3C0EA61902E1A52BA66B180E12
:10908800A51901E1A56B00016AAB09D00101406B8C
:10909800412B3B0E41650BD00001648D08D00101C6
:1090A800416B402B3B0E406502D00001649D0001DE
:1090B800010E64AB000E0201EA6F0001010E64ADFF
:1090C800000E0201EA1B14E0000164AD07D0070E90
:1090D8000201DD6F010EDE6FBAEC4FF0000164BDD6
:1090E80007D0080E0201DD6F010EDE6FBAEC4FF0FB
:1090F800000164AD02D0648B02D00001649B0301BF
:10910800942B0001617158A829D00101475126E02C
:10911800472F24D0495116E0010E02015F6F800EDF
:109128005E6FB36BB46B010EEDECC0F0010E5D6FBA
:10913800800E5C6FE8ECCAF00E0EDD6FDE6B010E80
:10914800BAEC4FF00101496B170E0201D06F260EE1
:10915800D16F51ECD0F00101476B456B58A829D06D
:109168000101465126E0462F24D0485116E0010E51
:1091780002015F6F800E5E6FB36BB46B020EEDEC95
:10918800C0F0010E5D6F800E5C6FE8ECCAF00E0E49
:10919800DD6FDE6B010EBAEC4FF00101486B350E46
:1091A8000201D06F260ED16F51ECD0F00101466B51
:1091B800446B58B857AE42D055A810D0000167B9D3
:1091C80007D0080E0201B36F010E91ECA4F006D08F
:1091D800090E0201B36F010E91ECA4F000016AA31D
:1091E8000FD067B707D0080E0201B36F020E91ECDB
:1091F800A4F006D0090E0201B36F020E91ECA4F0A0
:109208000101435101E04307430509E10201796B7C
:10921800B36BB46B010EEDECC0F0E8ECCAF00101E1
:10922800425101E04207420509E10201786BB36B44
:10923800B46B020EEDECC0F0E8ECCAF058A80DD003
:1092480003016F51701109E06F07D8A070076F51C3
:10925800701103E1539E53BC8A9C0301835101E0C2
:10926800830758A815D00101535112E0532F10D08D
:10927800558C51510DE0470E0201D06F2D0ED16F64
:1092880051ECD0F00E0EDD6FDE6B010EBAEC4FF034
:1092980003015F51601103E05F07D8A060075F51C9
:1092A800601102E18B908B9259A057D001013D517A
:1092B80006E1000161A102D08C8E01D08C9E0101D3
:1092C800365101E03607360501E13D6B3C513D1949
:1092D80044E03DC13CF13D511EE1360E0201D06F24
:1092E8002E0ED16F51ECD0F043C21EF144C21FF1D3
:1092F800380EA16F330EA06F9F6F390E9E6F9D6F52
:10930800300E9C6F320E9B6F300E9A6F060EBE6F3A
:10931800100EACECACF001013D051FE18C9E0A0E6D
:109328000201D06F2C0ED16F51ECD0F043C21EF168
:1093380044C21FF1380EA16F330EA06F9F6F390E14
:109348009E6F9D6F300E9C6F320E9B6F300E9A6F22
:10935800070EBE6F100EACECACF058A65FD059B635
:1093680006D0000161A102D08C8E01D08C9E010133
:10937800365101E03607360501E15996010E59A428
:10938800000E0201EA6F010E59A6000EEA1B46E024
:1093980059A602D0598401D0599459B61ED0A80EA6
:1093A8000201D06F2E0ED16F51ECD0F043C21EF1E6
:1093B80044C21FF1380EA16F330EA06F9F6F390E94
:1093C8009E6F9D6F300E9C6F320E9B6F300E9A6FA2
:1093D800060EBE6F100EACECACF059A61FD08C9EDA
:1093E800250E0201D06F2D0ED16F51ECD0F043C283
:1093F8001EF144C21FF1380EA16F330EA06F9F6F8C
:10940800390E9E6F9D6F300E9C6F320E9B6F300E23
:109418009A6F070EBE6F100EACECACF03C0E030159
:10942800941901E0E1D0946B510E0201D06F2A0E1D
:10943800D16F51ECD0F00101590519E102019951A0
:1094480009E09907170EB66F270EB56F99C2B7F2E4
:1094580067ECC8F0F60E0201D06F240ED16F51EC04
:10946800D0F00101596B0E6B0F6B0201966B010175
:10947800595101E0590758A85DD00201652B655183
:109488000A0D400EF324D96E040EF420DA6E110E84
:10949800DF6E65510A0D410EF324D96E040EF420D7
:1094A800DA6EDF6865510A0D420EF324D96E040E98
:1094B800F420DA6EDF6865510A0D430EF324D96E85
:1094C800040EF420DA6EDF6865510A0D440EF324A9
:1094D800D96E040EF420DA6EDF6865510A0D450E68
:1094E800F324D96E040EF420DA6EDF6865510A0D94
:1094F800460EF324D96E040EF420DA6EDF68655147
:109508000A0D470EF324D96E040EF420DA6EDF68D4
:1095180065510A0D480EF324D96E040EF420DA6E54
:10952800DF6865510A0D490EF324D96E040EF42044
:10953800DA6EDF68010E0201EC6F060EEC6501D0F1
:109548002CD0280EEC25D96EDA6A030EDA22DF2A2F
:10955800280EEC25D96EDA6A030EDA2201015B5176
:10956800DE1818E1210E0201EC25D96EDA6A030E25
:10957800DA22DF6A280EEC25D96EDA6A030EDA22BF
:10958800DF6AE10ED06F280ED16FECC2D2F2D36B36
:1095980051ECD0F00201EC2BD0D70301902B0F0E29
:1095A800901922E1F00E010157650BD0680E0201F7
:1095B800D06F280ED16F51ECD0F00301646B500EC0
:1095C800636F140E010157610BD0820E0201D06F38
:1095D800290ED16F51ECD0F02BC163F30301646BFA
:1095E8000301906B0101576B0301932B050E93192F
:1095F800D8A4120058A204D08D84640E01012A6FE9
:109608000301936B120000016AA547D057AE0BD037
:10961800230E02013F19401106E1050E0301F76F01
:10962800020EE6ECA0F002013F07D8A040073F5128
:10963800401101E04AD200016A955582060E0301E5
:10964800F76F020EE6ECA0F0000169AB04D0699F49
:1096580069AD698F699D02018D6B960E8E6F885179
:1096680001E133D2000169AF0BD0090E0501F96F92
:10967800020188050501FA6F020EADEC32F00AD03E
:10968800030E0501F96F020188050501FA6F020E44
:10969800ADEC32F00201886B18D26AA316D257AE2D
:1096A80008D00101195105E1230E185D02E20001FD
:1096B800678701011807D8A019071851191101E087
:1096C80004D200016A936797060E0301F76F020E32
:1096D800E6ECA0F000016A81D60E0501E86F210EC4
:1096E800E96F1DECD0F00201850523E15AA121D0D4
:1096F800140E0501E86F310EE96F1DECD0F0010E74
:10970800F96FFA6F020EADEC32F000016B8B69B99C
:1097180010D0140E0501E86F310EE96F1DECD0F082
:10972800020EF96F010EFA6F020EADEC32F0000175
:109738006B9B0201840521E15AA31FD0140E050179
:10974800E86F310EE96F1DECD0F0010EF96F020ED3
:10975800FA6FADEC32F000016B8969B50ED0140ECA
:109768000501E86F310EE96F1DECD0F0020EF96FBC
:10977800FA6FADEC32F000016B990201830524E128
:109788005AA522D0140E0501E86F310EE96F1DECC1
:10979800D0F0010EF96F030EFA6F020EADEC32F045
:1097A80000016B8768BF10D0140E0501E86F310EF9
:1097B800E96F1DECD0F0020EF96F030EFA6F020E7E
:1097C800ADEC32F000016B970201820524E15AA743
:1097D80022D0140E0501E86F310EE96F1DECD0F0B0
:1097E800010EF96F040EFA6F020EADEC32F00001B3
:1097F8006B8568BB10D0140E0501E86F310EE96F58
:109808001DECD0F0020EF96F040EFA6F020EADECEB
:1098180032F000016B950201810524E15AA922D09A
:10982800140E0501E86F310EE96F1DECD0F0010E42
:10983800F96F050EFA6F020EADEC32F000016B8382
:1098480068B710D0140E0501E86F310EE96F1DECF2
:10985800D0F0020EF96F050EFA6F020EADEC32F081
:1098680000016B930201800524E15AAB22D0140E4B
:109878000501E86F310EE96F1DECD0F0010EF96FAC
:10988800060EFA6F020EADEC32F000016B8168B380
:1098980010D0140E0501E86F310EE96F1DECD0F001
:1098A800020EF96F060EFA6F020EADEC32F00001EF
:1098B8006B9102017F0524E15AAD22D0140E0501F7
:1098C800E86F310EE96F1DECD0F0010EF96F070E4D
:1098D800FA6F020EADEC32F000016A8F67BF10D04C
:1098E800140E0501E86F310EE96F1DECD0F0020E81
:1098F800F96F070EFA6F020EADEC32F000016A9FA5
:1099080002017E0524E15AAF22D0140E0501E86F4A
:10991800310EE96F1DECD0F0010EF96F080EFA6FE9
:10992800020EADEC32F000016A8D67BB10D0140E48
:109938000501E86F310EE96F1DECD0F0020EF96FEA
:10994800080EFA6F020EADEC32F000016A9D0001BC
:1099580069A714D002015AA111D000016997F50E28
:109968000501E86F2F0EE96F1DECD0F0010EF96FBD
:10997800FA6F020EADEC32F000016B8B000169A3A7
:1099880014D002015AA311D000016993F50E050104
:10999800E86F2F0EE96F1DECD0F0010EF96F020E83
:1099A800FA6FADEC32F000016B89000169A115D0A6
:1099B80002015AA512D000016991F50E0501E86F60
:1099C8002F0EE96F1DECD0F0010EF96F030EFA6F40
:1099D800020EADEC32F000016B87000168AD15D0C6
:1099E80002015AA712D00001689DF50E0501E86F23
:1099F8002F0EE96F1DECD0F0010EF96F040EFA6F0F
:109A0800020EADEC32F000016B85000168A915D09B
:109A180002015AA912D000016899F50E0501E86FF4
:109A28002F0EE96F1DECD0F0010EF96F050EFA6FDD
:109A3800020EADEC32F000016B83000168A515D071
:109A480002015AAB12D000016895F50E0501E86FC6
:109A58002F0EE96F1DECD0F0010EF96F060EFA6FAC
:109A6800020EADEC32F000016B81000168A115D047
:109A780002015AAD12D000016891F50E0501E86F98
:109A88002F0EE96F1DECD0F0010EF96F070EFA6F7B
:109A9800020EADEC32F000016A8F000167AD15D0FF
:109AA80002015AAF12D00001679DF50E0501E86F5B
:109AB8002F0EE96F1DECD0F0010EF96F080EFA6F4A
:109AC800020EADEC32F000016A8D55A646D057AEB5
:109AD8000BD0230E02014119421106E1050E0301C4
:109AE800F76F010EE6ECA0F002014107D8A042078B
:109AF80041514211D8A4120055965584060E03010F
:109B0800F76F010EE6ECA0F054A604D0549454A2CA
:109B18005484549202018D6B960E8E6F8951D8B47D
:109B2800120054A40BD0090E0501F96F0201890532
:109B38000501FA6F010EADEC32F00AD0030E0501F3
:109B4800F96F020189050501FA6F010EADEC32F0DB
:109B58000201896B010E87EF2BF055A8120057AE52
:109B680008D001011B5105E1230E1A5D02E2000134
:109B7800678901011A07D8A01B071A511B11D8A41D
:109B88001200559800016799060E0301F76F010E40
:109B9800E6ECA0F000016C8DD90E0501E86F210EEE
:109BA800E96F1DECD0F00201850521E15BA11FD012
:109BB800140E0501E86F310EE96F1DECD0F0010EAF
:109BC800F96FFA6FADEC32F000016C8B52BA0FD01E
:109BD800140E0501E86F310EE96F1DECD0F0020E8E
:109BE800F96F010EFA6FADEC32F000016C9B0201C7
:109BF800840523E15BA321D0140E0501E86F310E23
:109C0800E96F1DECD0F0010EF96F020EFA6F010E2C
:109C1800ADEC32F000016C8952B80FD0140E05017A
:109C2800E86F310EE96F1DECD0F0020EF96FFA6F94
:109C3800010EADEC32F000016C990201830524E1BC
:109C48005BA522D0140E0501E86F310EE96F1DECFB
:109C5800D0F0010EF96F030EFA6F010EADEC32F081
:109C680000016C8752B610D0140E0501E86F310E52
:109C7800E96F1DECD0F0020EF96F030EFA6F010EBA
:109C8800ADEC32F000016C970201820524E15BA77C
:109C980022D0140E0501E86F310EE96F1DECD0F0EB
:109CA800010EF96F040EFA6F010EADEC32F00001EF
:109CB8006C8552B410D0140E0501E86F310EE96FAF
:109CC8001DECD0F0020EF96F040EFA6F010EADEC28
:109CD80032F000016C950201810524E15BA922D0D4
:109CE800140E0501E86F310EE96F1DECD0F0010E7E
:109CF800F96F050EFA6F010EADEC32F000016C83BE
:109D080052B210D0140E0501E86F310EE96F1DEC48
:109D1800D0F0020EF96F050EFA6F010EADEC32F0BD
:109D280000016C930201800524E15BAB22D0140E84
:109D38000501E86F310EE96F1DECD0F0010EF96FE7
:109D4800060EFA6F010EADEC32F000016C8152B0D4
:109D580010D0140E0501E86F310EE96F1DECD0F03C
:109D6800020EF96F060EFA6F010EADEC32F000012B
:109D78006C9102017F0524E15BAD22D0140E050130
:109D8800E86F310EE96F1DECD0F0010EF96F070E88
:109D9800FA6F010EADEC32F000016B8F6DB510D08B
:109DA800140E0501E86F310EE96F1DECD0F0020EBC
:109DB800F96F070EFA6F010EADEC32F000016B9FE0
:109DC80002017E0524E15BAF22D0140E0501E86F85
:109DD800310EE96F1DECD0F0010EF96F080EFA6F25
:109DE800010EADEC32F000016B8D6DB310D0140E86
:109DF8000501E86F310EE96F1DECD0F0020EF96F26
:109E0800080EFA6F010EADEC32F000016B9D53AAFB
:109E180012D002015BA10FD0539AF50E0501E86F2D
:109E28002F0EE96F1DECD0F0010EF96FFA6FADEC53
:109E380032F000016C8B53A814D002015BA311D03F
:109E48005398F50E0501E86F2F0EE96F1DECD0F061
:109E5800010EF96F020EFA6F010EADEC32F000013F
:109E68006C8953A614D002015BA511D05396F50E48
:109E78000501E86F2F0EE96F1DECD0F0010EF96FA8
:109E8800030EFA6F010EADEC32F000016C8753A49B
:109E980014D002015BA711D05394F50E0501E86FA9
:109EA8002F0EE96F1DECD0F0010EF96F040EFA6F5A
:109EB800010EADEC32F000016C8553A214D0020102
:109EC8005BA911D05392F50E0501E86F2F0EE96FCB
:109ED8001DECD0F0010EF96F050EFA6F010EADEC16
:109EE80032F000016C8353A014D002015BAB11D097
:109EF8005390F50E0501E86F2F0EE96F1DECD0F0B9
:109F0800010EF96F060EFA6F010EADEC32F000018A
:109F18006C8152AE14D002015BAD11D0529EF50E89
:109F28000501E86F2F0EE96F1DECD0F0010EF96FF7
:109F3800070EFA6F010EADEC32F000016B8F52ACD8
:109F4800120002015BAF1200529CF50E0501E86F8A
:109F58002F0EE96F1DECD0F0010EF96F080EFA6FA5
:109F6800010EADEC32F000016B8D1200E76F0201BB
:109F7800E70501E101D225D20F0ED06F240ED9ECEE
:109F880053F051ECD0F0538E53BC8A8C86513C0D63
:109F9800F3CF6FF3F4CF70F300016785C4EC5CF086
:109FA800A5EC5CF0F3EC53F0ACECACF010D079819C
:109FB80020D079831ED079851CD079871AD07989E9
:109FC80018D0798B16D0798D14D0798F12D00201E0
:109FD800DE51010AECE0030AECE0010AECE0070AB2
:109FE800ECE0010AECE0030AECE0010AECE00F0AFD
:109FF800ECE027EC54F0EDECC0F0E3D1390ED06F73
:10A00800230ED3DB51ECD0F0310ED2EC5CF0C5DB83
:10A01800A5EC5CF0EFDBACECACF0D3D1000166AFA3
:10A0280003D00201DE0531E0000166AD04D0020E66
:10A038000201DE192AE0000166AB04D0030E02011A
:10A04800DE1923E0000166A904D0040E0201DE191E
:10A058001CE0000166A704D0050E0201DE1915E018
:10A06800000166A504D0060E0201DE190EE000010B
:10A0780066A304D0070E0201DE1907E0000166A1FD
:10A0880019D0080E0201DE1915E1330EA16FDAECC2
:10A098002AF09F6F300E9E6F310EA5EC5CF09FDBAF
:10A0A800ACECACF02C0E0201D06F240E7EDB51EC30
:10A0B800D0F087D175DB71DBA5EC5CF090DBACEC04
:10A0C800ACF0538EAAEC5CF00001678510D0798162
:10A0D80020D079831ED079851CD079871AD07989C8
:10A0E80018D0798B16D0798D14D0798F12D00201BF
:10A0F800DE51010AECE0030AECE0010AECE0070A91
:10A10800ECE0010AECE0030AECE0010AECE00F0ADB
:10A11800ECE099DBEDECC0F00A0ED06F240E45DBC5
:10A1280051ECD0F04ED1000166AF03D00201DE053C
:10A1380031E0000166AD04D0020E0201DE192AE00A
:10A14800000166AB04D0030E0201DE1923E0000112
:10A1580066A904D0040E0201DE191CE0000166A7FE
:10A1680004D0050E0201DE1915E0000166A504D031
:10A17800060E0201DE190EE0000166A304D0070EE8
:10A188000201DE1907E0000166A125D0080E0201D0
:10A19800DE1921E1000166BF669F66BD669D66BB4C
:10A1A800669B66B9669966B7669766B5669566B33F
:10A1B800669366B16691B4EC5CF0310EA5EC5CF088
:10A1C80019DBACECACF0820E0201D06F210EEDDA97
:10A1D80051ECD0F0F6D0E4DAE0DAA5EC5CF00ADB7A
:10A1E800ACECACF0340E0201D06F230EDEDA51EC89
:10A1F800D0F0E7D0330EB5DA9D6F02DBBE6F000EEC
:10A20800ACECACF0B40E0201D06F240ECEDA51ECF7
:10A21800D0F0D7D0330EA5DAFBDABE6F000EACEC67
:10A22800ACF0C40E0201D06F230EBFDA51ECD0F0AF
:10A23800C8D0EF0ED06F220EB8DA51ECD0F05E9194
:10A24800F5DADEECC4F00109DF6FE7DADFC2B7F256
:10A2580067ECC8F0F0DACCECCFF08BDA82DAAADA65
:10A26800FBDAACECACF0ADD0EA0ED06F220E9DDA82
:10A2780051ECD0F0FEDADADADEECC4F00209E06F75
:10A28800CCDAE0C2B7F267ECC8F0D5DACCECCFF0A4
:10A2980070DA9ADA8FDAE0DAACECACF092D0050E2C
:10A2A800D06F220E82DA51ECD0F05E93BFDADEEC8A
:10A2B800C4F0FC0BE16FB1DAE1C2B7F267ECC8F0A9
:10A2C800BADACCECCFF055DA4CDA74DAB9DAACECAD
:10A2D800ACF077D0000ED06F220E67DA51ECD0F0D8
:10A2E800F50E5E17A3DADEECC4F0FC0BE26F95DA2C
:10A2F800E2C2B7F267ECC8F09EDACCECCFF039DAFC
:10A3080063DA58DA9DDAACECACF05BD08BDA3BDA86
:10A3180066DAACECACF0590E0201D06F250E45DAC6
:10A3280051ECD0F04ED07EDA2EDA64DAACECACF038
:10A33800920E0201D06F240E38DA51ECD0F041D0E1
:10A348009DDA370E20DA60DAACECACF02D0E0201A3
:10A35800D06F2A0ED16F51ECD0F033D08FDA380E8F
:10A3680012DA52DAACECACF0C40E0201D06F290E4E
:10A37800D16F51ECD0F025D0DD51010A01E1FCD5B7
:10A38800030A01E13BD6010A01E153D7070A87E036
:10A39800010A01E143D6030A01E1C5D6010A01E138
:10A3A80029D70F0A01E136D7010A01E15DD7030A6F
:10A3B80091E0010AABE0070AB6E0010AC1E0030A2E
:10A3C800CDE0020E0201E71901E1AFD11200530EF0
:10A3D800D06F240EEAD951ECD0F0FDD9AAEC5CF08C
:10A3E80004DAD8D9A5EC5CF0FAD9ACECACF010D012
:10A3F800788120D078831ED078851CD078871AD0B1
:10A40800788918D0788B16D0788D14D0788F12D0A0
:10A418000201DE51010AECE0030AECE0010AECE07B
:10A42800070AECE0010AECE0030AECE0010AECE0C0
:10A438000F0AECE018DAEDEFC0F05D0ED06F230ED6
:10A44800B4D951ECD0F0D1D9A5D9A5EC5CF0DE5146
:10A45800300F9A6F2FD1000165AF03D00201DE05DE
:10A4680031E0000165AD04D0020E0201DE192AE0D8
:10A47800000165AB04D0030E0201DE1923E00001E0
:10A4880065A904D0040E0201DE191CE0000165A7CD
:10A4980004D0050E0201DE1915E0000165A504D0FF
:10A4A800060E0201DE190EE0000165A304D0070EB6
:10A4B8000201DE1907E0000165A116D0080E0201AD
:10A4C800DE1912E1330EA16FDAEC2AF09F6F300E1D
:10A4D8009E6F320EA5EC5CF082D9ACECACF0700E3D
:10A4E8000201D06F240EAFD05BD954D9A5EC5CF033
:10A4F80076D9ACECACF0538EAAEC5CF00001678323
:10A5080010D0788120D078831ED078851CD07887A9
:10A518001AD0788918D0788B16D0788D14D0788F87
:10A5280012D00201DE51010AECE0030AECE0010A54
:10A53800ECE0070AECE0010AECE0030AECE0010AAF
:10A54800ECE00F0AECE08FD9EDECC0F04E0ED06FC6
:10A55800240E79D0000165AF03D00201DE0531E099
:10A56800000165AD04D0020E0201DE192AE00001E7
:10A5780065AB04D0030E0201DE1923E0000165A9D2
:10A5880004D0040E0201DE191CE0000165A704D006
:10A59800050E0201DE1915E0000165A504D0060EBE
:10A5A8000201DE190EE0000165A304D0070E0201C6
:10A5B800DE1907E0000165A122D0080E0201DE19AC
:10A5C8001EE1000165BF659F65BD659D65BB659B17
:10A5D80065B9659965B7659765B5659565B365931B
:10A5E80065B16591B4EC5CF0320EA5EC5CF002D973
:10A5F800ACECACF0AC0E0201D06F210E24D0D0D858
:10A60800C9D8A5EC5CF0F6D8ACECACF0580E020159
:10A61800D06F230E18D0330EA4D89D6FF1D8BE6F1B
:10A62800000EACECACF0D50E0201D06F240E0BD0AE
:10A63800330E97D8EDD8BE6F000EACECACF0E70E39
:10A648000201D06F230EB1D851EFD0F0140ED06FA5
:10A65800230EABD851ECD0F05C9115D9CCECCFF0EF
:10A6680088D87FD8ACD8F8D8ACECACF0170E02017B
:10A67800F6D8DEECC4F00409E36FCFD8E3C2B7F232
:10A6880067EFC8F00F0ED06F230E8FD851ECD0F0C3
:10A698005C915C87CBD8DEECC4F00809E46FBDD8C8
:10A6A800E4C2B7F267ECC8F0C6D8CCECCFF061D8FA
:10A6B8008BD885D8070E35D02D0ED06F220E75D8C1
:10A6C80051ECD0F05C93DFD8CCECCFF052D849D81D
:10A6D80076D8B6D8ACECACF0170E0201C0D8DEECD8
:10A6E800C4F0F30BE56F99D8E5C2B7F267EFC8F08D
:10A6F800280ED06F220E59D851ECD0F0F50E5C1709
:10A7080095D8DEECC4F0F30BE66F87D8E6C2B7F253
:10A7180067ECC8F090D8CCECCFF02BD855D84FD8F0
:10A72800060EBE6F000EACEFACF0DD51010A01E180
:10A738004ED6030A01E181D6010A88E0070ABCE087
:10A74800010A01E188D6030A01E104D7010A01E1FF
:10A7580062D70F0A01E16CD7010A94E0030AC8E046
:10A768001200A16F300EA06F310E9F6F300E9E6FDA
:10A77800300C9B6F9B51F60DF350DE259A6F300E0F
:10A788009A279B27340C9F6F300E9E6F9D6F9C6F8E
:10A798009B6F300C9F6F9E6F320C9F6F9E6F310CBA
:10A7A800310E0201A16FA06F300CD16FDEC2D2F260
:10A7B800D36B1200310E9D6F300E9C6F300C320E31
:10A7C8009D6F300E9C6F300CA16FA06F310E9F6F84
:10A7D800300E9E6F300C538E000167831200DE51DD
:10A7E800300F9A6F060EBE6F000C310EA16F330E3C
:10A7F800A06F300CDE51300F9A6F070EBE6F000C41
:10A808009C6F9B6F9A6F060C9A6F060EBE6F000CBA
:10A818009D6F9C6F9B6F9A6F070C170EB66F030E98
:10A82800B56F030C330EA16FA06F330C170EB76F03
:10A83800030EB66F030C0A0E0201B36FDE5112004D
:10A84800060EBE6F000C110E5F6F0401426F02010D
:10A85800B36B79C2B4F2010C070EBE6F000CB76F70
:10A86800030EB66F030C110E5D6FB36B78C2B4F2B2
:10A87800020C5E915E875EC241F41200360EA16F33
:10A88800320EA06F320C0A0EB36FDE5112000001B7
:10A898006AA541D057AE0AD0230E02013F194011D4
:10A8A80005E1050E016E020EA1EC9FF002013F07C3
:10A8B800D8A040073F51401101E02BD200016A9512
:10A8C8005582060E016E020EA1EC9FF0000169ABE5
:10A8D80004D0699F69AD698F699D02018D6B960EE1
:10A8E8008E6F885101E115D2000169AF09D0090EB8
:10A8F800396E020188053A6E020EBCEC58F008D099
:10A90800030E396E020188053A6E020EBCEC58F04F
:10A918000201886BFED16AA3FCD157AE08D00101B1
:10A92800195105E1230E185D02E200016787010154
:10A938001807D8A019071851191101E0EAD1000128
:10A948006A936797060E016E020EA1EC9FF0000154
:10A958006A81D60E1E6E210E1F6ED1ECD0F0020158
:10A96800850521E15AA11FD0140E1E6E310E1F6EEF
:10A97800D1ECD0F0010E396E3A6E020EBCEC58F0F4
:10A9880000016B8B69B90FD0140E1E6E310E1F6E4D
:10A99800D1ECD0F0020E396E010E3A6E020EBCEC0C
:10A9A80058F000016B9B020184051FE15AA31DD0DA
:10A9B800140E1E6E310E1F6ED1ECD0F0010E396EE2
:10A9C800020E3A6EBCEC58F000016B8969B50DD0E7
:10A9D800140E1E6E310E1F6ED1ECD0F0020E396EC1
:10A9E8003A6EBCEC58F000016B990201830522E134
:10A9F8005AA520D0140E1E6E310E1F6ED1ECD0F069
:10AA0800010E396E030E3A6E020EBCEC58F00001CE
:10AA18006B8768BF0FD0140E1E6E310E1F6ED1ECFF
:10AA2800D0F0020E396E030E3A6E020EBCEC58F0EE
:10AA380000016B970201820522E15AA720D0140E6B
:10AA48001E6E310E1F6ED1ECD0F0010E396E040E61
:10AA58003A6E020EBCEC58F000016B8568BB0FD053
:10AA6800140E1E6E310E1F6ED1ECD0F0020E396E30
:10AA7800040E3A6E020EBCEC58F000016B95020110
:10AA8800810522E15AA920D0140E1E6E310E1F6EC8
:10AA9800D1ECD0F0010E396E050E3A6E020EBCEC08
:10AAA80058F000016B8368B70FD0140E1E6E310E7C
:10AAB8001F6ED1ECD0F0020E396E050E3A6E020E02
:10AAC800BCEC58F000016B930201800522E15AABFF
:10AAD80020D0140E1E6E310E1F6ED1ECD0F0010E78
:10AAE800396E060E3A6E020EBCEC58F000016B810E
:10AAF80068B30FD0140E1E6E310E1F6ED1ECD0F05D
:10AB0800020E396E060E3A6E020EBCEC58F00001C9
:10AB18006B9102017F0522E15AAD20D0140E1E6E02
:10AB2800310E1F6ED1ECD0F0010E396E070E3A6E61
:10AB3800020EBCEC58F000016A8F67BF0FD0140EEC
:10AB48001E6E310E1F6ED1ECD0F0020E396E070E5C
:10AB58003A6E020EBCEC58F000016A9F02017E05B5
:10AB680022E15AAF20D0140E1E6E310E1F6ED1ECAA
:10AB7800D0F0010E396E080E3A6E020EBCEC58F099
:10AB880000016A8D67BB0FD0140E1E6E310E1F6E4A
:10AB9800D1ECD0F0020E396E080E3A6E020EBCEC03
:10ABA80058F000016A9D000169A713D002015AA15B
:10ABB80010D000016997F50E1E6E2F0E1F6ED1EC96
:10ABC800D0F0010E396E3A6E020EBCEC58F000015E
:10ABD8006B8B000169A313D002015AA310D00001A6
:10ABE8006993F50E1E6E2F0E1F6ED1ECD0F0010E7C
:10ABF800396E020E3A6EBCEC58F000016B89000108
:10AC080069A114D002015AA511D000016991F50E6D
:10AC18001E6E2F0E1F6ED1ECD0F0010E396E030E92
:10AC28003A6E020EBCEC58F000016B87000168AD6B
:10AC380014D002015AA711D00001689DF50E1E6EAE
:10AC48002F0E1F6ED1ECD0F0010E396E040E3A6E45
:10AC5800020EBCEC58F000016B85000168A914D005
:10AC680002015AA911D000016899F50E1E6E2F0E27
:10AC78001F6ED1ECD0F0010E396E050E3A6E020E41
:10AC8800BCEC58F000016B83000168A514D00201E8
:10AC98005AAB11D000016895F50E1E6E2F0E1F6E6F
:10ACA800D1ECD0F0010E396E060E3A6E020EBCECF5
:10ACB80058F000016B81000168A114D002015AAD5F
:10ACC80011D000016891F50E1E6E2F0E1F6ED1EC8B
:10ACD800D0F0010E396E070E3A6E020EBCEC58F039
:10ACE80000016A8F000167AD14D002015AAF11D07C
:10ACF8000001679DF50E1E6E2F0E1F6ED1ECD0F071
:10AD0800010E396E080E3A6E020EBCEC58F00001C6
:10AD18006A8D55A63ED057AE0AD0230E02014119BE
:10AD2800421105E1050E016E010EA1EC9FF0020132
:10AD38004107D8A0420741514211D8A412005596A4
:10AD48005584060E016E010EA1EC9FF054A604D0A6
:10AD5800549454A25484549202018D6B960E8E6FB3
:10AD68008951D8B4120054A408D0090E396E890547
:10AD78003A6E010EBCEC58F007D0030E396E890507
:10AD88003A6E010EBCEC58F00201896B010E89EF96
:10AD980039F055A8120057AE08D001011B5105E142
:10ADA800230E1A5D02E20001678901011A07D8A083
:10ADB8001B071A511B11D8A4120055980001679956
:10ADC800060E016E010EA1EC9FF000016C8DD90EEC
:10ADD8001E6E210E1F6ED1ECD0F0020185051FE119
:10ADE8005BA11DD0140E1E6E310E1F6ED1ECD0F07B
:10ADF800010E396E3A6EBCEC58F000016C8B52BAF9
:10AE08000ED0140E1E6E310E1F6ED1ECD0F0020E55
:10AE1800396E010E3A6EBCEC58F000016C9B0201D1
:10AE2800840521E15BA31FD0140E1E6E310E1F6E28
:10AE3800D1ECD0F0010E396E020E3A6E010EBCEC68
:10AE480058F000016C8952B80ED0140E1E6E310EE7
:10AE58001F6ED1ECD0F0020E396E3A6E010EBCECCA
:10AE680058F000016C990201830522E15BA520D00E
:10AE7800140E1E6E310E1F6ED1ECD0F0010E396E1D
:10AE8800030E3A6E010EBCEC58F000016C8752B606
:10AE98000FD0140E1E6E310E1F6ED1ECD0F0020EC4
:10AEA800396E030E3A6E010EBCEC58F000016C9737
:10AEB8000201820522E15BA720D0140E1E6E310E1E
:10AEC8001F6ED1ECD0F0010E396E040E3A6E010EF1
:10AED800BCEC58F000016C8552B40FD0140E1E6EF5
:10AEE800310E1F6ED1ECD0F0020E396E040E3A6EA0
:10AEF800010EBCEC58F000016C950201810522E1BD
:10AF08005BA920D0140E1E6E310E1F6ED1ECD0F04E
:10AF1800010E396E050E3A6E010EBCEC58F00001B8
:10AF28006C8352B20FD0140E1E6E310E1F6ED1EC10
:10AF3800D0F0020E396E050E3A6E010EBCEC58F0D8
:10AF480000016C930201800522E15BAB20D0140E56
:10AF58001E6E310E1F6ED1ECD0F0010E396E060E4A
:10AF68003A6E010EBCEC58F000016C8152B00FD063
:10AF7800140E1E6E310E1F6ED1ECD0F0020E396E1B
:10AF8800060E3A6E010EBCEC58F000016C910201FD
:10AF98007F0522E15BAD20D0140E1E6E310E1F6EB0
:10AFA800D1ECD0F0010E396E070E3A6E010EBCECF2
:10AFB80058F000016B8F6DB50FD0140E1E6E310E58
:10AFC8001F6ED1ECD0F0020E396E070E3A6E010EEC
:10AFD800BCEC58F000016B9F02017E0522E15BAFDB
:10AFE80020D0140E1E6E310E1F6ED1ECD0F0010E63
:10AFF800396E080E3A6E010EBCEC58F000016B8DEC
:10B008006DB30FD0140E1E6E310E1F6ED1ECD0F042
:10B01800020E396E080E3A6E010EBCEC58F00001B3
:10B028006B9D53AA11D002015BA10ED0539AF50E65
:10B038001E6E2F0E1F6ED1ECD0F0010E396E3A6ED7
:10B04800BCEC58F000016C8B53A813D002015BA331
:10B0580010D05398F50E1E6E2F0E1F6ED1ECD0F047
:10B06800010E396E020E3A6E010EBCEC58F000016A
:10B078006C8953A613D002015BA510D05396F50E28
:10B088001E6E2F0E1F6ED1ECD0F0010E396E030E1E
:10B098003A6E010EBCEC58F000016C8753A413D033
:10B0A80002015BA710D05394F50E1E6E2F0E1F6E73
:10B0B800D1ECD0F0010E396E040E3A6E010EBCECE4
:10B0C80058F000016C8553A213D002015BA910D07F
:10B0D8005392F50E1E6E2F0E1F6ED1ECD0F0010E9E
:10B0E800396E050E3A6E010EBCEC58F000016C8307
:10B0F80053A013D002015BAB10D05390F50E1E6E17
:10B108002F0E1F6ED1ECD0F0010E396E060E3A6E7E
:10B11800010EBCEC58F000016C8152AE13D0020154
:10B128005BAD10D0529EF50E1E6E2F0E1F6ED1EC29
:10B13800D0F0010E396E070E3A6E010EBCEC58F0D5
:10B1480000016B8F52AC120002015BAF1200529CDF
:10B15800F50E1E6E2F0E1F6ED1ECD0F0010E396E5B
:10B16800080E3A6E010EBCEC58F000016B8D12000F
:10B17800436E430401E1F2D117D20F0E1E6E240E66
:10B18800CDEC5CF0D1ECD0F0538EE0DB00016785AC
:10B19800F7DBD7DBD6EC5CF05EECADF018D0020143
:10B1A800798126D00201798323D00201798520D0C4
:10B1B800020179871DD0020179891AD00201798BA1
:10B1C80017D00201798D14D00201798F11D03A502D
:10B1D800010AE5E0030AE6E0010AE7E0070AE8E019
:10B1E800010AE9E0030AEAE0010AEBE00F0AECE0F1
:10B1F800F3DB2FECB7F0D8D1390E1E6E230EC9DB66
:10B20800D1ECD0F0BDDB9DDBD3DB5EECADF0CCD177
:10B21800000166AF02D03A0423E066AD03D0020E07
:10B228003A181EE066AB03D0030E3A1819E066A977
:10B2380003D0040E3A1814E066A703D0050E3A1896
:10B248000FE066A503D0060E3A180AE066A303D0FD
:10B25800070E3A1805E066A110D0080E3A180DE15D
:10B268007FDB310E6EDB9EDB5EECADF02C0E1E6ECE
:10B27800240E8FDBD1ECD0F097D1D4EC53F0D1EC85
:10B2880053F05FDB8FDB5EECADF0538E5FDB0001CC
:10B29800678518D00201798126D00201798323D0ED
:10B2A8000201798520D0020179871DD002017989B0
:10B2B8001AD00201798B17D00201798D14D00201BE
:10B2C800798F11D03A50010AE5E0030AE6E0010A55
:10B2D800E7E0070AE8E0010AE9E0030AEAE0010A10
:10B2E800EBE00F0AECE078DB2FECB7F00A0E1E6EED
:10B2F800240E4FDBD1ECD0F057D1000166AF02D05D
:10B308003A0423E066AD03D0020E3A181EE066AB9D
:10B3180003D0030E3A1819E066A903D0040E3A18B0
:10B3280014E066A703D0050E3A180FE066A503D00F
:10B33800060E3A180AE066A303D0070E3A1805E08D
:10B3480066A120D0080E3A181DE166BF669F66BD4B
:10B35800669D66BB669B66B9669966B7669766B56D
:10B36800669566B3669366B16691FADA310EE9DAE4
:10B378001FDB5EECADF0820E1E6E210E0ADBD1ECF7
:10B38800D0F012D1D4EC53F0D1EC53F0DADA10DB70
:10B398005EECADF0340E1E6E230EFBDAD1ECD0F06D
:10B3A80003D1330E0201B5EC53F09D6F04EC54F059
:10B3B800126E000E5EECADF0B40E1E6E240EE9DACD
:10B3C800D1ECD0F0F1D0330E0201B5EC53F00CEC17
:10B3D80054F0126E000E5EECADF0C40E1E6E230E1D
:10B3E800D8DAD1ECD0F0E0D0EF0E1E6E220ED1DA12
:10B3F800D1ECD0F002015E91EADAA2ECC6F00109C4
:10B408003B6EE0DA3BC00DF00DECCAF0FBDA6BECFA
:10B41800D0F08CDAB5EC53F0DEEC53F0E9DA5EEC00
:10B42800ADF0C2D0EA0E1E6E220EB3DAD1ECD0F027
:10B4380002013DEC54F0CBDAA2ECC6F002093C6EF6
:10B44800C1DA3CC00DF00DECCAF0DCDA6BECD0F0E0
:10B458006DDAE8EC53F0DEEC53F0CADA5EECADF0EE
:10B46800A3D0050E1E6E220E94DAD1ECD0F00201A4
:10B478005E93ADDAA2ECC6F0FC0B3D6EA3DA3DC0DC
:10B488000DF00DECCAF0BEDA6BECD0F04FDAB5EC8B
:10B4980053F0DEEC53F0A9DA5EECADF085D0000E87
:10B4A8001E6E220E76DAD1ECD0F0F50E02015E1790
:10B4B8008EDAA2ECC6F0FC0B3E6E84DA3EC00DF0CC
:10B4C8000DECCAF09FDA6BECD0F030DAE8EC53F010
:10B4D800DEEC53F08ADA5EECADF066D0330EA2EC07
:10B4E8002AF09E6F9D6F46DA80DA5EECADF0590E59
:10B4F8001E6E250E4EDAD1ECD0F056D0330EA2ECEB
:10B508002AF09E6F9D6F36DA73DA5EECADF0920E1C
:10B518001E6E240E3EDAD1ECD0F046D0360EE4ECA6
:10B528002AF0370EC7EC53F049DA5EECADF02D0E79
:10B538001E6E2A0E1F6ED1ECD0F036D0360EE4EC1B
:10B548002AF0380EC7EC53F039DA5EECADF0C40ED1
:10B558001E6E290E1F6ED1ECD0F026D03950010A8C
:10B5680001E10BD6030A01E147D6010A01E13CD704
:10B57800070A01E176D7010A01E14AD6030A01E187
:10B58800BCD6010A01E10DD70F0A01E11CD7010A57
:10B5980001E148D7030A83E0010AA0E0070AAEE008
:10B5A800010ABCE0030ACAE0020E431801E1A2D175
:10B5B8001200530E1E6E240EECD9D1ECD0F0EFEC35
:10B5C80053F0C4D9310EEAD9CEEC53F0BAD9EAD93E
:10B5D8005EECADF018D00201788126D002017883A4
:10B5E80023D00201788520D0020178871DD002017E
:10B5F80078891AD00201788B17D00201788D14D07F
:10B608000201788F11D03A50010AE5E0030AE6E01A
:10B61800010AE7E0070AE8E0010AE9E0030AEAE0CC
:10B62800010AEBE00F0AECE0E6D92FEFB7F05D0E68
:10B638001E6E230EAED9D1ECD0F0310E0201AED978
:10B64800CEEC53F07ED93A50300F9A6F14D10001E6
:10B6580065AF02D03A0423E065AD03D0020E3A1874
:10B668001EE065AB03D0030E3A1819E065A903D0B4
:10B67800040E3A1814E065A703D0050E3A180FE037
:10B6880065A503D0060E3A180AE065A303D0070E95
:10B698003A1805E065A10DD0080E3A180AE160D9FC
:10B6A800320E4FD97FD95EECADF0700E1E6E240EAF
:10B6B800A7D0D4EC53F0CEEC53F043D973D95EEC59
:10B6C800ADF0538E43D90001678318D00201788109
:10B6D80026D00201788323D00201788520D0020188
:10B6E80078871DD0020178891AD00201788B17D08B
:10B6F8000201788D14D00201788F11D03A50010AD6
:10B70800E5E0030AE6E0010AE7E0070AE8E0010AE3
:10B71800E9E0030AEAE0010AEBE00F0AECE06BD982
:10B728002FECB7F04E0E1E6E240E6AD0000165AFE6
:10B7380002D03A0423E065AD03D0020E3A181EE0A9
:10B7480065AB03D0030E3A1819E065A903D0040EBF
:10B758003A1814E065A703D0050E3A180FE065A55E
:10B7680003D0060E3A180AE065A303D0070E3A186C
:10B7780005E065A11DD0080E3A181AE165BF659F5E
:10B7880065BD659D65BB659B65B9659965B7659739
:10B7980065B5659565B3659365B16591E1D8320E78
:10B7A800D0D806D95EECADF0AC0E1E6E210E28D0B6
:10B7B800D4EC53F0CEEC53F0C4D8FAD85EECADF02C
:10B7C800580E1E6E230E1CD0330E0201B5EC53F03A
:10B7D8009D6F04EC54F0126E000E5EECADF0D50EC9
:10B7E8001E6E240E0DD0330E0201B5EC53F00CEC96
:10B7F80054F0126E000E5EECADF0E70E1E6E230ED6
:10B80800C8D8D1EFD0F0140E1E6E230EC2D8D1ECDA
:10B81800D0F002015C91F6D86BECD0F087D8B5EC8B
:10B8280053F0E3EC53F0E4D85EECADF0D0D8A2ECE2
:10B83800C6F004093F6EC6D83FC00DF00DEFCAF040
:10B848000F0E1E6E230EA5D8D1ECD0F002015C912C
:10B858005C87BDD8A2ECC6F00809406EB3D840C0DA
:10B868000DF00DECCAF0CED86BECD0F05FD8E8EC58
:10B8780053F0E3EC53F0070E39D02D0E1E6E220E56
:10B8880088D8D1ECD0F002015C93BCD86BECD0F036
:10B898004DD8B5EC53F0E3EC53F0A7D85EECADF01F
:10B8A80096D8A2ECC6F0F30B416E8CD841C00DF0CF
:10B8B8000DEFCAF0280E1E6E220E6BD8D1ECD0F018
:10B8C800F50E02015C1783D8A2ECC6F0F30B426EAA
:10B8D80079D842C00DF00DECCAF094D86BECD0F0DA
:10B8E80025D8E8EC53F0E3EC53F0060E126E000E88
:10B8F8005EEFADF03950010A01E15BD6030A01E1C0
:10B9080096D6010A80E0070AB8E0010A01E19FD64D
:10B91800030A01E10BD7010A01E156D70F0A01E139
:10B9280062D7010A8DE0030AC5E0120002019B6F8D
:10B938009B51F60DF3503A249A6F300E9A279B27A5
:10B94800340C9D6F300E9C6F9B6F300C53BC8A8CEF
:10B95800020186513C0DF3CF6FF3F4CF70F3120060
:10B96800330E0201A16F370EA06F330E9F6F300E9A
:10B978009E6F300C9C6F9B6F3A50300F9A6F12007D
:10B98800310E0201A16F330EA06F300E9F6F9E6FB4
:10B99800310C1F6E3AC020F0216A1200A16F330EDD
:10B9A800A06F300C3A50300F9A6F060E126E000CD2
:10B9B8003A50300F9A6F070E126E000C9A6F060EEF
:10B9C800126E000C170E0C6E030E0B6E030C170E86
:10B9D800056E030E046E030C110E02015F6F040165
:10B9E800426F016A79C202F0010C060E126E000C59
:10B9F800070E126E000C110E02015D6F016A78C20B
:10BA080002F0020C0A0E016E3A5012009A0E05015D
:10BA1800E86F2E0EE96F1DECD0F052C640F626EE08
:10BA280055F0DF50FA6FF96B0601426B6BDB26EEBF
:10BA380056F0DF5042110501F96F000E060143115F
:10BA48000501FA6FF00EF9150601426F5BDB06017E
:10BA580057510F0B640DF3CFF9F5F4CFFAF558C62B
:10BA6800FBF50501FB390F0B0A0DF350F92506010B
:10BA7800446FF4500501FA210601456F060158513B
:10BA88000F0B06014427000E03D0E00E4427FF0EDB
:10BA980045234551FAE1210E445DF7E2F20E050116
:10BAA800E86F2C0EE96F40C6EAF5EB6B42C6ECF581
:10BAB80043C6EDF544C6EEF545C6EFF51DECD0F0EE
:10BAC800060E0601401908E1100E4319421104E15F
:10BAD8004451451101E1F30C060E401908E1110E1D
:10BAE8004319421104E14451451101E1F10C060EDC
:10BAF800401908E1120E4319421104E1445145115D
:10BB080001E1F20C060E401907E1100E421904E19A
:10BB1800120E431901E1F00C060E40191DE1700EDA
:10BB280042191AE1130E431917E1455103E1110EA9
:10BB3800445D08E3456B0F0E446F44516009416F43
:10BB4800415112004451451103E1446B456BF5D74F
:10BB58004407D8A04507F1D7070E40191EE1700E1B
:10BB680042191BE1130E431918E1455103E1110E67
:10BB7800445D07E3456B0F0E446F44C641F64151DF
:10BB880012004451451103E1446B456B03D044074F
:10BB9800D8A0450744C641F6D3D7110E4319421120
:10BBA80044E0200E421903E1120E43193EE0300E24
:10BBB800421903E1120E431938E0900E421903E1CD
:10BBC800120E431932E0130E431942112EE0100EE3
:10BBD800421903E1130E431928E0200E421903E12C
:10BBE800130E431922E0300E421903E1130E4319D4
:10BBF8001CE0400E421903E1130E431916E0500EE3
:10BC0800421903E1130E431910E0600E421903E1D3
:10BC1800130E43190AE0140E4319421106E0400EB0
:10BC2800421941E1080E43193EE1060E40191CE194
:10BC3800455103E1110E445D0BE3455103E1210E2B
:10BC4800445D02E355DA01D058DA4451B00977D798
:10BC58004451451105E1446B456B445130096FD798
:10BC68004407D8A04507F9D7070E40191CE14551EC
:10BC780003E1110E445D0BE3455103E1210E445DE0
:10BC880002E336DA01D039DA4451C00958D74451B1
:10BC9800451105E1446B456B4451400950D74407B1
:10BCA800D8A04507F9D7060E401907E1100E42192A
:10BCB80004E1300E431901E1930C070E401907E126
:10BCC800100E421904E1300E431901E1F90C060E79
:10BCD800401907E1200E421904E1300E431901E131
:10BCE800920C070E401907E1200E421904E1300EAC
:10BCF800431901E1F80C060E401907E1900E4219AC
:10BD080004E1300E431901E1920C070E401907E1D6
:10BD1800900E421904E1300E431901E1F80C060EA9
:10BD2800401907E1100E421904E1310E431901E1EF
:10BD3800920C070E401907E1100E421904E1310E6A
:10BD4800431901E1F80C060E401907E1100E4219DB
:10BD580004E1320E431901E1910C070E401907E185
:10BD6800100E421904E1320E431901E1F70C060ED8
:10BD7800401907E1300E421904E1330E431901E17D
:10BD8800980C070E401907E1300E421904E1330EF2
:10BD9800431901E1FE0C060E40190AE1300E421962
:10BDA80007E1370E431904E14451451101E1940CB0
:10BDB800070E40190AE1300E421907E1370E431900
:10BDC80004E14451451101E1FA0C060E40190AE15B
:10BDD800400E421907E1380E431904E14451451158
:10BDE80001E1990C070E40190AE1400E421907E1DA
:10BDF800380E431904E14451451101E1FF0C370E97
:10BE08004319421122E0100E421903E1370E43197B
:10BE18001CE0200E421903E1370E431916E0300EDC
:10BE2800421903E1370E431910E0380E4319421145
:10BE38000CE0300E421903E1380E431906E0400EBB
:10BE480042192FE1380E43192CE1060E401913E16F
:10BE5800455103E1110E445D04E359D94451700979
:10BE68006ED64451451103E1446B456BF7D744073F
:10BE7800D8A04507F3D7070E401913E1455103E150
:10BE8800110E445D04E343D94451800958D6445106
:10BE9800451103E1446B456BF7D74407D8A0450724
:10BEA800F3D7600E421904E1450E431901E1F60C7F
:10BEB800600E421904E1400E431901E1FC0C400EEA
:10BEC8004319421136E0100E421903E1400E43199E
:10BED80030E0200E421903E1400E43192AE0300EEB
:10BEE800421903E1400E431924E0700E421903E1A0
:10BEF800400E43191EE0800E421903E1400E43191B
:10BF080018E0900E421903E1400E431912E0100E9A
:10BF1800421903E1440E43190CE0200E421903E1D3
:10BF2800440E431906E0800E421941E1450E4319BB
:10BF38003EE1060E40191CE1455103E1110E445D36
:10BF48000BE3455103E1210E445D02E3D1D801D052
:10BF5800D4D84451D009F3D54451451105E1446B77
:10BF6800456B44511009EBD54407D8A04507F9D7CC
:10BF7800070E40191CE1455103E1110E445D0BE326
:10BF8800455103E1210E445D02E3B2D801D0B5D892
:10BF98004451E009D4D54451451105E1446B456B42
:10BFA80044512009CCD54407D8A04507F9D7570EE6
:10BFB8004319421112E0100E421903E1570E4319BA
:10BFC8000CE0200E421903E1570E431906E0300E2B
:10BFD80042191FE1570E43191CE1070E401901E1F0
:10BFE800A70C060E401915E1455103E1110E445DF9
:10BFF80006E3456B0F0E446F44515009A0D54451D8
:10C00800451103E1446B456BF7D74407D8A04507B2
:10C01800F3D7060E401907E1200E421904E1530E2A
:10C02800431901E1950C060E401907E1200E42194B
:10C0380004E1600E431901E1900C060E401907E176
:10C04800600E421904E1620E431901E1FB0C060E71
:10C05800401907E1700E421904E1620E431901E12B
:10C06800F50C060E401907E1200E421904E1820E74
:10C07800431901E1A90C070E401907E1200E4219E6
:10C0880004E1820E431901E1AA0C060E401907E1EA
:10C09800300E421904E1830E431901E1AB0C070E7F
:10C0A800401907E1300E421904E1830E431901E1FA
:10C0B800AC0C830E4319421110E1060E401903E13E
:10C0C8004451A0093CD5070E401907E1090E442741
:10C0D800000E45234451900932D5060E401907E158
:10C0E800200E421904E1600E431901E1AE0CAF0CB9
:10C0F800456B0F0E446F456B0F0CEF0E4427FF0E78
:10C108004523FF0C0501FA510601436F1200456BE8
:10C118000F0E446F0F0C22D2E1DAC9DA2AECD5F0FF
:10C128000D6B12009EDA010E2AECD5F0F9D799DAD8
:10C13800040E2AECD5F0F4D7060EC0EC45F0E8DA88
:10C148002AECD5F0EDD785DAE7E0010AEBE0030A3F
:10C15800EEE0010AD8A41200EFD7060E9ADAC8DA80
:10C168002AECD5F0DDD7060EC0EC45F0C4DA2AEC8F
:10C17800D5F066DA93ECCEF097D2060EC0EC45F017
:10C18800010E0201B36F2AECD5F05ADA93ECCEF027
:10C198008BD2060EC0EC45F0BEDA2AECD5F050DAA8
:10C1A80093ECCEF081D2060EC0EC45F0B8DA2AEC5A
:10C1B800D5F046DA93ECCEF077D2060EC0EC45F017
:10C1C800A3DA2AECD5F03CDA93ECCEF06DD2070E68
:10C1D800C0EC45F090DA2AECD5F032DA93ECCEF0E8
:10C1E80063D2070EC0EC45F0010E0201B36F2AECD2
:10C1F800D5F026DA93ECCEF057D2070EC0EC45F016
:10C208008ADA2AECD5F01CDA93ECCEF04DD2070E80
:10C21800C0EC45F084DA2AECD5F012DA93ECCEF0D3
:10C2280043D2070EC0EC45F06FDA2AECD5F008DAF5
:10C2380093ECCEF039D2060E1CDA60DA2AECD5F08F
:10C24800FFD993ECCEF030D2060E13DA010E43DAA2
:10C258002AECD5F0F5D993ECCEF026D2060E09DA01
:10C26800020E39DA2AECD5F0EBD993ECCEF01CD2D9
:10C27800060EFFD9030E2FDA2AECD5F0E1D993EC9C
:10C28800CEF012D2060EF5D9040E25DA2AECD5F036
:10C29800D7D993ECCEF008D2070EEBD92FDA2AECD7
:10C2A800D5F0CED993ECCEF0FFD1070EE2D9010E2E
:10C2B80012DA2AECD5F0C4D993ECCEF0F5D1070EFA
:10C2C800D8D9020E08DA2AECD5F0BAD993ECCEF018
:10C2D800EBD1070ECED9030EFED92AECD5F0B0D992
:10C2E80093ECCEF0E1D1070EC4D9040EF4D92AECB0
:10C2F800D5F0A6D993ECCEF0D7D1C7D9E0D92AEC9E
:10C30800D5F09ED993ECCEF0CFD1BFD90A6F010EEC
:10C31800E2D92AECD5F094D993ECCEF0C5D1B5D9B1
:10C328000A6F020ED8D92AECD5F08AD993ECCEF050
:10C33800BBD1ABD90A6F030ECED92AECD5F080D980
:10C3480093ECCEF0B1D1A1D90A6F040EC4D92AEC6E
:10C35800D5F076D993ECCEF0A7D1060E8AD9E7D9D5
:10C368002AECD5F06DD993ECCEF09ED1060E81D98A
:10C37800010EC7D92AECD5F063D993ECCEF094D14D
:10C38800060E77D9020EBDD92AECD5F059D993EC0F
:10C39800CEF08AD1060E6DD9030EB3D92AECD5F0AA
:10C3A8004FD993ECCEF080D1060E63D9040EA9D9EB
:10C3B8002AECD5F045D993ECCEF076D1060E92D979
:10C3C80076D92AECD5F0ACD6060E09EC46F073D92E
:10C3D8002AECD5F0A5D6060E5CD98AD92AECD5F078
:10C3E8009FD6060E56D987D92AECD5F099D6060ECF
:10C3F8007CD999D92AECD5F093D6060E3FD9060EEA
:10C408002AECD5F08DD625D9D9E0010ADDE0030A5A
:10C41800E2E0010AE6E0070AEAE0010AD8A412000D
:10C42800ECD7070E5FD943D92AECD5F079D6070E99
:10C4380009EC46F040D92AECD5F072D6070E29D976
:10C4480057D92AECD5F06CD6070E23D954D92AEC43
:10C45800D5F066D6070E49D966D92AECD5F060D64C
:10C46800070E0CD9060E2AECD5F05AD6070E010194
:10C47800076F350E20D92AECD5F052D6070EF9D819
:10C4880056D92AECD5F04CD6E4D8CBE0010ACFE057
:10C49800030AD4E0010AD8E0070ADCE0010AE0E078
:10C4A800030AE4E0010AD8A41200E8D7060EE6D889
:10C4B800070E2AECD5F0C4D893ECCEF0F5D00ED9FF
:10C4C800F6D82AECD5F02CD602D9F9D82AECD5F032
:10C4D80027D6FDD80A6F0201B36B050E2AECD5F0FA
:10C4E8001FD6F1D8ECD82AECD5F01AD6D7D800D96F
:10C4F8002AECD5F015D6D2D8FBD82AECD5F010D630
:10C50800CDD806D92AECD5F00BD6C8D80201B36B22
:10C51800090E2AECD5F004D6D6D8CDD82AECD5F019
:10C52800FFD5060EC0EC45F0E9D82AECD5F0F8D5D1
:10C5380090D8C5E0010AC8E0030ACBE0010AD1E0BF
:10C54800070AD4E0010AD7E0030ADAE0010ADDE0CD
:10C558000F0AE2E0020AD8A41200E3D7C1C2D9FF49
:10C56800C2C2DAFFDF50010A01E1EDD5030A01E199
:10C57800F4D5120A01E1F7D5010A01E1FED5030A53
:10C5880001E107D6010A01E10ED6070A01E115D635
:10C59800340A01E11CD6010A01E123D6030A01E1AC
:10C5A8002CD6010A01E133D6070A01E13AD6140A6A
:10C5B80001E141D6010A01E147D6030A01E14ED65D
:10C5C800010A01E155D6070A01E15CD6740A01E1C6
:10C5D80063D6010A01E169D6030A01E170D6010AAE
:10C5E80001E177D6070A01E17ED6140A01E185D672
:10C5F800010A01E18AD6030A01E191D6010A01E1A3
:10C6080098D6070A01E19FD6240A01E1A6D6010AB5
:10C6180001E1ACD6030A01E1B3D6010A01E1BAD6B9
:10C62800070A01E1C1D6E40A01E1EDD6300A01E1C9
:10C638002BD7700A01E13AD7200A01E179D7120015
:10C64800020120EE01F0C151D926C251DA22DF5091
:10C65800120020EE01F0C151D926C251DA22DF5072
:10C668001200060E0101076F350E0A6F0201B36B47
:10C67800350C0101076F130E0A6F130C0101076FC8
:10C68800620E0A6F0201B36B620C060E0101076F9E
:10C69800570C0101076F300E0A6F300C060E0101AE
:10C6A800076F450E0A6F450C01010D6F12000A6FE6
:10C6B8000201B36B020C0A6F0201B36B010C0A6F23
:10C6C8000201B36B000C060E0101076F120C060E77
:10C6D8000101076F110C0201B36F000C060E010176
:10C6E800076F600C0101076F310C0101076F370CF0
:10C6F8000201B36B020C0201B36B010C0201B36BB4
:10C70800000C0201B36F070C040E0201B36F010C99
:10C718000201B36B060C020E0201B36F010C030E8B
:10C728000201B36F010C0A6F0201B36B030C020123
:10C73800B36B070CE86F0201E8A707D0B30ED06F00
:10C748002F0ED16F51ECD0F006D00E0ED06F2F0EF9
:10C75800D16F51ECD0F07DB74CD1820501E082D089
:10C7680055A605D0E8B754A612005482120000015D
:10C778006AA507D00201E8A71200000169BB698D0C
:10C78800120055B455A2120055A802D06AB312007F
:10C798006CBD02D06AA12CD000F00201E8A714D029
:10C7A800010EDD6F040EDE6F010EBAEC4FF0010EC4
:10C7B8000201DD6F040EDE6F020EBAEC4FF00001CD
:10C7C8006C8500016B851200020EDD6F040EDE6FB2
:10C7D800010EBAEC4FF0020E0201DD6F040EDE6F9F
:10C7E800020EBAEC4FF000016C9500016B95120037
:10C7F8000201E8A71200558800016A83648F54B4C7
:10C8080002D069AF03D04AC11AF102D04BC11AF164
:10C8180001011B6B1AC1B3F21BC1B4F20201B66B62
:10C82800030EB56F01ECD3F0B3C21AF1B4C21BF119
:10C838001AC118F11BC119F101011A511B1104E0A9
:10C8480018511911D8A41200559800016C8D6A93DB
:10C858006A81010E0201DD6F040EDE6F010EBAEC73
:10C868004FF0D8D1050E821913E1E8A708D0010EC0
:10C87800DD6F040EDE6F010EBAEC4FF0CBD1020E65
:10C88800DD6F040EDE6F010EBAEC4FF0020EC3D15D
:10C89800030E821933E155B803D000016AA305D00D
:10C8A8000201E8B753840001688D55A86AB31200E5
:10C8B80055B455A212000201E8A710D0010EDD6F91
:10C8C800040EDE6F010EBAEC4FF0010E0201DD6FAF
:10C8D800040EDE6F020EBAEC4FF071D7020EDD6F58
:10C8E800040EDE6F010EBAEC4FF0020E0201DD6F8E
:10C8F800040EDE6F020EBAEC4FF075D7020E8219E5
:10C9080025E155B455A21200E8A710D0010EDD6F3D
:10C91800040EDE6F010EBAEC4FF0010E0201DD6F5E
:10C92800040EDE6F020EBAEC4FF049D7020EDD6F2F
:10C93800040EDE6F010EBAEC4FF0020E0201DD6F3D
:10C94800040EDE6F020EBAEC4FF04DD7070E8219B7
:10C9580022E1E8A710D0050EDD6F040EDE6F010E90
:10C96800BAEC4FF0050E0201DD6F040EDE6F020E09
:10C97800BAEC4FF024D7060EDD6F040EDE6F010E01
:10C98800BAEC4FF0060E0201DD6F040EDE6F020EE8
:10C99800BAEC4FF028D7040E8219D8B455A4120067
:10C9A80055B254B41200000169BF12000201E8A791
:10C9B80010D0010EDD6F040EDE6F010EBAEC4FF0E1
:10C9C800010E0201DD6F040EDE6F020EBAEC4FF0AD
:10C9D800F6D6020EDD6F040EDE6F010EBAEC4FF0D4
:10C9E800020E0201DD6F040EDE6F020EBAEC4FF08C
:10C9F800FAD65BA7B8D0820549E15294E8B75284C9
:10CA080055B6B0D655B455B8120000016CAD18D063
:10CA180000F00201E8A70AD0010EDD6F040EDE6FF8
:10CA2800010EBAEC4FF000016C851200020EDD6FAA
:10CA3800040EDE6F010EBAEC4FF000016C95120087
:10CA48000201E8A71200558854A403D04AC11AF17C
:10CA580002D04BC11AF101011B6B1AC1B3F21BC101
:10CA6800B4F20201B66B030EB56F01ECD3F0B3C29A
:10CA78001AF1B4C21BF101011A511B11D8A41200FA
:10CA8800559800016C8D010E020106D0050E821921
:10CA980009E1010EE8A7020EDD6F040EDE6F010E3C
:10CAA800BAEF4FF0030E821919E155B8E8A701D083
:10CAB800538455A855A41200E8A708D0010EDD6FCD
:10CAC800040EDE6F010EBAEC4FF0ADD7020EDD6F2B
:10CAD800040EDE6F010EBAEC4FF0AFD7020E8219CA
:10CAE80014E155A41200E8A708D0010EDD6F040E6A
:10CAF800DE6F010EBAEC4FF096D7020EDD6F040E12
:10CB0800DE6F010EBAEC4FF098D7070E821912E1CA
:10CB1800E8A708D0050EDD6F040EDE6F010EBAEC33
:10CB28004FF081D7060EDD6F040EDE6F010EBAECF2
:10CB38004FF083D7040E8219D8B455A4120054B408
:10CB48001200E8A708D0010EDD6F040EDE6F010E9B
:10CB5800BAEC4FF068D7020EDD6F040EDE6F010EDF
:10CB6800BAEC4FF06AD75AA71200820556E10001C5
:10CB7800689B0201E8A702D00001688B00016AB532
:10CB8800F9D555B26AB312006AA11AD000F0B00EF6
:10CB98000201D06F2B0ED16F51ECD0F0E8A708D06E
:10CBA800010EDD6F040EDE6F020EBAEC4FF009D6EF
:10CBB800020EDD6F040EDE6F020EBAEC4FF015D6D2
:10CBC800DC0E0201D06F2D0ED16F51ECD0F0E8A72A
:10CBD800120000016A8369AF03D04AC118F102D07C
:10CBE8004BC118F10101196B18C1B3F219C1B4F2A4
:10CBF8000201B66B030EB56F01ECD3F0B3C218F1A6
:10CC0800B4C219F1010118511911D8A41200000178
:10CC18006A936A81010E020106D0050E821909E1A4
:10CC2800010EE8A7020EDD6F040EDE6F020EBAEFEA
:10CC38004FF0030E82191FE100016AA305D002011B
:10CC4800E8A302D00001688D00016AA355A2120072
:10CC58000201E8A708D0010EDD6F040EDE6F020E98
:10CC6800BAEC4FF0AED5020EDD6F040EDE6F020E89
:10CC7800BAEC4FF0BAD5020E821914E155A212008F
:10CC8800E8A708D0010EDD6F040EDE6F020EBAECC5
:10CC98004FF097D5020EDD6F040EDE6F020EBAEC70
:10CCA8004FF0A3D5070E821912E1E8A708D0050EA8
:10CCB800DD6F040EDE6F020EBAEC4FF082D5060E61
:10CCC800DD6F040EDE6F020EBAEC4FF08ED5040E47
:10CCD8008219D8B455A21200000169BF12000201DE
:10CCE800E8A708D0010EDD6F040EDE6F020EBAEC65
:10CCF8004FF067D5020EDD6F040EDE6F020EBAEC40
:10CD08004FF073D558A8120058B002D057ACDFD0F6
:10CD180055AC05D0559C0101515101E0516B54A807
:10CD280003D0549877ECB0F057BC55AE0BD0559E55
:10CD3800010E0501FB6F3DEC8BF0050103E3070EC7
:10CD480002018F6F55BE55BA1200558A170E03019E
:10CD5800FB6F300EFA6F33ECC3F0E8060DE0170EE8
:10CD68000501D76F300ED66F96ECCFF04F0EE86FF7
:10CD7800280EE96F1DEFD0F0170EFA6F300EF96F1D
:10CD8800BAECCDF017E355A855B610D055B40ED06F
:10CD98000101515102E0B1EFCEF00D0E0501F96F1E
:10CDA800FA6B010EADEC32F0B1EFCEF0070E0201D6
:10CDB8008F6F070C170E06014C6F370E4B6F4A69C1
:10CDC8004D6B0F0E4D6501D02AD04BC6FAF34CC6F9
:10CDD800FBF333ECC3F0E80615E14BC6F9F44CC697
:10CDE800FAF4BAECCDF014E306014D294A6FEB0EC4
:10CDF8000501E86F2D0EE96F4AC6EAF5EB6B1DECED
:10CE0800D0F00DD006014A2903E14D51110F4A6FA8
:10CE1800070E06014B27000E4C234D2BD2D70601D7
:10CE280049690101515113E10F0E06014A6503D00A
:10CE3800496501D0BBD7110E4A6109D04A290501BD
:10CE4800FB6F010E3DEC8BF00501B0E21200010111
:10CE580051513DE0100E06014A65A8D7110E4961EF
:10CE680001D0A4D7010151051AE106014A299EE023
:10CE7800100E4A5F4A51070D300EF3244B6F170E00
:10CE8800F4204C6FF90E0501E86F280EE96F1DECD0
:10CE9800D0F04BC6D6F54CC6D7F596EFCFF0020EBC
:10CEA800511915E10601492981E0100E495F4951E0
:10CEB800050DAB0EF3244B6F170EF4204C6F990E33
:10CEC8000501E86F280EE96F1DECD0F0E2D757AEE8
:10CED800120054A803D0549877ECB0F000016DA16B
:10CEE800F8D00101495101E0AED0170E06014C6F90
:10CEF800B00E4B6F02017C6906014D6B0F0E4D653C
:10CF080001D027D04BC6F9F44CC6FAF4DD0E040163
:10CF1800FB6F030EFC6F3AECCAF002017A6F030E46
:10CF28007A1910E04DC67CF2810E0501E86F280ED3
:10CF3800E96F7CC2EAF5EB6B7AC2ECF5ED6B1DECA0
:10CF4800D0F007D0050E06014B27000E4C234D2BC1
:10CF5800D5D702017C290FE1B60E0501E86F2E0E28
:10CF6800E96F1DECD0F0010E0301F76FE6ECA0F0BD
:10CF780000016D9112007C513DE1020E0301F76F33
:10CF8800010EE6ECA0F055A455B22DD0000167A51E
:10CF980067B329D002018B6B89ECC1F00101492BE1
:10CFA800B10E0501E86F280EE96F49C1EAF5EB6B90
:10CFB8001DECD0F00D0EF96FFA6B010EADEC32F0EE
:10CFC80001014905D5E1A60E02015F6F820E5E6F71
:10CFD800200E0301F76FF86B010ECCECBBF0A60E28
:10CFE80002015D6FC5D7070E0301F76F010EE6EC6E
:10CFF800A0F0BED77A5102E07A0518E10101496B29
:10D00800476B020E0301F76F010EE6ECA0F0020178
:10D018007C290501FB6F010E3DEC8BF0A9E3070E9F
:10D028000301F76F010EE6ECA0F0A2D7B60E0501DA
:10D03800E86F2E0EE96F1DECD0F0010E0301F76FBB
:10D04800E6ECA0F095D7020E491943E106014D6BB5
:10D05800060E4D6501D015D08B0E0501E86F310E17
:10D06800E96FDD0E06014D25D96EDA6A030EDA2264
:10D07800DF500501EA6FEB6B1DECD0F006014D2B7C
:10D08800E7D7D10E0501E86F2B0EE96F1DECD0F044
:10D098000301DD510A0DF350DE250601496F4951A0
:10D0A800050DB00EF3244B6F170EF4204C6FB90E1C
:10D0B8000501E86F2A0EE96F1DECD0F04BC6F9F5B3
:10D0C8004CC6FAF5DD0EFB6F030EFC6F20ECCCF0BE
:10D0D8004FD700016CAF12000101485101E0AFD0F9
:10D0E800170E06014C6FB00E4B6F02017B690601EB
:10D0F8004D6B0F0E4D6501D027D04BC6F9F44CC6C9
:10D10800FAF4D40E0401FB6F030EFC6F3AECCAF07C
:10D1180002017A6F030E7A1910E04DC67BF2810E78
:10D128000501E86F280EE96F7BC2EAF5EB6B7AC25E
:10D13800ECF5ED6B1DECD0F007D0050E06014B2782
:10D14800000E4C234D2BD5D702017B2910E1B60EDA
:10D158000501E86F2E0EE96F1DECD0F0010E0301FA
:10D16800F76F020EE6ECA0F000016C9F12007B51F5
:10D178003CE1020E0301F76FE6ECA0F055A455B2AE
:10D188002DD0000167A567B329D002018B6B89EC0C
:10D19800C1F00101482BB10E0501E86F280EE96FB7
:10D1A80048C1EAF5EB6B1DECD0F00D0EF96FFA6B88
:10D1B800010EADEC32F001014805D6E1A60E0201E0
:10D1C8005F6F820E5C6F200E0301F76FF86B020E23
:10D1D800CCECBBF0A60E02015D6FC6D7070E0301AB
:10D1E800F76F020EE6ECA0F0BFD77A5103E0020E0B
:10D1F8007A1917E10101486B466B020E0301F76FBC
:10D20800E6ECA0F002017B290501FB6F020E3DEC64
:10D218008BF0AAE3070E0301F76F020EE6ECA0F00D
:10D22800A3D7B60E0501E86F2E0EE96F1DECD0F0FE
:10D23800010E0301F76F020EE6ECA0F095D7020E7F
:10D248004819D8A4120006014D6B060E4D6501D091
:10D2580015D08B0E0501E86F310EE96FD40E06016B
:10D268004D25D96EDA6A030EDA22DF500501EA6F1E
:10D27800EB6B1DECD0F006014D2BE7D7D10E050165
:10D28800E86F2B0EE96F1DECD0F00301D4510A0DA5
:10D29800F350D5250601496F4951050DB00EF32409
:10D2A8004B6F170EF4204C6FB90E0501E86F2A0E6C
:10D2B800E96F1DECD0F04BC6F9F54CC6FAF5D40E63
:10D2C800FB6F030EFC6F20ECCCF04ED7E86F020129
:10D2D800E8AF07D0DF0ED06F2F0ED16F51ECD0F032
:10D2E80006D03E0ED06F2F0ED16F51ECD0F07DBF1F
:10D2F8004CD17E0501E082D055A605D0E8BF54A6E2
:10D3080012005482120000016AA507D00201E8AF9A
:10D318001200000169BB698D120055B455A21200B4
:10D3280055A802D06AB312006CBD02D06AA12CD0F5
:10D3380000F00201E8AF14D0010EDD6F080EDE6FB9
:10D34800010EBAEC4FF0010E0201DD6F080EDE6F20
:10D35800020EBAEC4FF000016B8D00016A8D1200CD
:10D36800020EDD6F080EDE6F010EBAEC4FF0020EF2
:10D378000201DD6F080EDE6F020EBAEC4FF00001FD
:10D388006B9D00016A9D12000201E8A712005588F2
:10D3980000016A83648F54B402D069AF03D04AC1D4
:10D3A8001AF102D04BC11AF101011B6B1AC1B3F279
:10D3B8001BC1B4F20201B66B030EB56F01ECD3F0DA
:10D3C800B3C21AF1B4C21BF11AC118F11BC119F189
:10D3D80001011A511B1104E018511911D8A41200A7
:10D3E800559800016C8D6A936A81010E0201DD6F08
:10D3F800080EDE6F010EBAEC4FF0D2D1050E7E1981
:10D4080013E1E8AF08D0010EDD6F080EDE6F010EE4
:10D41800BAEC4FF0C5D1020EDD6F080EDE6F010EBB
:10D42800BAEC4FF0020EBDD1030E7E1933E155B8A8
:10D4380003D000016AA305D00201E8BF528C0001A5
:10D44800678D55A86AB3120055B455A2120002019F
:10D45800E8AF10D0010EDD6F080EDE6F010EBAECDA
:10D468004FF0010E0201DD6F080EDE6F020EBAECFE
:10D478004FF071D7020EDD6F080EDE6F010EBAECA9
:10D488004FF0020E0201DD6F080EDE6F020EBAECDD
:10D498004FF075D7020E7E1925E155B455A212003A
:10D4A800E8AF10D0010EDD6F080EDE6F010EBAEC8A
:10D4B8004FF0010E0201DD6F080EDE6F020EBAECAE
:10D4C8004FF049D7020EDD6F080EDE6F010EBAEC81
:10D4D8004FF0020E0201DD6F080EDE6F020EBAEC8D
:10D4E8004FF04DD7070E7E1922E1E8AF10D0050E98
:10D4F800DD6F080EDE6F010EBAEC4FF0050E02016B
:10D50800DD6F080EDE6F020EBAEC4FF024D7060E60
:10D51800DD6F080EDE6F010EBAEC4FF0060E020149
:10D52800DD6F080EDE6F020EBAEC4FF028D7040E3E
:10D538007E19D8B455A4120055B254B41200000193
:10D5480069BF12000201E8AF10D0010EDD6F080EAE
:10D55800DE6F010EBAEC4FF0010E0201DD6F080E0E
:10D56800DE6F020EBAEC4FF0F6D6020EDD6F080E33
:10D57800DE6F010EBAEC4FF0020E0201DD6F080EED
:10D58800DE6F020EBAEC4FF0FAD65BAFBED07E0566
:10D598004FE100016D930201E8AF02D000016D83F5
:10D5A80055A602D00201AAD655B455B812000001FA
:10D5B8006CAD18D000F00201E8AF0AD0010EDD6FA3
:10D5C800080EDE6F010EBAEC4FF000016B8D1200F1
:10D5D800020EDD6F080EDE6F010EBAEC4FF000018F
:10D5E8006B9D12000201E8AF1200558854A403D0C5
:10D5F8004AC11AF102D04BC11AF101011B6B1AC1C1
:10D60800B3F21BC1B4F20201B66B030EB56F01ECA5
:10D61800D3F0B3C21AF1B4C21BF101011A511B11A4
:10D62800D8A41200559800016C8D010E020106D095
:10D63800050E7E1909E1010EE8AF020EDD6F080E36
:10D64800DE6F010EBAEF4FF0030E7E1919E155B8DF
:10D65800E8AF01D0528C55A855A41200E8AF08D005
:10D66800010EDD6F080EDE6F010EBAEC4FF0ADD77C
:10D67800020EDD6F080EDE6F010EBAEC4FF0AFD769
:10D68800020E7E1914E155A41200E8AF08D0010E6D
:10D69800DD6F080EDE6F010EBAEC4FF096D7020E62
:10D6A800DD6F080EDE6F010EBAEC4FF098D7070E4B
:10D6B8007E1912E1E8AF08D0050EDD6F080EDE6FA7
:10D6C800010EBAEC4FF081D7060EDD6F080EDE6F43
:10D6D800010EBAEC4FF083D7040E7E19D8B455A4C6
:10D6E800120054B41200E8AF08D0010EDD6F080E26
:10D6F800DE6F010EBAEC4FF068D7020EDD6F080E30
:10D70800DE6F010EBAEC4FF06AD75AAF12007E05F1
:10D718004AE10001679B0201E8AF02D00001678B74
:10D7280000016AB5F3D555B26AB312006AA114D0E4
:10D7380000F00201E8AF08D0010EDD6F080EDE6FC1
:10D74800020EBAEC4FF009D6020EDD6F080EDE6F3E
:10D75800020EBAEC4FF015D60201E8AF1200000134
:10D768006A8369AF03D04AC118F102D04BC118F1DE
:10D778000101196B18C1B3F219C1B4F20201B66BF9
:10D78800030EB56F01ECD3F0B3C218F1B4C219F1AE
:10D79800010118511911D8A4120000016A936A8175
:10D7A800010E020106D0050E7E1909E1010EE8AF4F
:10D7B800020EDD6F080EDE6F020EBAEF4FF0030E99
:10D7C8007E191FE100016AA305D00201E8A302D077
:10D7D8000001678D00016AA355A212000201E8AF9B
:10D7E80008D0010EDD6F080EDE6F020EBAEC4FF0A6
:10D7F800B4D5020EDD6F080EDE6F020EBAEC4FF0E4
:10D80800C0D5020E7E1914E155A21200E8AF08D067
:10D81800010EDD6F080EDE6F020EBAEC4FF09DD5DB
:10D82800020EDD6F080EDE6F020EBAEC4FF0A9D5BE
:10D83800070E7E1912E1E8AF08D0050EDD6F080E5D
:10D84800DE6F020EBAEC4FF088D5060EDD6F080EBB
:10D85800DE6F020EBAEC4FF094D5040E7E19D8B4E0
:10D8680055A21200000169BF12000201E8AF08D0FA
:10D87800010EDD6F080EDE6F020EBAEC4FF06DD5AB
:10D88800020EDD6F080EDE6F020EBAEC4FF079D58E
:10D89800E86F0201E8AD07D0D40ED06F2F0ED16F1C
:10D8A80051ECD0F006D0320ED06F2F0ED16F51EC64
:10D8B800D0F07DBD4CD17F0501E082D055A605D0C2
:10D8C800E8BD54A612005482120000016AA507D0D0
:10D8D8000201E8AD1200000169BB698D120055B460
:10D8E80055A2120055A802D06AB312006CBD02D02E
:10D8F8006AA12CD000F00201E8AD14D0010EDD6F52
:10D90800070EDE6F010EBAEC4FF0010E0201DD6F5B
:10D91800070EDE6F020EBAEC4FF000016B8F0001AC
:10D928006A8F1200020EDD6F070EDE6F010EBAEC71
:10D938004FF0020E0201DD6F070EDE6F020EBAEC29
:10D948004FF000016B9F00016A9F12000201E8ADD1
:10D958001200558800016A83648F54B402D069AFFD
:10D9680003D04AC11AF102D04BC11AF101011B6B55
:10D978001AC1B3F21BC1B4F20201B66B030EB56F44
:10D9880001ECD3F0B3C21AF1B4C21BF11AC118F1F9
:10D998001BC119F101011A511B1104E01851191189
:10D9A800D8A41200559800016C8D6A936A81010E03
:10D9B8000201DD6F070EDE6F010EBAEC4FF0D2D117
:10D9C800050E7F1913E1E8AD08D0010EDD6F070ED3
:10D9D800DE6F010EBAEC4FF0C5D1020EDD6F070EF7
:10D9E800DE6F010EBAEC4FF0020EBDD1030E7F19A7
:10D9F80033E155B803D000016AA305D00201E8BDA0
:10DA0800528E0001688155A86AB3120055B455A218
:10DA180012000201E8AD10D0010EDD6F070EDE6FB7
:10DA2800010EBAEC4FF0010E0201DD6F070EDE6F3A
:10DA3800020EBAEC4FF071D7020EDD6F070EDE6FE3
:10DA4800010EBAEC4FF0020E0201DD6F070EDE6F19
:10DA5800020EBAEC4FF075D7020E7F1925E155B4C6
:10DA680055A21200E8AD10D0010EDD6F070EDE6F73
:10DA7800010EBAEC4FF0010E0201DD6F070EDE6FEA
:10DA8800020EBAEC4FF049D7020EDD6F070EDE6FBB
:10DA9800010EBAEC4FF0020E0201DD6F070EDE6FC9
:10DAA800020EBAEC4FF04DD7070E7F1922E1E8AD10
:10DAB80010D0050EDD6F070EDE6F010EBAEC4FF0C9
:10DAC800050E0201DD6F070EDE6F020EBAEC4FF095
:10DAD80024D7060EDD6F070EDE6F010EBAEC4FF08D
:10DAE800060E0201DD6F070EDE6F020EBAEC4FF074
:10DAF80028D7040E7F19D8B455A4120055B254B4CF
:10DB08001200000169BF12000201E8AD10D0010E39
:10DB1800DD6F070EDE6F010EBAEC4FF0010E020149
:10DB2800DD6F070EDE6F020EBAEC4FF0F6D6020E6E
:10DB3800DD6F070EDE6F010EBAEC4FF0020E020128
:10DB4800DD6F070EDE6F020EBAEC4FF0FAD65BAD52
:10DB5800BED07F054FE100016D950201E8AD02D00E
:10DB680000016D8555A602D00201AAD655B455B854
:10DB7800120000016CAD18D000F00201E8AD0AD027
:10DB8800010EDD6F070EDE6F010EBAEC4FF00001DB
:10DB98006B8F1200020EDD6F070EDE6F010EBAECFE
:10DBA8004FF000016B9F12000201E8AD120055888A
:10DBB80054A403D04AC11AF102D04BC11AF1010191
:10DBC8001B6B1AC1B3F21BC1B4F20201B66B030E90
:10DBD800B56F01ECD3F0B3C21AF1B4C21BF1010165
:10DBE8001A511B11D8A41200559800016C8D010E12
:10DBF800020106D0050E7F1909E1010EE8AD020EFB
:10DC0800DD6F070EDE6F010EBAEF4FF0030E7F19BE
:10DC180019E155B8E8AD01D0528E55A855A41200A7
:10DC2800E8AD08D0010EDD6F070EDE6F010EBAEC0D
:10DC38004FF0ADD7020EDD6F070EDE6F010EBAECA6
:10DC48004FF0AFD7020E7F1914E155A41200E8ADCA
:10DC580008D0010EDD6F070EDE6F010EBAEC4FF033
:10DC680096D7020EDD6F070EDE6F010EBAEC4FF08D
:10DC780098D7070E7F1912E1E8AD08D0050EDD6FC1
:10DC8800070EDE6F010EBAEC4FF081D7060EDD6F7E
:10DC9800070EDE6F010EBAEC4FF083D7040E7F1922
:10DCA800D8B455A4120054B41200E8AD08D0010E3F
:10DCB800DD6F070EDE6F010EBAEC4FF068D7020E6B
:10DCC800DD6F070EDE6F010EBAEC4FF06AD75AAD62
:10DCD80012007F054AE10001679F0201E8AD02D00A
:10DCE8000001678F00016AB5F3D555B26AB3120017
:10DCF8006AA114D000F00201E8AD08D0010EDD6F72
:10DD0800070EDE6F020EBAEC4FF009D6020EDD6F79
:10DD1800070EDE6F020EBAEC4FF015D60201E8AD21
:10DD2800120000016A8369AF03D04AC118F102D01A
:10DD38004BC118F10101196B18C1B3F219C1B4F242
:10DD48000201B66B030EB56F01ECD3F0B3C218F144
:10DD5800B4C219F1010118511911D8A41200000117
:10DD68006A936A81010E020106D0050E7F1909E146
:10DD7800010EE8AD020EDD6F070EDE6F020EBAEF80
:10DD88004FF0030E7F191FE100016AA305D00201BD
:10DD9800E8A302D00001688100016AA355A212001D
:10DDA8000201E8AD08D0010EDD6F070EDE6F020E2E
:10DDB800BAEC4FF0B4D5020EDD6F070EDE6F020E1F
:10DDC800BAEC4FF0C0D5020E7F1914E155A212002B
:10DDD800E8AD08D0010EDD6F070EDE6F020EBAEC5B
:10DDE8004FF09DD5020EDD6F070EDE6F020EBAEC06
:10DDF8004FF0A9D5070E7F1912E1E8AD08D0050E3E
:10DE0800DD6F070EDE6F020EBAEC4FF088D5060EF6
:10DE1800DD6F070EDE6F020EBAEC4FF094D5040EDC
:10DE28007F19D8B455A21200000169BF120002017F
:10DE3800E8AD08D0010EDD6F070EDE6F020EBAECFA
:10DE48004FF06DD5020EDD6F070EDE6F020EBAECD5
:10DE58004FF079D5E86F0201E8A507D0A80ED06F7A
:10DE68002F0ED16F51ECD0F006D0020ED06F2F0ECE
:10DE7800D16F51ECD0F07DB54CD1830501E082D053
:10DE880055A605D0E8B554A6120054821200000128
:10DE98006AA507D00201E8A51200000169BB698DD7
:10DEA800120055B455A2120055A802D06AB3120048
:10DEB8006CBD02D06AA12CD000F00201E8A514D0F4
:10DEC800010EDD6F030EDE6F010EBAEC4FF0010E8E
:10DED8000201DD6F030EDE6F020EBAEC4FF0000197
:10DEE8006C8700016B871200020EDD6F030EDE6F78
:10DEF800010EBAEC4FF0020E0201DD6F030EDE6F69
:10DF0800020EBAEC4FF000016C9700016B971200FB
:10DF18000201E8A51200558800016A83648F54B491
:10DF280002D069AF03D04AC11AF102D04BC11AF12D
:10DF380001011B6B1AC1B3F21BC1B4F20201B66B2B
:10DF4800030EB56F01ECD3F0B3C21AF1B4C21BF1E2
:10DF58001AC118F11BC119F101011A511B1104E072
:10DF680018511911D8A41200559800016C8D6A93A4
:10DF78006A81010E0201DD6F030EDE6F010EBAEC3D
:10DF88004FF0CCD1050E831913E1E8A508D0010E96
:10DF9800DD6F030EDE6F010EBAEC4FF0BFD1020E3B
:10DFA800DD6F030EDE6F010EBAEC4FF0020EB7D133
:10DFB800030E831933E155B803D000016AA305D0D5
:10DFC8000201E8B553860001698155A86AB31200B9
:10DFD80055B455A212000201E8A510D0010EDD6F5C
:10DFE800030EDE6F010EBAEC4FF0010E0201DD6F79
:10DFF800030EDE6F020EBAEC4FF071D7020EDD6F22
:10E00800030EDE6F010EBAEC4FF0020E0201DD6F57
:10E01800030EDE6F020EBAEC4FF075D7020E8319AD
:10E0280025E155B455A21200E8A510D0010EDD6F08
:10E03800030EDE6F010EBAEC4FF0010E0201DD6F28
:10E04800030EDE6F020EBAEC4FF049D7020EDD6FF9
:10E05800030EDE6F010EBAEC4FF0020E0201DD6F07
:10E06800030EDE6F020EBAEC4FF04DD7070E831980
:10E0780022E1E8A510D0050EDD6F030EDE6F010E5C
:10E08800BAEC4FF0050E0201DD6F030EDE6F020ED3
:10E09800BAEC4FF024D7060EDD6F030EDE6F010ECB
:10E0A800BAEC4FF0060E0201DD6F030EDE6F020EB2
:10E0B800BAEC4FF028D7040E8319D8B455A412002F
:10E0C80055B254B41200000169BF12000201E8A55C
:10E0D80010D0010EDD6F030EDE6F010EBAEC4FF0AB
:10E0E800010E0201DD6F030EDE6F020EBAEC4FF077
:10E0F800F6D6020EDD6F030EDE6F010EBAEC4FF09E
:10E10800020E0201DD6F030EDE6F020EBAEC4FF055
:10E11800FAD65BA5B8D0830549E15296E8B5528690
:10E1280055B6B0D655B455B8120000016CAD18D02C
:10E1380000F00201E8A50AD0010EDD6F030EDE6FC4
:10E14800010EBAEC4FF000016C871200020EDD6F71
:10E15800030EDE6F010EBAEC4FF000016C9712004F
:10E168000201E8A51200558854A403D04AC11AF147
:10E1780002D04BC11AF101011B6B1AC1B3F21BC1CA
:10E18800B4F20201B66B030EB56F01ECD3F0B3C263
:10E198001AF1B4C21BF101011A511B11D8A41200C3
:10E1A800559800016C8D010E020106D0050E8319E9
:10E1B80009E1010EE8A5020EDD6F030EDE6F010E08
:10E1C800BAEF4FF0030E831919E155B8E8A501D04D
:10E1D800538655A855A41200E8A508D0010EDD6F96
:10E1E800030EDE6F010EBAEC4FF0ADD7020EDD6FF5
:10E1F800030EDE6F010EBAEC4FF0AFD7020E831993
:10E2080014E155A41200E8A508D0010EDD6F030E35
:10E21800DE6F010EBAEC4FF096D7020EDD6F030EDB
:10E22800DE6F010EBAEC4FF098D7070E831912E192
:10E23800E8A508D0050EDD6F030EDE6F010EBAECFF
:10E248004FF081D7060EDD6F030EDE6F010EBAECBC
:10E258004FF083D7040E8319D8B455A4120054B4D0
:10E268001200E8A508D0010EDD6F030EDE6F010E67
:10E27800BAEC4FF068D7020EDD6F030EDE6F010EA9
:10E28800BAEC4FF06AD75AA5120083054AE100019B
:10E29800689F0201E8A502D00001688F00016AB5F5
:10E2A800F9D555B26AB312006AA114D000F0020180
:10E2B800E8A508D0010EDD6F030EDE6F020EBAEC82
:10E2C8004FF00FD6020EDD6F030EDE6F020EBAECB2
:10E2D8004FF01BD60201E8A5120000016A8369AF5E
:10E2E80003D04AC118F102D04BC118F10101196BD2
:10E2F80018C1B3F219C1B4F20201B66B030EB56FBF
:10E3080001ECD3F0B3C218F1B4C219F101011851EC
:10E318001911D8A4120000016A936A81010E020142
:10E3280006D0050E831909E1010EE8A5020EDD6F7E
:10E33800030EDE6F020EBAEF4FF0030E83191FE1D2
:10E3480000016AA305D00201E8A302D00001698197
:10E3580000016AA355A212000201E8A508D0010E27
:10E36800DD6F030EDE6F020EBAEC4FF0BAD5020E67
:10E37800DD6F030EDE6F020EBAEC4FF0C6D5020E4B
:10E38800831914E155A21200E8A508D0010EDD6F2B
:10E39800030EDE6F020EBAEC4FF0A3D5020EDD6F4E
:10E3A800030EDE6F020EBAEC4FF0AFD5070E8319DD
:10E3B80012E1E8A508D0050EDD6F030EDE6F020E30
:10E3C800BAEC4FF08ED5060EDD6F030EDE6F020E2F
:10E3D800BAEC4FF09AD5040E8319D8B455A212009E
:10E3E800000169BF12000201E8A508D0010EDD6F27
:10E3F800030EDE6F020EBAEC4FF073D5020EDD6F1E
:10E40800030EDE6F020EBAEC4FF07FD5E86F020103
:10E41800E8AB07D0C90ED06F2F0ED16F51ECD0F0FA
:10E4280006D0260ED06F2F0ED16F51ECD0F07DBBE9
:10E438004AD1800501E082D055A605D0E8BB54A694
:10E4480012005482120000016AA507D00201E8AB4D
:10E458001200000169BB698D120055B455A2120063
:10E4680055A802D06AB312006CBD02D06AA12CD0A4
:10E4780000F00201E8AB14D0010EDD6F060EDE6F6E
:10E48800010EBAEC4FF0010E0201DD6F060EDE6FD1
:10E49800020EBAEC4FF000016C8100016B81120092
:10E4A800020EDD6F060EDE6F010EBAEC4FF0020EA3
:10E4B8000201DD6F060EDE6F020EBAEC4FF00001AE
:10E4C8006C9100016B9112000201E8AB12005588B3
:10E4D80000016A83648F54B402D069AF03D04AC183
:10E4E8001AF102D04BC11AF101011B6B1AC1B3F228
:10E4F8001BC1B4F20201B66B030EB56F01ECD3F089
:10E50800B3C21AF1B4C21BF11AC118F11BC119F137
:10E5180001011A511B1104E018511911D8A4120055
:10E52800559800016C8D6A936A81010E0201DD6FB6
:10E53800060EDE6F010EBAEC4FF0C9D1050E801938
:10E5480013E1E8AB08D0010EDD6F060EDE6F010E99
:10E55800BAEC4FF0BCD1020EDD6F060EDE6F010E75
:10E56800BAEC4FF0020EB4D1030E801933E155B85E
:10E5780003D000016AA305D00201E8BB5380000163
:10E58800688555A86AB3120055B455A21200020155
:10E59800E8AB10D0010EDD6F060EDE6F010EBAEC8F
:10E5A8004FF0010E0201DD6F060EDE6F020EBAECAF
:10E5B8004FF071D7020EDD6F060EDE6F010EBAEC5A
:10E5C8004FF0020E0201DD6F060EDE6F020EBAEC8E
:10E5D8004FF075D7020E801925E155B455A21200E7
:10E5E800E8AB10D0010EDD6F060EDE6F010EBAEC3F
:10E5F8004FF0010E0201DD6F060EDE6F020EBAEC5F
:10E608004FF049D7020EDD6F060EDE6F010EBAEC31
:10E618004FF0020E0201DD6F060EDE6F020EBAEC3D
:10E628004FF04DD7070E801920E1E8AB10D0050E4A
:10E63800DD6F060EDE6F010EBAEC4FF0050E02011B
:10E64800DD6F060EDE6F020EBAEC4FF024D7060E11
:10E65800DD6FDE6F010EBAEC4FF0060E0201DD6FC2
:10E66800DE6F020EBAEC4FF02AD7040E8019D8B428
:10E6780055A4120055B254B41200000169BF12002B
:10E688000201E8AB10D0010EDD6F060EDE6F010E41
:10E69800BAEC4FF0010E0201DD6F060EDE6F020EBE
:10E6A800BAEC4FF0F8D6020EDD6F060EDE6F010EE3
:10E6B800BAEC4FF0020E0201DD6F060EDE6F020E9D
:10E6C800BAEC4FF0FCD65BABB7D0800549E152906D
:10E6D800E8BB528055B6B2D655B455B81200000101
:10E6E8006CAD18D000F00201E8AB0AD0010EDD6F66
:10E6F800060EDE6F010EBAEC4FF000016C811200BD
:10E70800020EDD6F060EDE6F010EBAEC4FF000014F
:10E718006C9112000201E8AB1200558854A403D092
:10E728004AC11AF102D04BC11AF101011B6B1AC17F
:10E73800B3F21BC1B4F20201B66B030EB56F01EC64
:10E74800D3F0B3C21AF1B4C21BF101011A511B1163
:10E75800D8A41200559800016C8D010E020106D054
:10E76800050E801909E1010EE8AB020EDD6F060EF9
:10E77800DE6F010EBAEF4FF0030E801919E155B89C
:10E78800E8AB01D0538055A855A41200E8AB08D0D7
:10E79800010EDD6F060EDE6F010EBAEC4FF0ADD73D
:10E7A800020EDD6F060EDE6F010EBAEC4FF0AFD72A
:10E7B800020E801914E155A41200E8AB08D0010E2E
:10E7C800DD6F060EDE6F010EBAEC4FF096D7020E23
:10E7D800DD6F060EDE6F010EBAEC4FF098D7070E0C
:10E7E800801911E1E8AB08D0050EDD6F060EDE6F6B
:10E7F800010EBAEC4FF081D7060EDD6FDE6F010E09
:10E80800BAEC4FF084D7040E8019D8B455A412007E
:10E8180054B41200E8AB08D0010EDD6F060EDE6FAF
:10E82800010EBAEC4FF069D7020EDD6F060EDE6FEF
:10E83800010EBAEC4FF06BD75AAB120080054AE1D3
:10E84800000168930201E8AB02D00001688300016F
:10E858006AB5FCD555B26AB312006AA114D000F0AB
:10E868000201E8AB08D0010EDD6F060EDE6F020E66
:10E87800BAEC4FF012D6020EDD6F060EDE6F020EF6
:10E88800BAEC4FF01ED60201E8AB120000016A8311
:10E8980069AF03D04AC118F102D04BC118F1010188
:10E8A800196B18C1B3F219C1B4F20201B66B030EA9
:10E8B800B56F01ECD3F0B3C218F1B4C219F101017C
:10E8C80018511911D8A4120000016A936A81010E27
:10E8D800020106D0050E801909E1010EE8AB020E0F
:10E8E800DD6F060EDE6F020EBAEF4FF0030E8019D1
:10E8F8001FE100016AA305D00201E8A302D00001CC
:10E90800688500016AA355A212000201E8AB08D08D
:10E91800010EDD6F060EDE6F020EBAEC4FF0BDD5AC
:10E92800020EDD6F060EDE6F020EBAEC4FF0C9D58F
:10E93800020E801914E155A21200E8AB08D0010EAE
:10E94800DD6F060EDE6F020EBAEC4FF0A6D5020E92
:10E95800DD6F060EDE6F020EBAEC4FF0B2D5070E71
:10E96800801911E1E8AB08D0050EDD6F060EDE6FE9
:10E97800020EBAEC4FF091D5060EDD6FDE6F020E77
:10E98800BAEC4FF09ED5040E8019D8B455A21200E7
:10E99800000169BF12000201E8AB08D0010EDD6F6B
:10E9A800060EDE6F020EBAEC4FF077D5020EDD6F61
:10E9B800060EDE6F020EBAEC4FF083D5E86F020147
:10E9C800E8A907D0BE0ED06F2F0ED16F51ECD0F052
:10E9D80006D01A0ED06F2F0ED16F51ECD0F07DB942
:10E9E8004AD1810501E082D055A605D0E8B954A6E0
:10E9F80012005482120000016AA507D00201E8A99A
:10EA08001200000169BB698D120055B455A21200AD
:10EA180055A802D06AB312006CBD02D06AA12CD0EE
:10EA280000F00201E8A914D0010EDD6F050EDE6FBB
:10EA3800010EBAEC4FF0010E0201DD6F050EDE6F1C
:10EA4800020EBAEC4FF000016C8300016B831200D8
:10EA5800020EDD6F050EDE6F010EBAEC4FF0020EEE
:10EA68000201DD6F050EDE6F020EBAEC4FF00001F9
:10EA78006C9300016B9312000201E8A912005588FB
:10EA880000016A83648F54B402D069AF03D04AC1CD
:10EA98001AF102D04BC11AF101011B6B1AC1B3F272
:10EAA8001BC1B4F20201B66B030EB56F01ECD3F0D3
:10EAB800B3C21AF1B4C21BF11AC118F11BC119F182
:10EAC80001011A511B1104E018511911D8A41200A0
:10EAD800559800016C8D6A936A81010E0201DD6F01
:10EAE800050EDE6F010EBAEC4FF0C9D1050E811983
:10EAF80013E1E8A908D0010EDD6F050EDE6F010EE7
:10EB0800BAEC4FF0BCD1020EDD6F050EDE6F010EC0
:10EB1800BAEC4FF0020EB4D1030E811933E155B8A7
:10EB280003D000016AA305D00201E8B953820001AD
:10EB3800688955A86AB3120055B455A2120002019B
:10EB4800E8A910D0010EDD6F050EDE6F010EBAECDC
:10EB58004FF0010E0201DD6F050EDE6F020EBAECFA
:10EB68004FF071D7020EDD6F050EDE6F010EBAECA5
:10EB78004FF0020E0201DD6F050EDE6F020EBAECD9
:10EB88004FF075D7020E811925E155B455A2120030
:10EB9800E8A910D0010EDD6F050EDE6F010EBAEC8C
:10EBA8004FF0010E0201DD6F050EDE6F020EBAECAA
:10EBB8004FF049D7020EDD6F050EDE6F010EBAEC7D
:10EBC8004FF0020E0201DD6F050EDE6F020EBAEC89
:10EBD8004FF04DD7070E811920E1E8A90ED0050E98
:10EBE800DD6FDE6F010EBAEC4FF0050E0201DD6F2E
:10EBF800DE6F020EBAEC4FF026D7060EDD6F050E5B
:10EC0800DE6F010EBAEC4FF0060E0201DD6F050E45
:10EC1800DE6F020EBAEC4FF02AD7040E8119D8B471
:10EC280055A4120055B254B41200000169BF120075
:10EC38000201E8A910D0010EDD6F050EDE6F010E8E
:10EC4800BAEC4FF0010E0201DD6F050EDE6F020E09
:10EC5800BAEC4FF0F8D6020EDD6F050EDE6F010E2E
:10EC6800BAEC4FF0020E0201DD6F050EDE6F020EE8
:10EC7800BAEC4FF0FCD65BA9B7D0810549E15292B6
:10EC8800E8B9528255B6B2D655B455B8120000014B
:10EC98006CAD18D000F00201E8A90AD0010EDD6FB2
:10ECA800050EDE6F010EBAEC4FF000016C83120006
:10ECB800020EDD6F050EDE6F010EBAEC4FF000019B
:10ECC8006C9312000201E8A91200558854A403D0DD
:10ECD8004AC11AF102D04BC11AF101011B6B1AC1CA
:10ECE800B3F21BC1B4F20201B66B030EB56F01ECAF
:10ECF800D3F0B3C21AF1B4C21BF101011A511B11AE
:10ED0800D8A41200559800016C8D010E020106D09E
:10ED1800050E811909E1010EE8A9020EDD6F050E45
:10ED2800DE6F010EBAEF4FF0030E811919E155B8E5
:10ED3800E8A901D0538255A855A41200E8A908D023
:10ED4800010EDD6F050EDE6F010EBAEC4FF0ADD788
:10ED5800020EDD6F050EDE6F010EBAEC4FF0AFD775
:10ED6800020E811914E155A41200E8A908D0010E79
:10ED7800DD6F050EDE6F010EBAEC4FF096D7020E6E
:10ED8800DD6F050EDE6F010EBAEC4FF098D7070E57
:10ED9800811911E1E8A907D0050EDD6FDE6F010EBC
:10EDA800BAEC4FF082D7060EDD6F050EDE6F010E4E
:10EDB800BAEC4FF084D7040E8119D8B455A41200C8
:10EDC80054B41200E8A908D0010EDD6F050EDE6FFD
:10EDD800010EBAEC4FF069D7020EDD6F050EDE6F3B
:10EDE800010EBAEC4FF06BD75AA9120081054AE11F
:10EDF800000168970201E8A902D0000168870001B4
:10EE08006AB5FCD555B26AB312006AA114D000F0F5
:10EE18000201E8A908D0010EDD6F050EDE6F020EB3
:10EE2800BAEC4FF012D6020EDD6F050EDE6F020E41
:10EE3800BAEC4FF01ED60201E8A9120000016A835D
:10EE480069AF03D04AC118F102D04BC118F10101D2
:10EE5800196B18C1B3F219C1B4F20201B66B030EF3
:10EE6800B56F01ECD3F0B3C218F1B4C219F10101C6
:10EE780018511911D8A4120000016A936A81010E71
:10EE8800020106D0050E811909E1010EE8A9020E5A
:10EE9800DD6F050EDE6F020EBAEF4FF0030E81191B
:10EEA8001FE100016AA305D00201E8A302D0000116
:10EEB800688900016AA355A212000201E8A908D0D6
:10EEC800010EDD6F050EDE6F020EBAEC4FF0BDD5F8
:10EED800020EDD6F050EDE6F020EBAEC4FF0C9D5DB
:10EEE800020E811914E155A21200E8A908D0010EFA
:10EEF800DD6F050EDE6F020EBAEC4FF0A6D5020EDE
:10EF0800DD6F050EDE6F020EBAEC4FF0B2D5070EBC
:10EF1800811911E1E8A907D0050EDD6FDE6F020E39
:10EF2800BAEC4FF092D5060EDD6F050EDE6F020EBD
:10EF3800BAEC4FF09ED5040E8119D8B455A2120030
:10EF4800000169BF12000201E8A908D0010EDD6FB7
:10EF5800050EDE6F020EBAEC4FF077D5020EDD6FAC
:10EF6800050EDE6F020EBAEC4FF083D5E86F020192
:10EF7800E8A107D0920ED06F2F0ED16F51ECD0F0D0
:10EF880006D0EA0ED06F2E0ED16F51ECD0F07DB1C5
:10EF980038D185057CE155A605D0E8B154A6120004
:10EFA8005482120000016AA507D00201E8A11200EC
:10EFB800000169BB698D120055B455A2120055A80D
:10EFC80002D06AB312006CBD02D06AA128D000F04A
:10EFD8000201E8A111D0010EDD6FDE6FBAEC4FF02F
:10EFE800010E0201DD6FDE6F020EBAEC4FF0000178
:10EFF8006C8B00016B8B1200020EDD6F010EDE6F51
:10F00800BAEC4FF0020E0201DD6F010EDE6F020E48
:10F01800BAEC4FF000016C9B00016B9B12000201DF
:10F02800E8A11200558800016A83648F54B402D0A5
:10F0380069AF03D04AC11AF102D04BC11AF10101DC
:10F048001B6B1AC1B3F21BC1B4F20201B66B030EFB
:10F05800B56F01ECD3F0B3C21AF1B4C21BF11AC1F7
:10F0680018F11BC119F101011A511B1104E01851C3
:10F078001911D8A41200559800016C8D6A936A8101
:10F08800010E0201DD6FDE6FBAEC4FF00AD0050EFB
:10F09800851914E1E8A109D0010EDD6FDE6FBAEC25
:10F0A8004FF0010E0201DD6FADD1020EDD6F010ED2
:10F0B800DE6FBAEC4FF0020E0201B0D1030E8519D3
:10F0C8002FE155B803D000016AA305D00201E8B1C9
:10F0D800538A0001698755A86AB3120055B455A22E
:10F0E80012000201E8A10DD0010EDD6FDE6FBAEC4F
:10F0F8004FF0010E0201DD6FDE6F020EBAEC4FF029
:10F1080076D7020EDD6F010EDE6FBAEC4FF0020EFD
:10F118000201DD6F010EDE6F020EBAEC4FF07AD7F6
:10F12800020E851921E155B455A21200E8A10DD0AF
:10F13800010EDD6FDE6FBAEC4FF0010E0201DD6FDC
:10F14800DE6F020EBAEC4FF052D7020EDD6F010EE1
:10F15800DE6FBAEC4FF0020E0201DD6F010EDE6FBA
:10F16800020EBAEC4FF056D7070E851920E1E8A138
:10F178000FD0050EDD6F010EDE6FBAEC4FF0050EF5
:10F188000201DD6F010EDE6F020EBAEC4FF02FD7D1
:10F19800060EDD6F010EDE6FBAEC4FF0060E0201AF
:10F1A800DD6F010EDE6F020EBAEC4FF033D7040E9E
:10F1B8008519D8B455A4120055B254B412000001F0
:10F1C80069BF12000201E8A10DD0010EDD6FDE6FEC
:10F1D800BAEC4FF0010E0201DD6FDE6F020EBAECE1
:10F1E8004FF005D7020EDD6F010EDE6FBAEC4FF05F
:10F1F800020E0201DD6F010EDE6F020EBAEC4FF057
:10F2080009D75BA1B4D0850546E1529AE8B1528A84
:10F2180055B6C3D655B455B8120000016CAD15D01B
:10F2280000F00201E8A108D0010EDD6FDE6FBAEC34
:10F238004FF000016C8B1200020EDD6F010EDE6FC5
:10F24800BAEC4FF000016C9B12000201E8A1120019
:10F25800558854A403D04AC11AF102D04BC11AF1FF
:10F2680001011B6B1AC1B3F21BC1B4F20201B66BE8
:10F27800030EB56F01ECD3F0B3C21AF1B4C21BF19F
:10F2880001011A511B11D8A41200559800016C8D68
:10F29800010E020106D0050E85190AE1E8A103D086
:10F2A800010EDD6F02D0020E5FD0DE6FBAEF4FF0B5
:10F2B800030E851916E155B8E8A101D0538A55A85F
:10F2C80055A41200E8A106D0010EDD6FDE6FBAEC7E
:10F2D8004FF0AFD7020EDD6F010EDE6FBAEC4FF0C4
:10F2E800B1D7020E851911E155A41200E8A106D084
:10F2F800010EDD6FDE6FBAEC4FF09BD7020EDD6FAB
:10F30800010EDE6FBAEC4FF09DD7070E851910E19C
:10F31800E8A107D0050EDD6F010EDE6FBAEC4FF0E5
:10F3280088D7060EDD6F010EDE6FBAEC4FF08AD774
:10F33800040E851912E155B454B41200E8A106D0A0
:10F34800010EDD6FDE6FBAEC4FF073D7020EDD6F82
:10F35800010EDE6FBAEC4FF075D7060E8519D8A4EA
:10F368001200060EE8A1080EDD6F010E9ED75AA105
:10F37800120085054BE1000169990201E8A102D05C
:10F388000001698900016AB510D655B26AB3120046
:10F398006AA113D000F00201E8A107D0010EDD6FC9
:10F3A800DE6F020EBAEC4FF024D6020EDD6F010EAE
:10F3B800DE6F020EBAEC4FF02FD60201E8A1120060
:10F3C80000016A8369AF03D04AC118F102D04BC16A
:10F3D80018F10101196B18C1B3F219C1B4F2020195
:10F3E800B66B030EB56F01ECD3F0B3C218F1B4C21B
:10F3F80019F1010118511911D8A4120000016A93DA
:10F408006A814FD6DE6F020EBAEF4FF0050E8519EE
:10F4180008E1E8A102D0010E46D6020EDD6F010E0A
:10F42800F1D7030E85191EE100016AA305D0020178
:10F43800E8A102D00001698700016AA355A2120061
:10F448000201E8A107D0010EDD6FDE6F020EBAECF3
:10F458004FF0CFD5020EDD6F010EDE6F020EBAEC53
:10F468004FF0DAD5020E851913E155A21200E8A172
:10F4780007D0010EDD6FDE6F020EBAEC4FF0B9D582
:10F48800020EDD6F010EDE6F020EBAEC4FF0C4D52E
:10F49800070E851912E1E8A108D0050EDD6F010EEF
:10F4A800DE6F020EBAEC4FF0A4D5060EDD6F010E2A
:10F4B800DE6F020EBAEC4FF0AFD5040E8519D8B442
:10F4C80055A21200000169BF12000201E8A107D08D
:10F4D800010EDD6FDE6F020EBAEC4FF08AD5020E18
:10F4E800DD6F010EDE6F020EBAEC4FF095D5E86FB6
:10F4F8000201E8A307D09D0ED06F2F0ED16F51ECFB
:10F50800D0F006D0F60ED06F2E0ED16F51ECD0F0A1
:10F518007DB33DD184057EE155A605D0E8B354A658
:10F5280012005482120000016AA507D00201E8A364
:10F538001200000169BB698D120055B455A2120072
:10F5480055A802D06AB312006CBD02D06AA128D0B7
:10F5580000F00201E8A313D0010EDD6F020EDE6F8A
:10F56800010EBAEC4FF0010E0201DD6F020EDE6FE4
:10F57800BAEC4FF000016C8900016B891200020E91
:10F58800DD6FDE6F010EBAEC4FF0020E0201DD6F87
:10F59800DE6FBAEC4FF000016C9900016B99120014
:10F5A8000201E8A31200558800016A83648F54B4ED
:10F5B80002D069AF03D04AC11AF102D04BC11AF187
:10F5C80001011B6B1AC1B3F21BC1B4F20201B66B85
:10F5D800030EB56F01ECD3F0B3C21AF1B4C21BF13C
:10F5E8001AC118F11BC119F101011A511B1104E0CC
:10F5F80018511911D8A41200559800016C8D6A93FE
:10F608006A81010E0201DD6F020EDE6F010EBAEC97
:10F618004FF00CD0050E841917E1E8A30CD0010EA9
:10F62800DD6F020EDE6F010EBAEC4FF0010E020123
:10F63800DD6F020EAED1020EDD6FDE6F010EBAEC89
:10F648004FF0020E0201B0D1030E84192FE155B814
:10F6580003D000016AA305D00201E8B35388000172
:10F66800698355A86AB3120055B455A21200020165
:10F67800E8A30FD0010EDD6F020EDE6F010EBAECAB
:10F688004FF0010E0201DD6F020EDE6FBAEC4FF093
:10F6980071D7020EDD6FDE6F010EBAEC4FF0020E6D
:10F6A8000201DD6FDE6FBAEC4FF075D7020E8419D8
:10F6B80021E155B455A21200E8A30FD0010EDD6F69
:10F6C800020EDE6F010EBAEC4FF0010E0201DD6F83
:10F6D800020EDE6FBAEC4FF04DD7020EDD6FDE6F13
:10F6E800010EBAEC4FF0020E0201DD6FDE6FBAECCC
:10F6F8004FF051D7070E841920E1E8A30FD0050E6B
:10F70800DD6F020EDE6F010EBAEC4FF0050E02013E
:10F71800DD6F020EDE6FBAEC4FF02CD7060EDD6FF0
:10F72800020EDE6F010EBAEC4FF0060E0201DD6F1D
:10F73800020EDE6FBAEC4FF02ED7040E8419D8B43F
:10F7480055A4120055B254B41200000169BF12004A
:10F758000201E8A30FD0010EDD6F020EDE6F010E6D
:10F76800BAEC4FF0010E0201DD6F020EDE6FBAEC4B
:10F778004FF000D7020EDD6FDE6F010EBAEC4FF0CE
:10F78800020E0201DD6FDE6FBAEC4FF004D75BA307
:10F79800B7D0840548E15298E8B3528855B6BED62A
:10F7A80055B455B8120000016CAD17D000F0020135
:10F7B800E8A30AD0010EDD6F020EDE6F010EBAEC6F
:10F7C8004FF000016C891200020EDD6FDE6F010E32
:10F7D800BAEC4FF000016C9912000201E8A3120084
:10F7E800558854A403D04AC11AF102D04BC11AF16A
:10F7F80001011B6B1AC1B3F21BC1B4F20201B66B53
:10F80800030EB56F01ECD3F0B3C21AF1B4C21BF109
:10F8180001011A511B11D8A41200559800016C8DD2
:10F82800010E020106D0050E84190CE1E8A304D0EC
:10F83800010EDD6F020E02D0020EDD6FDE6F010ECB
:10F84800BAEF4FF0030E841918E155B8E8A301D0B8
:10F85800538855A855A41200E8A308D0010EDD6FFF
:10F86800020EDE6F010EBAEC4FF0ABD7020EDD6F61
:10F87800DE6F010EBAEC4FF0ADD7020E841913E11A
:10F8880055A41200E8A308D0010EDD6F020EDE6F4A
:10F89800010EBAEC4FF095D7020EDD6FDE6F010E48
:10F8A800BAEC4FF097D7070E841912E1E8A308D0F5
:10F8B800050EDD6F020EDE6F010EBAEC4FF081D738
:10F8C800060EDD6F020EDE6F010EBAEC4FF082D726
:10F8D800040E8419D8B455A4120054B41200E8A335
:10F8E80008D0010EDD6F020EDE6F010EBAEC4FF08C
:10F8F80068D7020EDD6FDE6F010EBAEC4FF06AD7E3
:10F908005AA31200840548E1000169950201E8A3A1
:10F9180002D00001698500016AB508D655B26AB3FC
:10F9280012006AA111D000F00201E8A307D0010E6D
:10F93800DD6F020EDE6FBAEC4FF01ED6020EDD6FE1
:10F94800DE6FBAEC4FF029D60201E8A312000001DD
:10F958006A8369AF03D04AC118F102D04BC118F1CC
:10F968000101196B18C1B3F219C1B4F20201B66BE7
:10F97800030EB56F01ECD3F0B3C218F1B4C219F19C
:10F98800010118511911D8A4120000016A936A8163
:10F998004DD6DE6FBAEF4FF0050E841907E1E8A3E4
:10F9A80002D0010E45D6020EDD6FF3D7030E84197F
:10F9B8001CE100016AA305D00201E8A302D00001FE
:10F9C800698300016AA355A212000201E8A307D0C7
:10F9D800010EDD6F020EDE6FBAEC4FF0CDD5020ED0
:10F9E800DD6FDE6FBAEC4FF0D8D5020E841911E145
:10F9F80055A21200E8A307D0010EDD6F020EDE6FDC
:10FA0800BAEC4FF0B9D5020EDD6FDE6FBAEC4FF0ED
:10FA1800C4D5070E841910E1E8A307D0050EDD6FE1
:10FA2800020EDE6FBAEC4FF0A7D5060EDD6F020EA0
:10FA3800DE6FBAEC4FF0B1D5040E8419D8B455A2D4
:10FA48001200000169BF12000201E8A307D0010EED
:10FA5800DD6F020EDE6FBAEC4FF08ED5020EDD6F51
:10FA6800DE6FBAEC4FF099D558A8120058B002D002
:10FA780057ACCAD055AC05D0559C0101515101E095
:10FA8800516B54A803D05498A2ECB2F057BC55AEB1
:10FA980009D0559E010E446ED7EC7FF003E3070EA4
:10FAA80002018F6F55BE55BA1200558A170E056EA2
:10FAB800300E046EA2ECC6F0E8060CE0170E136ECA
:10FAC800300E126E3AECD3F04F0E1E6E280E1F6EDB
:10FAD800D1EFD0F0170E0C6E300E0B6E55ECCEF049
:10FAE80016E355A855B60FD055B40DD001015151A4
:10FAF80002E036EFCEF00D0E396E3A6A010EBCEC1C
:10FB080058F036EFCEF0070E02018F6F070C170E74
:10FB18004B6E370E4A6E49684C6A0F0E4C6401D022
:10FB280026D04AC004F04BC005F0A2ECC6F0E806A7
:10FB380013E14AC00BF04BC00CF055ECCEF011E3CA
:10FB48004C28496EEB0E1E6E2D0E1F6E49C020F01C
:10FB5800216AD1ECD0F00BD0492803E14C50110FA9
:10FB6800496E070E4A26000E4B224C2AD6D7486803
:10FB78000101515110E10F0E496403D0486401D0CE
:10FB8800C2D7110E496007D04928446E010ED7EC40
:10FB98007FF0B9E21200515137E0100E4964B3D733
:10FBA800110E486001D0AFD7510518E14928ABE0E4
:10FBB800100E495E4950070D300EF3244A6E170E99
:10FBC800F4204B6EF90E1E6E280E1F6ED1ECD0F08D
:10FBD8004AC012F04BC013F03AEFD3F0020E51199D
:10FBE80013E1482890E0100E485E4850050DAB0E12
:10FBF800F3244A6E170EF4204B6E990E1E6E280ED3
:10FC08001F6ED1ECD0F0E4D757AE120054A803D041
:10FC18005498A2ECB2F000016DA1E0D00101495165
:10FC280001E09ED0170E4B6EB00E4A6E02017C6941
:10FC38004C6A0F0E4C6401D024D04AC00BF04BC064
:10FC48000CF0DD0E0D6E030E0E6EAEECCCF0020164
:10FC58007A6F030E7A190FE04CC07CF2810E1E6E8B
:10FC6800280E1F6E7CC220F0216A7AC222F0236A15
:10FC7800D1ECD0F006D0050E4A26000E4B224C2AB5
:10FC8800D8D702017C290DE1B60E1E6E2E0E1F6E0E
:10FC9800D1ECD0F0010E016EA1EC9FF000016D9146
:10FCA80012007C5139E1020E016E010EA1EC9FF0A9
:10FCB80055A455B22BD0000167A567B327D0020120
:10FCC8008B6B3AECCBF00101492BB10E1E6E280E5E
:10FCD8001F6E49C120F0216AD1ECD0F00D0E396EAB
:10FCE8003A6A010EBCEC58F001014905D7E1A60EAD
:10FCF80002015F6F820E5E6F200E016E026A010EB6
:10FD08002FECB7F0A60E02015D6FC8D7070E016E83
:10FD1800010EA1EC9FF0C2D77A5102E07A0515E1F5
:10FD28000101496B476B020E016E010EA1EC9FF0B9
:10FD380002017C29446E010ED7EC7FF0AFE3070E79
:10FD4800016E010EA1EC9FF0A9D7B60E1E6E2E0E05
:10FD58001F6ED1ECD0F0010E016EA1EC9FF09ED782
:10FD6800020E49193BE14C6A060E4C6401D011D0D1
:10FD78008B0E1E6E310E1F6EDD0E4C24D96EDA6AA4
:10FD8800030EDA22DF50206E216AD1ECD0F04C2A23
:10FD9800EBD7D10E1E6E2B0E1F6ED1ECD0F00301E7
:10FDA800DD510A0DF350DE25486E4850050DB00EA2
:10FDB800F3244A6E170EF4204B6EB90E1E6E2A0EEF
:10FDC8001F6ED1ECD0F04AC039F04BC03AF0DD0ECE
:10FDD8003B6E030E3C6EF3ECCCF060D700016CAFC9
:10FDE80012000101485101E09FD0170E4B6EB00E72
:10FDF8004A6E02017B694C6A0F0E4C6401D024D014
:10FE08004AC00BF04BC00CF0D40E0D6E030E0E6EF4
:10FE1800AEECCCF002017A6F030E7A190FE04CC0F9
:10FE28007BF2810E1E6E280E1F6E7BC220F0216AA7
:10FE38007AC222F0236AD1ECD0F006D0050E4A2609
:10FE4800000E4B224C2AD8D702017B290EE1B60EB0
:10FE58001E6E2E0E1F6ED1ECD0F0010E016E020E3A
:10FE6800A1EC9FF000016C9F12007B5138E1020E5B
:10FE7800016EA1EC9FF055A455B22BD0000167A5E7
:10FE880067B327D002018B6B3AECCBF00101482B0A
:10FE9800B10E1E6E280E1F6E48C120F0216AD1ECEB
:10FEA800D0F00D0E396E3A6A010EBCEC58F0010123
:10FEB8004805D8E1A60E02015F6F820E5C6F200E26
:10FEC800016E026A020E2FECB7F0A60E02015D6FFA
:10FED800C9D7070E016E020EA1EC9FF0C3D77A5165
:10FEE80003E0020E7A1914E10101486B466B020E19
:10FEF800016EA1EC9FF002017B29446E020ED7EC43
:10FF08007FF0B0E3070E016E020EA1EC9FF0AAD7B6
:10FF1800B60E1E6E2E0E1F6ED1ECD0F0010E016EC5
:10FF2800020EA1EC9FF09ED7020E4819D8A4120029
:10FF38004C6A060E4C6401D011D08B0E1E6E310E29
:10FF48001F6ED40E4C24D96EDA6A030EDA22DF5003
:10FF5800206E216AD1ECD0F04C2AEBD7D10E1E6E60
:10FF68002B0E1F6ED1ECD0F00301D4510A0DF350C3
:10FF7800D525486E4850050DB00EF3244A6E170E6D
:10FF8800F4204B6EB90E1E6E2A0E1F6ED1ECD0F007
:10FF98004AC039F04BC03AF0D40E3B6E030E3C6EAB
:10FFA800F3ECCCF05FD7456E450401E0FAD055B6C6
:10FFB80002D055A499D057BC54B00AD09C0E1E6EDE
:10FFC8002D0E1F6ED1ECD0F08BC28CF2D89012009F
:10FFD80002015E9327DAA1EC9FF0D3D9BAD953BCBA
:10FFE8008A9C55A475D054A405D00A0EEED9BCEC51
:08FFF80058F004D0040EE9D911
:020000040001F9
:10000000BCEC58F0000164AF05D0ACD9016E020E13
:10001000A1EC9FF000016CAB0BD002015BA108D0FA
:1000200000016C9B020E396E010E3A6EBCEC58F06A
:1000300000016CA90BD002015BA308D000016C99F0
:10004000020E396E3A6E010EBCEC58F000016CA73E
:1000500009D002015BA506D000016C97C3D9010E3F
:10006000BCEC58F000016CA509D002015BA706D0DA
:1000700000016C95C1D9010EBCEC58F000016CA3D5
:1000800007D002015BA904D093D9010EBCEC58F053
:1000900000016CA109D002015BAB06D000016C919C
:1000A000B0D9010EBCEC58F000016BAF09D00201D1
:1000B0005BAD06D000016B9FA9D9010EBCEC58F0D6
:1000C00000016BAD09D002015BAF06D000016B9D52
:1000D0007BD9010EBCEC58F064D901E17BD7040E4A
:1000E000016E79C202F0010E2FECB7F0AAD972D7D7
:1000F00057BC54A007D0E10E1E6E2C0E1F6ED1EC23
:10010000D0F068D753BE03D0000167A50DD0000121
:10011000679523D9016A026A010E2FECB7F002013C
:10012000796B53BC8A9C56D755A025D07FD9A1ECBA
:100130009FF075D9016E010EA1EC9FF04ED941C21E
:1001400001F042C202F085D94DECD3F001C041F27A
:1001500002C042F2425108E1240E415D05E2050E63
:10016000016E010EA1EC9FF057AC02D062D932D7DC
:1001700044C089F22FD702018CA102D0010E13D006
:100180008CA302D0020E0FD08CA502D0030E0BD090
:100190008CA702D0040E07D08CA902D0050E03D084
:1001A0008CABE6D0060E8A6FE3D0020E4518D8A4B9
:1001B000120000016AB502D055A28DD002015C93F5
:1001C00032D9A1EC9FF0DCD8C8D853BC8A9C55A288
:1001D00076D0000169AF05D00A0E1DD9BCEC58F0ED
:1001E00004D0040E18D9BCEC58F0000164AF05D05F
:1001F000B9D8016E010EA1EC9FF000016BAB0CD0E1
:1002000002015AA109D000016B9B020E396E010E4A
:100210003A6E020EBCEC58F000016BA90AD0020144
:100220005AA307D000016B99020E396E3A6EBCECEE
:1002300058F000016BA709D002015AA506D00001B1
:100240006B97D0D8020EBCEC58F000016BA509D01A
:1002500002015AA706D000016B95CED8020EBCEC65
:1002600058F000016BA307D002015AA904D0A0D80E
:10027000020EBCEC58F000016BA109D002015AAB90
:1002800006D000016B91BDD8020EBCEC58F0000105
:100290006AAF09D002015AAD06D000016A9FB6D8F4
:1002A000020EBCEC58F000016AAD09D002015AAF51
:1002B00006D000016A9D88D8020EBCEC58F06AD8BE
:1002C00001E188D6040E016E78C202F0020E2FEC16
:1002D000B7F0B3D87FD653BE02D067A30BD03DD8BA
:1002E00000016793016A026A020E2FECB7F0020167
:1002F000786B17D754AE25D096D8A1EC9FF05FD875
:10030000016E020EA1EC9FF072D83FC201F040C214
:1003100002F09FD84DECD3F001C03FF202C040F292
:10032000405108E1240E3F5D05E2050E016E020E0C
:10033000A1EC9FF057AC02D088D84CD644C088F2CC
:1003400049D602018CB11AD78CB31CD78CB51ED7F5
:100350008CB720D78CB922D723D7539E03016F6B5C
:10036000706B120055986A936C9D6A91649F060C9D
:10037000020E8A03F3508A6F548A549CD88012006C
:1003800000016A936A916A951200559800016C9D6C
:1003900055961200000167935592699D02017851AC
:1003A0001200559454920001679502017951120090
:1003B00000016C93020E396E050E3A6E050C0001B9
:1003C0006A8502015C83040C020E396E080E3A6ED7
:1003D000080C396E44043A6E010C87C241F20201E6
:1003E000426B1200020E396E030E3A6E030C87C286
:1003F0003FF20201406B1200020E396E040E3A6E9B
:10040000040C020E396E060E3A6E060C020E396EA0
:10041000070E3A6E070C396E44043A6E020C55868C
:1004200002015E83040C060E016E020C060E016EC4
:10043000010C010E0201896F010C1E0E0101426FB9
:100440001E0C1E0E0101436F1E0C010E0201886F6F
:10045000010C046A030E036E030CABB15A8EABA100
:100460005A9E010E5AAC000EDD6F010E5AAE000E00
:10047000DD1B47E001015A510301225D42E2222BBC
:10048000296B5ABE14D0EDD9310E9A6FA9A106D0AE
:1004900020DA51ECD0F0F7D9ACECACF00201A9B104
:1004A00006D003DA51ECD0F0F2D9ACECACF05AAE95
:1004B00014D0D7D9310E9A6FA9A106D0F6D951EC34
:1004C000D0F0E5D9ACECACF00201A9B106D001DA6C
:1004D00051ECD0F0D8D9ACECACF05AAE02D05A8C7A
:1004E00001D05A9C01015A51030122190AE1060E5A
:1004F0000201D06F270ED16F51ECD0F0010EC4EC89
:10050000D5F00201ABB35A8AABA35A9A010E5AA88E
:10051000000EDD6F010E5AAA000EDD1B4DE0010139
:100520005A510301235D48E2232B2A6B5ABA17D094
:1005300098D9320E9A6FA9A306D0D5D951ECD0F034
:10054000A2D9ACECACF00201A9B309D0410ED06F36
:100550002A0ED16F51ECD0F09AD9ACECACF05AAA7B
:1005600017D07FD9320E9A6FA9A309D0050ED06F8C
:100570002B0ED16F51ECD0F08AD9ACECACF002016B
:10058000A9B306D0B0D951ECD0F07DD9ACECACF029
:100590005AAA02D05A8801D05A9801015A5103012F
:1005A00023190AE1220E0201D06F270ED16F51EC00
:1005B000D0F0020EC4ECD5F00201ABB55A86ABA563
:1005C0005A96010E5AA4000EDD6F010E5AA6000EB7
:1005D000DD1B47E001015A510301245D42E2242B57
:1005E0002B6B5AB614D03DD9330E9A6FA9A506D0FD
:1005F00061D951ECD0F047D9ACECACF00201A9B50F
:1006000006D06CD951ECD0F042D9ACECACF05AA683
:1006100014D027D9330E9A6FA9A506D05FD951EC13
:10062000D0F035D9ACECACF00201A9B506D042D976
:1006300051ECD0F028D9ACECACF05AA602D05A84D8
:1006400001D05A9401015A51030124190AE13E0EC6
:100650000201D06F270ED16F51ECD0F0030EC4EC25
:10066000D5F00201ABB75A82ABA75A92010E5AA03D
:10067000000EDD6F010E5AA2000EDD1B47E00101E6
:100680005A510301255D42E2252B2C6B5AB214D03E
:10069000E8D8340E9A6FA9A706D02FD951ECD0F024
:1006A000F2D8ACECACF00201A9B706D0F4D851EC0A
:1006B000D0F0EDD8ACECACF05AA214D0D2D8340EB5
:1006C0009A6FA9A706D0E7D851ECD0F0E0D8ACECEF
:1006D000ACF00201A9B706D010D951ECD0F0D3D8B4
:1006E000ACECACF05AA202D05A8001D05A90010171
:1006F0005A51030125190AE15A0E0201D06F270E43
:10070000D16F51ECD0F0040EC4ECD5F00201ABB9BE
:10071000598EABA9599E010E59AC000EDD6F010E2A
:1007200059AE000EDD1B47E001015A510301265D61
:1007300042E2262B2D6B59BE14D093D8350E9A6FFA
:10074000A9A906D0BCD851ECD0F09DD8ACECACF047
:100750000201A9B906D0B8D851ECD0F098D8ACECC9
:10076000ACF059AE14D07DD8350E9A6FA9A906D039
:10077000ABD851ECD0F08BD8ACECACF00201A9B9FD
:1007800006D09DD851ECD0F07ED8ACECACF059AE90
:1007900002D0598C01D0599C01015A5103012619EC
:1007A0000AE1760E0201D06F270ED16F51ECD0F026
:1007B000050EC4ECD5F00201ABBB598AABAB599A1C
:1007C000010E59A8000EDD6F010E59AA000EDD1BA7
:1007D000D8B4120001015A510301275DD8B01200AC
:1007E000272B2E6B59BA14D03CD8360E9A6FA9AB72
:1007F00006D07ED851ECD0F046D8ACECACF002017B
:10080000A9BB06D04DD851ECD0F041D8ACECACF03F
:1008100059AA14D026D8360E9A6FA9AB06D040D864
:1008200051ECD0F034D8ACECACF00201A9BB06D04E
:100830005FD851ECD0F027D8ACECACF059AA02D07C
:10084000598801D0599801015A5103012719D8A498
:100850001200920E0201D06F270ED16F51ECD0F032
:10086000060C43C21EF144C21FF1380E0201A16FF3
:10087000330EA06F300E9F6F390E9E6F9D6F300E3E
:100880009C6F9B6F300C060EBE6FDE511200070E80
:10089000BE6FDE5112002B0ED06F2B0ED16F1200E7
:1008A000510ED06F2B0ED16F1200F20ED06F2A0EA8
:1008B000D16F1200520ED06F2C0ED16F1200760E37
:1008C000D06F2C0ED16F12003E0ED06F2B0ED16F59
:1008D00012002E0ED06F2C0ED16F1200180ED06F9A
:1008E0002B0ED16F1200400ED06F2C0ED16F120064
:1008F000880ED06F2C0ED16F1200640ED06F2C0EAC
:10090000D16F1200E90E0501E86F260EE96F1DECAC
:10091000D0F00D0E0501FA6F2D0EF96FD70EE82EEF
:10092000FED7F92FFCD7FA2FFAD700D00501FD6BBF
:10093000FE6BB9D9FB6B0EECBBF0BBD9040EFE5DB0
:10094000F8E3120EFE6FFD6BAED9FB6B0EECBBF045
:10095000B0D9160EFE5DF8E3040EFE6FFD6BA3D951
:10096000FB690EECBBF0A5D9120EFE5DF8E30401A5
:10097000FA6B0C0EFFD90BECC7F00401FA6B0D0EED
:10098000F9D90BECC7F00401FA6B0E0EF96F550E96
:10099000FB6F0BECC7F00401FA6B0F0EF96F4B0EF7
:1009A000FB6F0BECC7F00401FA6B100EF96F3C0EF5
:1009B000FB6F0BECC7F0170E0401FA6F060EF96F10
:1009C000A50EFB6F0BECC7F00401FA6B7A0EAFD9E2
:1009D0000BECC7F00401FA6B640EC8D90BECC7F03E
:1009E0000401FA6B650EC2D90BECC7F00401FA6B77
:1009F000660EF96F780EFB6F0BECC7F00401FA6B13
:100A0000670E89D90BECC7F00401FA6B680E8FD919
:100A10000BECC7F00401FA6B690EF96F030EFB6F64
:100A20000BECC7F00401FA6B6A0E7DD90BECC7F032
:100A30000401FA6B6B0E77D90BECC7F00401FA6B6B
:100A40006C0E71D90BECC7F00401FA6B6D0E6BD90B
:100A50000BECC7F00401FA6B6E0EF96FFB6B0BEC3D
:100A6000C7F00401FA6B6F0EF96FFB6B0BECC7F06C
:100A70000401FA6B780EF96F3F0EFB6F0BECC7F0B9
:100A80000401FA6B790EF96FFB6B0BECC7F024ECE9
:100A9000C4F00BECC7F0170E0401FA6F040EF96FE7
:100AA000FB6B0BECC7F02BD90BECC7F008D90BECA8
:100AB000C7F01DD90BECC7F012D90BECC7F007D962
:100AC0000BECC7F00501FE6B010EFD6F090EFD2555
:100AD0000401F96F170E0501FE210401FA6FFB6B8B
:100AE0000BECC7F00501FD4BFE2BFE5103E1100E90
:100AF000FD5DECE30401FA6B12D90BECC7F00401C5
:100B0000FA6B040E14D90BECC7F00401FA6B050E56
:100B10000ED90BECC7F00401FA6B0A0E23D90BECCB
:100B2000C7F0040E15D9F96FFB6B0BECC7F0040E80
:100B30000401FA6FF4D80BECC7F0040E0401FA6F4D
:100B4000F96BFB6F0BECC7F0040EF5D8E4D80BEC97
:100B5000C7F0170E0401FA6F270EF96FFB6B0BEC51
:100B6000C7F00401FA6B060EF96FFB6B0BECC7F0D4
:100B70000401FA6B070E02D90BECC7F00401FA6B03
:100B8000080EF96F0F0EFB6F0BECC7F00401FA6B48
:100B9000120EC1D80BECC7F00401FA6B110EDED8AF
:100BA0000BECC7F00401FA6B1B0EF96FFB6B0BEC3F
:100BB000C7F00401FA6B140EE1D80BECC7F0040186
:100BC000FA6B150ECFD80BECC7F00401FA6B1D0EB3
:100BD000F96F480EFB6F0BECC7F098D833ECC3F0FD
:100BE0000501F96FF9A10CD0AED8170E0301FB6F08
:100BF000050EFA6F33ECC3F0FB6F0BECC7F00CD0B3
:100C0000170E0401FA6F050EF96FFB6B0BECC7F0C2
:100C10009AD8FB6B0BECC7F079D833ECC3F0050125
:100C2000F96FF9A31CD0170EABECC3F033ECC3F093
:100C30000501FB6F170E0301FB6F020EFA6F33EC19
:100C4000C3F00501FC6F7AD8FBC5FBF40BECC7F0D1
:100C500082D8F96FFCC5FBF40BECC7F013D07BD83E
:100C60005AD80BECC7F06AD8D20EFB6F0BECC7F06A
:100C7000170E61D873D80BECC7F0170E69D84BD894
:100C80000BECC7F00401FA6B090EF96F3FD833EC97
:100C9000C3F0FB6F0BECC7F01B0E0501E86F280ECD
:100CA000E96F1DEFD0F0FDC5F9F3FEC5FAF30301BE
:100CB0001200200E0501FD27000EFE23000C170E6A
:100CC0000401FA6FB10EF96F010EFB6F010C170EE4
:100CD0000401FA6FB40EF96F040EFB6F040C170ECB
:100CE0000401FA6FB30EF96F030EFB6F030C170EBE
:100CF0000401FA6FB20EF96F020EFB6F020C170EB1
:100D00000401FA6FB00EF96FFB6BB00C170E030104
:100D1000FB6FFA6B170CF96F040EFB6F040C030EDC
:100D2000F96FFB6B030CF96F020EFB6F020CF96F8E
:100D3000010EFB6F010C0401FA6F010C0401FA6B48
:100D4000010EF96F010C0401FA6B0B0EF96F0B0C1D
:100D50000401FA6F020C0401FA6B020CF96FD20E57
:100D6000FB6FD20CF96F050EFB6F050CF96F1E0EB1
:100D7000FB6F1E0CF96F0A0EFB6F0A0CF96F080E61
:100D8000FB6F080C200E01015E6101D0200C65B2E2
:100D900012000201765101E1E0D11200560E0A6EF6
:100DA000050E0B6E400E0C6E6CECC6F0B36FB351BB
:100DB000D8B41200FDD96D0E036E310E0ADAF7ECCD
:100DC000C8F00150021007E1010E0301956F580EA3
:100DD0001E6E2D0E84D0F1D9790E036E310EF9D925
:100DE000F7ECC8F00150021007E1020E0301956F05
:100DF000690E1E6E2A0E73D0E0D97F0E036E310E7F
:100E0000E8D9F7ECC8F00150021007E1030E030126
:100E1000956F030E1E6E2A0E62D0CFD9850E036E1B
:100E2000310ED7D9F7ECC8F00150021007E1040EDB
:100E30000301956FCC0E1E6E2D0E51D0BED9450EFE
:100E4000036E310ECBD9F7ECC8F00150021007E168
:100E5000050E0301956F530E1E6E260E40D0ADD9C0
:100E60004C0E036E310EBAD9F7ECC8F001500210E7
:100E700007E1060E0301956F710E1E6E260E2FD030
:100E80009CD9530E036E310EA9D9F7ECC8F001506E
:100E9000021007E1070E0301956F350E1E6E280E36
:100EA0001ED086D9730E036E310E93D9F7ECC8F0BD
:100EB0000150021004E1080E0301956F080C78D967
:100EC0005A0E036E310E8AD9F7ECC8F001500210A9
:100ED00009E1090E0301956FD40E1E6E2B0E1F6ED5
:100EE000D1EFD0F065D9690E036E310E81D9F7ECE0
:100EF000C8F00150021002E1B2EFAEF059D98F0EE6
:100F0000036E310E75D9F7ECC8F00150021002E102
:100F10005EEFA3F04DD9270E036E300E046E066A05
:100F2000090E056EF7ECC8F00150021004E10B0E3B
:100F30000301956F0B0C3CD94C0E036E300E046E02
:100F4000066A070E056EF7ECC8F00150021004E1C6
:100F50000C0E0301956F0C0C2BD93A0E036E300E5C
:100F6000046E066A080E056EF7ECC8F00150021018
:100F7000D8A412000D0E0301956F0D0C9F0E1E6E6E
:100F8000010E1F6EDD0E206E2E0E216E0F0E236ED3
:100F9000BB0E226ED1ECCCF09F0E016E010E026EE4
:100FA0000E0E036E79ECD4F00301956B1200C5ECC4
:100FB000D5F0E80604E1BEECCAF0E80606E12C6ACA
:100FC0002B6A040E2E6E2D6A1ED0EBD879ECD4F06D
:100FD000EBD7140E016E2D0E026E100E036E79EC1F
:100FE000D4F001012C6BE0D7C5ECD5F0E80604E1A4
:100FF000BEECCAF0E8060DE1040E2C6E2B6A0D0E55
:101000002E6EE80E2D6E5F0E2F6E010E306E64EFA9
:1010100094F0C7D879ECD4F0C7D7BEECCAF0E80694
:1010200008E1E1D80D6A0DECCAF0CCD879ECD4F027
:10103000BBD7B7D879ECD4F0B7D7BEECCAF0E80686
:1010400009E1D1D8800E0D6E0DECCAF0BBD879EC59
:10105000D4F0AAD7A6D879ECD4F0A6D7BEECCAF0C3
:10106000E8061FE10501646B600E076E050E086E51
:101070009EECBFF007C0B5F108C0B6F13F0E0C6E94
:10108000FE0E0B6EB6C10DF00DECCAF03F0E0C6EED
:101090000B68B5C10DF00DECCAF094D879ECD4F022
:1010A00083D77FD879ECD4F07FD70C6A0B6A0D68B0
:1010B0000DECCAF0270E016E290E026E180E036E9B
:1010C00079ECD4F071D7040E0101B46FB4C10BF008
:1010D0000C6A0D680DECCAF00101B42BF7D7170E9E
:1010E0000C6E0B6A0D6A0DECCAF00C6A090E0B6EE1
:1010F0000D6A0DECCAF07A0E016E2F0E7ED879ECD7
:10110000D4F04A0E1E6E2F0E1F6ED1ECD0F04CD7CD
:10111000FEECADF00D6A0DECCAF09D0E016E2B0ECB
:10112000026E120E036E79ECD4F0CC0E1E6E2A0EF7
:101130001F6ED1ECD0F038D77BECA4F00DECCAF0E8
:10114000860E016E2F0E59D879ECD4F0560E1E6E15
:101150002F0E1F6ED1ECD0F027D70301955101E17E
:101160001DD6010A01E10AD7030A01E120D7010ACD
:1011700001E12FD7070A01E137D7010A01E14DD775
:10118000030A01E15AD7010A01E168D70F0A8DE08D
:10119000010A99E0020AA3E0070ABAE0010ACCE0DA
:1011A0001200EA0E016E2F0E026E0A0E036E0A0C7A
:1011B000560E016E050E026E12005A0E016E050EDD
:1011C000026E12001D0E016E300E026E090E036ECD
:1011D000090C046E066A050E056E050C046E066A9F
:1011E000060E056E060C3F0E0C6EFD0E0B6EFD0C12
:1011F000046E066A030E056E030C026E0B0E036E80
:101200000B0C010E0501FB6F110EFB2511EC9EF07E
:10121000090EFB250301FA6FFB6B170EFB2333EC62
:10122000C3F0DF6E110E0501FB2511EC9EF0460E9A
:10123000FB2528EC9EF0FB2B0F0EFB65E5D7140E6B
:1012400003013C6FC00E3D6F400E3E6FFB6B040E02
:10125000FA6F33ECC3F003018D6FFB6B050EFA6F71
:1012600033ECC3F003018C6FFB6B0A0EFA6F33ECA7
:10127000C3F001012B6F2BC163F30301646BFB6BA4
:101280000B0EFA6F33ECC3F00201546F170E03011B
:10129000FB6F270EFA6F33ECC3F00201996F030165
:1012A000FB6B030EFA6F33ECC3F00201516F0301C5
:1012B000FB6B0C0EFA6F33ECC3F00201AA6F030153
:1012C000FB6B0D0EFA6F33ECC3F003018A6FFB6BFF
:1012D0000E0EFA6F33ECC3F003018B6FFB6B0F0E36
:1012E000FA6F33ECC3F00201526F0301FB6B100E77
:1012F000FA6F33ECC3F00301866F020151A703D0EC
:101300000001618902D000016199170E0301FB6F92
:10131000060EFA6F33ECC3F0A50A06E10001618BFB
:101320008B8081ECB1F004D00001619B8B908B929B
:101330000301FB6B060EFA6F33ECC3F0FF0A0201E8
:10134000A96F0301FB6B070EFA6F33ECC3F00101C9
:101350005A6F0301FB6B080EFA6F33ECC3F0010107
:101360005B6F7CD933ECC3F00501F96FF9A109D0AB
:10137000578E5890579C090EE86F2E0EE96F1DECA2
:10138000D0F06CD933ECC3F00501F96FF9A309D0A3
:10139000579E5880579C270EE86F2E0EE96F1DEC64
:1013A000D0F05CD933ECC3F00501F96FF9A509D091
:1013B000579E5890578CE60EE86F2B0EE96F1DEC88
:1013C000D0F00301FB6B640EFA6F33ECC3F0010144
:1013D0004B6F0301FB6B650EFA6F33ECC3F0010139
:1013E0004A6F0301FB6B660EFA6F33ECC3F0020128
:1013F000876F0301FB6B670EFA6F33ECC3F00201DA
:10140000866F538C0301FB6B680EFA6F33ECC3F0ED
:101410000201856F0301FB6B690EFA6F33ECC3F0B9
:101420000201846F0301FB6B6A0EFA6F33ECC3F0A9
:101430000201836F0301FB6B6B0EFA6F33ECC3F099
:101440000201826F0301FB6B6C0EFA6F33ECC3F089
:101450000201816F0301FB6B6D0EFA6F33ECC3F079
:101460000201806F0301FB6B6E0EFA6F33ECC3F069
:1014700002017F6F0301FB6B6F0EFA6F33ECC3F059
:1014800002017E6FEBD833ECC3F00501F96FF9B7B9
:1014900058840301FB6B780EFA6F33ECC3F0020142
:1014A0005B6F0301FB6B790EFA6F33ECC3F0020143
:1014B0005A6F58B002D057AC03D03F0E5B175A6B2F
:1014C000040E851902E15BB123D0040E841902E1F8
:1014D0005BB31ED0040E831902E15BB519D0040E74
:1014E000821902E15BB714D0040E811902E15BB9E5
:1014F0000FD0040E801902E15BBB0AD0040E7F19E5
:1015000002E15BBD05D0040E7E1904E15BAF02D0A1
:10151000548601D05496040E851902E15AB123D0A5
:10152000040E841902E15AB31ED0040E831902E19D
:101530005AB519D0040E821902E15AB714D0040E1C
:10154000811902E15AB90FD0040E801902E15ABB89
:101550000AD0040E7F1902E15ABD05D0040E7E198F
:1015600005E15AAF03D00001698B02D00001699BED
:10157000060E0201851902E15B915A91060E84194B
:1015800002E15B935A93060E831902E15B955A952B
:10159000060E821902E15B975A97060E811902E145
:1015A0005B995A99060E801902E15B9B5A9B060EC5
:1015B0007F1902E15B9D5A9D060E7E1902E15B9F39
:1015C0005A9F5B515A15FF0A7D6F170E0301FB6F7F
:1015D000030EFA6F33ECC3F00501FA6FFAA102D0E3
:1015E00054825584FAA302D054845584FAA503D0BA
:1015F0000001698D55820501FAA703D00001698FAA
:101600005582170E0301FB6F040EFA6F33ECC3F023
:101610000201776F0301FB6B1B0EFA6F33ECC3F013
:101620000201496F0301FB6B140EFA6F33ECC3F038
:101630000201476F0301FB6B150EFA6F33ECC3F029
:101640000201466F0301FB6B1D0EFA6F33ECC3F012
:101650000301896F020151B106D00AD00301FB6B6F
:101660007A0EFA6F7A0C000160876099609512001B
:1016700000016097608960951200FC6F0501FC0510
:1016800001E001D155B602D055A49BD057BC54B04F
:101690000AD09C0EE86F2D0EE96F1DECD0F08BC2C6
:1016A0008CF2D890120002015E93DCD9E6ECA0F037
:1016B000C5EC81F0ADEC81F053BC8A9C55A472D08E
:1016C00054A406D00A0EC5D9010EADEC32F005D0F7
:1016D000040EBFD9010EADEC32F0000164AF05D0AD
:1016E000B2EC81F0E7D9E6ECA0F000016CAB08D0D9
:1016F00002015BA105D000016C9BB8D9ADEC32F0C2
:1017000000016CA909D002015BA306D000016C990D
:10171000D7D9010EADEC32F000016CA709D002015F
:101720005BA506D000016C97BFD9010EADEC32F07D
:1017300000016CA509D002015BA706D000016C95E1
:101740009BD9010EADEC32F000016CA307D0020171
:101750005BA904D076D9010EADEC32F000016CA18A
:1017600009D002015BAB06D000016C918BD9010E50
:10177000ADEC32F000016BAF09D002015BAD06D0D9
:1017800000016B9F85D9010EADEC32F000016BAD0D
:1017900009D002015BAF06D000016B9D7FD9010E1D
:1017A000ADEC32F0D1EC81F001E17BD7040E030106
:1017B000F76F79C2F8F3010ECCECBBF021EC82F0AC
:1017C00070D757BC54A007D0E10EE86F2C0EE96F1C
:1017D0001DECD0F066D753BE03D0000167A50ED034
:1017E00000016795ADEC81F0F76BF86B010ECCEC66
:1017F000BBF00201796B53BC8A9C53D755A027D00C
:1018000031D9E6ECA0F00FEC82F057D9E6ECA0F06D
:10181000EDEC81F041C2F7F342C2F8F356D91CEC6B
:10182000D2F0F7C341F2F8C342F20201425107E19C
:10183000240E415D04E2050E40D9E6ECA0F057AC61
:1018400003D019EC82F02DD7FBC589F22AD702010B
:101850008CA102D0010E14D08CA302D0020E10D0A5
:101860008CA502D0030E0CD08CA702D0040E08D099
:101870008CA902D0050E04D08CABB8EF81F0060E17
:101880008A6FB8EF81F0020EFC19D8A41200000193
:101890006AB502D055A28FD002015C93DFD8E6EC86
:1018A000A0F0C0EC81F0ADEC81F053BC8A9C55A255
:1018B00073D0000169AF06D00A0ECBD8020EADEC92
:1018C00032F005D0040EC5D8020EADEC32F00001A6
:1018D00064AF05D0B2EC81F0F0D8E6ECA0F00001E6
:1018E0006BAB09D002015AA106D000016B9BBED898
:1018F000020EADEC32F000016BA908D002015AA330
:1019000005D000016B99DCD8ADEC32F000016BA77B
:1019100009D002015AA506D000016B97C5D8020E66
:10192000ADEC32F000016BA509D002015AA706D038
:1019300000016B95A1D8020EADEC32F000016BA353
:1019400007D002015AA904D07CD8020EADEC32F0C7
:1019500000016BA109D002015AAB06D000016B91C6
:1019600091D8020EADEC32F000016AAF09D002014D
:101970005AAD06D000016A9F8BD8020EADEC32F052
:1019800000016AAD09D002015AAF06D000016A9D7C
:1019900085D8020EADEC32F0CAEC81F001E181D6BF
:1019A000040E0301F76F78C2F8F3020ECCECBBF023
:1019B0001DEC82F076D653BE02D067A30DD0ADECFD
:1019C00081F0000167930301F76BF86B020ECCEC1A
:1019D000BBF00201786B0FD754AE27D03FD8E6ECAE
:1019E000A0F0DFEC81F066D8E6ECA0F0F7EC81F037
:1019F0003FC2F7F340C2F8F368D81CECD2F0F7C34B
:101A00003FF2F8C340F20201405107E1240E3F5D6E
:101A100004E2050E4FD8E6ECA0F057AC03D025EC5D
:101A200082F03FD6FBC588F23CD602018CB112D7BA
:101A30008CB314D78CB516D78CB718D78CB91AD7E6
:101A40001BD700016C93020E0501F96F050EFA6FAA
:101A5000050C0501F96FFB05FA6F1200060E030174
:101A6000F76F020C060E0301F76F010C020E050161
:101A7000F96F010EFA6F010C020E0501F96F040EE9
:101A8000FA6F040C020E0501F96F060EFA6F060CD0
:101A9000020E0501F96F070EFA6F070C020E050121
:101AA000F96F080EFA6F080C020E0501F96F030EAC
:101AB000FA6F030C0301F76F020C0301F76F010CBF
:101AC000020E0501F96FFA6F020C0301FA6B030EA7
:101AD000F96F030C995172ECC3F0F9C446F6FAC4DD
:101AE00047F60601486B520E4825CAD9485146258B
:101AF0000301FA6F000E060147210301FB6F33EC6F
:101B0000C3F0DF6E0601482B0D0E4865ECD70201CD
:101B10002D6B2E6B53C6FCF56DD9030E0301FA6FC6
:101B2000E80EF96F1CECD2F046D9060153510F0BA9
:101B3000640DF3CF49F6F4CF4AF60601495102018C
:101B40002D2763D954C6FCF555D90301FA6B0A0E4B
:101B5000F96F1CECD2F02FD9060154510F0B06017E
:101B6000496F4A6B495102012D274FD92DC2F6F416
:101B70002EC2F7F469D98BECCBF0F65102014C6F11
:101B80004CC2F7F311D91CECD2F002012D5156D9F9
:101B90002E5140D98BECCBF0F65102014B6F4CC269
:101BA000F7F302D91CECD2F0F7C3FCF5F8C3FDF54E
:101BB0004BC2F7F355D91CECD2F00301F7510501E4
:101BC000FC270301F8510501FD2302012D510501F8
:101BD000FC250401F66F02012E510501FD2122D9D9
:101BE0008BECCBF0F65102014A6F4C51180DF3CF3C
:101BF000FCF54B519C0DF3CFFDF54A51F60DF3501A
:101C00000501FD25FC2502012D250301826F000140
:101C100060A91FD0010E0201506F4A514A250E0BD8
:101C200050134B39F00B700B50134C41800B501379
:101C3000D8904C31030B4F6FFBD803018239F00B66
:101C400002014F13000161A703D002014D6B01D0C7
:101C50001CD9000160A73AD0700E0501E86F2E0E66
:101C6000E96F2DC2EAF52EC2EBF51DECD0F0010EA6
:101C70000201506FFBD80501D890FD33FC33D8909A
:101C8000FD33FC33D890FD33FC33FC51FE0B0201D5
:101C90005013ECD80B0E0501FE6FD890FD33FC33CA
:101CA000FE2FFBD7FC51030B02014F6F2D39F00BB8
:101CB0004F13BED8000161A703D002014D6B01D0C4
:101CC000E4D84941E8423F0B010B4D13000161A7E5
:101CD00004D0A00E02014E6F08D00AEC5DF00201A4
:101CE0004E6FAF0E4E1901E1C6D0DDECBCF0020123
:101CF000C2D84D5106014B6F6BD8FCC5FFF50501ED
:101D0000FE6BA8D84D6B0501FF5106014E6F3CD804
:101D10004E5106014B6F5CD8FDC5FFF5FCC5FEF5C5
:101D2000050198D80501FE5106014D6F4E6B2CD868
:101D30004F515AD84BC6FDF54CC6FEF54DC6FFF5C2
:101D40000501FC6B06014B6B0501FD5106014C6F53
:101D50004D6B4E6B19D8505147D84C6B4D6B4E6B39
:101D600013D8F90E0501E86F250EE96F4DC2EAF5AB
:101D7000EB6B4EC2ECF5ED6B4FC2EEF5EF6B50C264
:101D8000F0F5F16B1DEFD0F04B510201231306016A
:101D90004C510201241306014D5102012513060185
:101DA0004E510201261312000301F86BFC0EFA6F6C
:101DB000180EF96F180CF7C349F6F8C34AF6060176
:101DC000495102012D2706014A5102012E2312001A
:101DD0004C6B4D6B4E6B4BC6FCF54CC6FDF54DC6C2
:101DE000FEF54EC6FFF5120006014B6F4C6B4D6BB6
:101DF0004E6B12000501FC390F0B0601496F4A6B4F
:101E000049C6F7F34AC6F8F3120006014A51020127
:101E10002E2312000301F8210401F76FF96B640E01
:101E2000F86F640C0401F76FF96B0A0EF86F0A0C77
:101E30004945E846FC0B0C0B4F1312000301F72534
:101E40000401F66F02011200030E0401F96FE80E9F
:101E5000F86FE80CFD6BFC6B06014B6B4C6B1200D2
:101E60000301F86BFA699C0EF96F9C0C2DC2FCF50E
:101E70002EC2FDF51200236B246B256B266B12001E
:101E8000D96EDA6A060EDA221200020E02014D6FD6
:101E9000020C81B00AD0819AF18C180EB8D90201D7
:101EA000712B786A7684A496A38681A0AED1F19C2A
:101EB000819A740EACD9050E0001F11901E186D0AA
:101EC000CFD00001F0BFCCD07AD00001F0BDC8D097
:101ED00076D00001F0BBC4D072D00001F0B9C0D000
:101EE0006ED00001F0B7BCD06AD00001F0B5B8D018
:101EF00066D00001F0B3B4D062D00001F0A1818AB5
:101F0000F069AED00001EFBFABD059D00001EFBDFA
:101F1000A7D055D00001EFBBA3D051D00001EFB93D
:101F20009FD04DD00001EFB79BD049D00001EFB555
:101F300097D045D00001EFB393D041D00001EFA17D
:101F4000818AEF698DD00001EEBF8AD038D00001C0
:101F5000EEBD86D034D00001EEBB82D030D000017F
:101F6000EEB97ED02CD00001EEB77AD028D0000197
:101F7000EEB576D024D00001EEB372D020D00001AF
:101F8000EEA1818AEE696CD00001EDBF69D017D057
:101F90000001EDBD65D013D00001EDBB61D00FD0C5
:101FA0000001EDB95DD00BD00001EDB759D007D0DD
:101FB0000001EDB555D003D00001EDB351D0818AB9
:101FC0004FD00001EDA1818AED694AD00201715123
:101FD000090A01E176D7030A01E177D7010A01E195
:101FE00078D7070A01E179D7010A01E17AD7030A14
:101FF00001E17BD7010A01E17CD71F0A01E17DD70E
:10200000010A80E0030A82E0010A84E0070A86E010
:10201000010A88E0030A8AE0010A8CE00F0A8EE0D8
:10202000210A91E0030A93E0010A95E0070A97E08C
:10203000010A99E0030A9BE0010A9DE07F0A9FE004
:10204000010AA2E0030AA4E0010AA6E0070AA8E048
:10205000010AAAE0030AACE0010AAEE00F0AB1E00F
:102060001B0E0001F11901E186D0CFD00001ECBFB9
:10207000CCD07AD00001ECBDC8D076D00001ECBB4A
:10208000C4D072D00001ECB9C0D06ED00001ECB762
:10209000BCD06AD00001ECB5B8D066D00001ECB37A
:1020A000B4D062D00001ECA1818AEC69AED000010D
:1020B000EBBFABD059D00001EBBDA7D055D000018C
:1020C000EBBBA3D051D00001EBB99FD04DD00001A4
:1020D000EBB79BD049D00001EBB597D045D00001BC
:1020E000EBB393D041D00001EBA1818AEB698DD095
:1020F0000001EABF8AD038D00001EABD86D034D0D2
:102100000001EABB82D030D00001EAB97ED02CD0E9
:102110000001EAB77AD028D00001EAB576D024D001
:102120000001EAB372D020D00001EAA1818AEA69F5
:102130006CD00001E9BF69D017D00001E9BD65D0BE
:1021400013D00001E9BB61D00FD00001E9B95DD027
:102150000BD00001E9B759D007D00001E9B555D03F
:1021600003D00001E9B351D0818A4FD00001E9A129
:10217000818AE9694AD002017151090A01E176D7E1
:10218000030A01E177D7010A01E178D7070A01E1E3
:1021900079D7010A01E17AD7030A01E17BD7010A65
:1021A00001E17CD71F0A01E17DD7010A80E0030A23
:1021B00082E0010A84E0070A86E0010A88E0030A57
:1021C0008AE0010A8CE00F0A8EE0210A91E0030AFE
:1021D00093E0010A95E0070A97E0010A99E0030AF3
:1021E0009BE0010A9DE07F0A9FE0010AA2E0030A4A
:1021F000A4E0010AA6E0070AA8E0010AAAE0030A8F
:10220000ACE0010AAEE00F0AB1E0F2921200D66E25
:10221000F294F28AD58E1200A496BC0E776E786A7C
:1022200056A42AD00001F551F81905E1F092F08882
:10223000A39656941200F95105E18A92F82B0A0EE2
:10224000F96F0A0CF90506E1F85102E18A9211D002
:102250008A820FD00A0EF919FBE0A20E7AD9DFA00C
:1022600002D08A9201D08A82A20E000172D9D8903F
:10227000DF320001F90712000001F6513DE05684FB
:102280000A0EF96FF86BF60508E1060E68D9A20E82
:102290004ED960ECB6F06DD92DD0020EF6190AE1D8
:1022A000060E5DD9A10E43D960ECB6F062D95CD9B7
:1022B0008C8E20D0030EF61909E1040E50D9400E81
:1022C000A36F480EA46F500EA56F14D0040EF6191C
:1022D00011E1050E44D9440EA36FA46BA20E016E4A
:1022E000030E026EF5C003F060ECB6F0DBC0A5F3A0
:1022F0001CC1A6F30001F66B56A60DD1F95101E001
:10230000FFD05696F092F088A39681B4B2D7A20E71
:1023100020D90101551DDF6E0001F82B310EF86543
:1023200001D0F86BA20E016E030E026EF8C003F02E
:10233000D6ECCBF002E3040EF66F0101545131E10B
:10234000A20E016E030E026EF8C003F0AAECD1F0EB
:1023500001E2CDD01E0E366F5986A20EF4D860EC85
:10236000B6F001E2C4D0020190510301A51901E1C8
:10237000BED056A204D0A5C390F25692B8D090C257
:10238000F7F0B80E0001F71902E1F76B01D0F72B57
:10239000010E0101546F130E0301726F880E716FED
:1023A000A6D0540517E1A20E016E030E026EF8C00E
:1023B00003F0E7ECCFF001E29AD0A20EC4D860ECB3
:1023C000B6F001E294D0010E0001F66F020E010199
:1023D000546F8DD0020E54193AE1A20E016E030E15
:1023E000026EF8C003F0C1ECD1F001E280D0A20E81
:1023F000AAD860ECB6F07BE3020E0001F66F030E84
:102400000101546F0A0E0301A41903E10501006BD9
:1024100002D0A4C300F50A0E0301A51903E10501CA
:10242000016B02D0A5C301F50A0E0301A61903E151
:102430000501026B02D0A6C302F50A0E0301A7191B
:1024400003E10501036B53D0A7C303F550D0030E7E
:1024500054194DE1A20E016E030E026EF8C003F096
:10246000D8ECD1F044E3A20E6ED860ECB6F03FE3B6
:10247000030E0001F66F0101546BF7C090F20301E7
:10248000A7290501046FAAC339F0060E3A6ED89049
:1024900039323A2EFCD7030E39160301A9390F0B36
:1024A0000C0B39100501056F052B8C8E5DD8F5ECF2
:1024B000B5F07A0E1E6E2D0E1F6ED1ECD0F0A50E6B
:1024C0001E6E2A0E1F6E00C520F0216A01C522F083
:1024D000236A02C524F0256A03C526F0276A04C5CD
:1024E00028F0296A05C52AF02B6AD1ECD0F000014A
:1024F000F65101E1BED67768786AF098A386B9D61E
:10250000F90503E181A4F86BB4D6D89081B4D880E2
:1025100001015533AED656B881A412000101556BA6
:1025200056985686090E0001F96FF098090CA36FB2
:102530004E0EA46FF7C0A5F3A20E016E030E026E3D
:10254000F5C003F01200016E030E026EF8C003F036
:102550001200F825D96EDA6A030EDA221200F56F3E
:10256000080E0301A26F080C0301766BFA0E756F5B
:10257000FA0CDBC0A6F31CC1A7F312002E0E060155
:10258000436FE00E426F01D004008FD9FDE1432973
:10259000FBE19B8CEA0E436F600E426F01D004009A
:1025A00084D9FDE14329FBE1F26AF06A9D6AA06AE1
:1025B000BB6AB66AC66AAC6AC26A060EC16EC088D9
:1025C000C16AF80EC26EC098896A8C6A2F0E926E2C
:1025D0000F0E956E8A6A8D6A050E936E020E966EC8
:1025E000F19E8B6A8E6AC40E946E3C0E976E8B9031
:1025F0008B928F6A656A180E986E868E8D848C8E8B
:102600008F80416BFD0E436FE80E426F01D00400D6
:102610004CD9FDE14329FBE1412B090E4165F2D77D
:10262000170ECA6E9F929E929D82080ECD6E9F904D
:102630009E909D90010EFDECD3F0810E796EF60E0A
:102640007B6E3C0E7A6EA192A282A092A586A8947F
:10265000260EAB6E9C8E9C98A88AA49AA39A3A1FC9
:10266000FB6BFA6B33ECC3F0280A14E00301FB6B3D
:10267000FA6B33ECC3F0280A0DE00201735101E05C
:10268000D6D082EC84F00401FA6BF96B280EFB6F54
:102690000BECC7F001EC89F0C7EC98F0E6EC95F094
:1026A000140E0201A26F010EA36FA46F0101216B32
:1026B00003017B6B0601446B320E4425D96EDA6A46
:1026C000050EDA22DF6A442B140E4465F5D7010E9D
:1026D00001013D6F3C6F598659841E0E366F030110
:1026E000616B626B3F6B406B416B426B640E02012E
:1026F000976F00016493639F64A302D0648502D046
:102700000001649563AF02D0648102D0000164913E
:102710000201656B810E5E6F010E5F6F810E5C6F53
:10272000010E5D6F54A402D08A0ECAD854A202D002
:10273000820EC6D8000169AF02D08A0EBCD8000153
:1027400069AD02D0820EB7D8050E0201646F5EC279
:1027500063F25FC262F25CC261F25DC260F20601C6
:10276000446B280E4425D96EDA6A030EDA22DF6A3A
:10277000210E4425D96EDA6A030EDA22DF6A442B71
:10278000060E4465EED70401F56BF46B0FECB5F063
:102790000201AB6FABC2A8F2ABB15A8EABA15A9E8D
:1027A000ABB35A8AABA35A9AABB55A86ABA55A9625
:1027B000ABB75A82ABA75A92ABB9598EABA9599E07
:1027C000ABBB598AABAB599A5AAE02D05A8C01D0E6
:1027D0005A9C5AAA02D05A8801D05A985AA602D0B6
:1027E0005A8401D05A945AA202D05A8001D05A90E9
:1027F00059AE02D0598C01D0599C59AA02D059889F
:1028000001D059980001649D649B58A80DD058A42C
:1028100003D0A8C28BF204D00201A851A9198B6F72
:102820008BC24CF18BC28CF29E9C9F8C9D8CA0889D
:10283000A2880201596B89888B908B92000161AB51
:102840000ED083500F0B0601406F0F0E401902E0AF
:102850008D94F7D78B8000F000F08B82A0828F9050
:102860008C9ED08EF28CF28E310E0501E86F300E08
:10287000E96F1DECD0F00201966B010E986FCD6AE6
:10288000569A8A0E0501E86F2B0EE96F1DECD0F009
:1028900043C21EF1EFECB7F0300EA06F380EF5EC2E
:1028A000B7F0A5EC5CF09A6F300C06014207D8A097
:1028B00043074229120002015C6F010E5D6F010C9B
:1028C0005E6F010E5F6F010C2D502E1001E11200A2
:1028D000056A046AA2ECC6F00201735101E012001D
:1028E000030169516A113CE12D502B24316E2E50A9
:1028F0002C20326E31C047F332C048F3496B4A6B2B
:102900004ABF0AD04A51491106E14705800E48598D
:10291000D8B0120001D012002BC067F32CC068F3AE
:102920002BC012F12CC013F100017E6B7D0E016EE5
:102930002A0E026E130E036E79ECD4F03DD92D6B86
:10294000EA0E0001B06F600EAF6F01D000F0000121
:10295000AF07D8A0B007AF29F9E1B029F7E112001D
:1029600001011251316E1351326E336A346A030120
:102970004751315C48513258495133583450800ADC
:10298000356E4A51800A355801E3B2D000017E6BA2
:1029900012C167F313C168F3B56BB46B08D967C391
:1029A00004F068C305F0A2ECC6F0DF6E0301674BCC
:1029B000682B0001FCD8DE2802E0010EB56FB42BB5
:1029C0000F0EB465EBD7B55106E1100E01011227C9
:1029D000000E1323000C7E0E016E670E026E310E88
:1029E000036E5EECCFF0100E0001B26F13C1B3F0B6
:1029F000E8D81DECD4F0C7D8B3390F0BF9ECD4F0FC
:102A0000ADD8B3510F0BF9ECD4F0B2D812C1B3F07A
:102A10000001D7D81DECD4F0B6D8B3390F0BF9ECC0
:102A2000D4F09CD8B3510F0BF9ECD4F0A1D87E0EA2
:102A3000016E900E026E310E036E5EECCFF000015F
:102A4000B46BB5D8DF50B16F0101124B132B0001ED
:102A5000B151B2277E0E016E1DECD4F094D8B1397D
:102A60000F0BF9ECD4F07AD8B1510F0BF9ECD4F08C
:102A70007FD80001B42B0F0EB465E3D7B251000824
:102A8000B26F7E0E016E1DECD4F07DD8B2390F0B03
:102A9000F9ECD4F063D8B2510F0BF9ECD4F0DF6E3F
:102AA000B5C031F0020E312676D80D0EDF6EB5C0FE
:102AB00031F0030E31266FD80A0EDF6EB5C031F04B
:102AC000040E312668D8DF6A7E0E016E1DECD4F04C
:102AD00001500001B56F7E0E016E026AB5C003F0B1
:102AE00079ECD4F001012D6B0301694B6A2B1200C4
:102AF000020E01012D61020C2D510DE100017E6BD2
:102B0000C20E016E2B0E026E110E036E79ECD4F024
:102B100053D82D2B12002D05D8A412007E0E40D8BC
:102B200069C322F06AC323F0D1ECCCF01E5000013F
:102B3000B46F7E0E016E026AB4C003F079ECD4F07B
:102B4000050156695769586959695A695B695C6931
:102B50005D690301956B696B6A6B1200DF6EB5C02E
:102B600031F0312A31507E0FD96EDA6A000112003D
:102B7000DF6EB5C031F0020E312631507E0FD96EB6
:102B8000DA6ADF6A120001500001B56FB5517E0F9D
:102B9000D96EDA6A120031507E0FD96EDA6A1200ED
:102BA0001E6E1F6A3E0E206E310E216E1200B45151
:102BB0006E0FD96EDA6A12000301694B6A2B0101AC
:102BC0001200B351B2277E0E016E120059B002D02E
:102BD00059A209D0F292F288450ED56EF184F29492
:102BE000F29A440E66D959A205D0040EBB6E9E948B
:102BF0009F849D8458AA06D0AD947E86010E7F6E78
:102C0000370E3ED958AE0BD0290EE86F310EE96F62
:102C10001DECD0F0AD847E867F6A670E31D958AC4A
:102C200006D0AD947E86090E7F6EC20E29D958A6B5
:102C300009D0F188F092F08EF088060E766E0201CF
:102C40009069568258A8120057AE7FD0C50ED56E37
:102C5000A30ED66EF184F294F28A4C0E2AD91ED9B4
:102C600001D00400020171077129FBE1726B040EAF
:102C700003ECD1F00501FB6F3E0EFB6103D00201B6
:102C8000729302D002017283080E03ECD1F00501A9
:102C9000FB6F3E0EFB6103D00201729502D0020170
:102CA00072850C0E03ECD1F00501FB6F3E0EFB614B
:102CB00003D00201729702D002017287F5D801D0C9
:102CC0000400020171077129FBE10501F96B040E93
:102CD00003ECD1F00501FB6F3E0EFB6102D0F993CE
:102CE00001D0F983080E03ECD1F00501FB6F3E0E15
:102CF000FB6102D0F99501D0F9850C0E03ECD1F0FF
:102D00000501FB6F3E0EFB6102D0F99701D0F987F8
:102D1000020172510501F919FB6FFBB309D0AE0E28
:102D2000E86F270EE96F1DECD0F0EEECC3F00AD08F
:102D3000FBB508D0380EE86F250EE96F1DECD0F01A
:102D400015ECCDF086969886120058B002D057AC9C
:102D50001200D56AD00ED76EF00ED66EF294F184C2
:102D6000F28AD58E280E766EA586A496DD0E776E35
:102D7000A38676948DD833ECC3F0E80607E088D8B4
:102D800033ECC3F0E80602E058ECD5F087D801D068
:102D90000400020171077129FBE1726B040E03EC60
:102DA000D1F00501FC6F3E0EFC6103D0020172936D
:102DB00002D002017283080E03ECD1F00501FC6F12
:102DC0003E0EFC6103D00201729502D002017285B1
:102DD0000C0E03ECD1F00501FC6F3E0EFC6103D03C
:102DE0000201729702D0020172875ED801D00400FE
:102DF000020171077129FBE10501FA6B040E03EC76
:102E0000D1F00501FC6F3E0EFC6102D0FA9301D0B7
:102E1000FA83080E03ECD1F00501FC6F3E0EFC6155
:102E200002D0FA9501D0FA850C0E03ECD1F0050121
:102E3000FC6F3E0EFC6102D0FA9701D0FA870201C6
:102E400072510501FA19FC6FFCB309D0CA0EE86F84
:102E5000270EE96F1DECD0F058ECD5F00AD0FCB588
:102E600008D0790EE86F250EE96F1DECD0F0CEEC9E
:102E7000CEF086969886949C8B9C949482941200B3
:102E8000B06EAC8EAC88AD8A9F8A9E9A9D8A1200E5
:102E9000170E0301FB6F300EFA6F300C8696989672
:102EA000E80E0201716FE80C721F8686E80E716FE2
:102EB000E80C766EA586A496A3961200CA6BCB6B1F
:102EC000FAD0250ECF1919E022D9DE50DE10DE101F
:102ED0002EE01DD901D80BD00500FA6EDE50FD6E34
:102EE000DE50FE6EDE50FF6EFA50CF51120002012E
:102EF000CA4BCB2BE0D033D9FAD7CC6B21D0CC8FB7
:102F00002FD0F4D8DF50CF6F02D9DE50DE10DE10A4
:102F10000EE0FDD801D8EBD70500FA6EDE50FD6E4D
:102F2000DE50FE6EDE50FF6EFA50CF511200BFC26F
:102F3000D9FFF4D8CFC2DFFFDED7C00ECC1310D03C
:102F400001D901E1BBD0580ADAE03B0ADAE0070A0E
:102F500007E00D0A05E01C0AF0E00D0AD0E0D4D726
:102F6000CCC2C5F2C00EC5170BE1C0D80BD9CEAF8D
:102F70002AD0030ECC13CD6DCE1FD8B0CE2B23D0CC
:102F8000B5D800D920D0010ECF6FCF51A3D89BD890
:102F9000F550CD5D0900F550CE591CE3CF2B050E41
:102FA000CF1918E0F2D7010ECF6FCF5199D88BD837
:102FB000F550CD5D0900F550CE590CE3CF2B040E32
:102FC000CF1908E0F2D7CC51C00BDDE0800AEBE06E
:102FD000400AD9E0CCC2C5F2030EC5171DE097D850
:102FE000DE50DE10DE1011E092D801D80AD00500C4
:102FF000FA6EDE50FD6EDE50FE6EDE50FF6EFA5051
:103000002D0C0201CA4BCB2B07D0BFC2D9FF86D8EB
:103010002D0EDF6EA4D8F5D7CFC2C9F249D0C95161
:1030200059D851D8A4D8A9D8B1ECCBF0B3C2BAF2D0
:10303000B4C2BBF2BD6B0A0EBC6FF8ECCDF0BA5156
:10304000300FCF6F17D099D8C9514AD83CD88FD8F4
:10305000B1ECCBF0B3510F0BC86FD00EC82569D8B7
:10306000F5CFCFF207D0CC51C00BD9E0800AEBE00E
:10307000400AD5E04CD8DE50DE10DE1012E047D812
:1030800001D80BD00500FA6EDE50FD6EDE50FE6EEC
:10309000DE50FF6EFA50CF5112000201CA4BCB2B0B
:1030A00007D0BFC2D9FF3AD8CFC2DFFF58D8F5D773
:1030B000C907C929D8E146D801E003D7CAC2BFF27F
:1030C000CBC2C0F21200F420F76EF86A000EF822AC
:1030D00009001200020DA70EF324F66E200E120056
:1030E000020DB10EF324F66E200E1200C3C2D9FFFA
:1030F000C4C2DAFFDFCFC5F2020EDE26DFCFC6F292
:10310000000EDD22C5C2D9FFC6C2DAFF000C20EED8
:1031100002F0BF51D926C051DA221200C0C2DAFF34
:10312000DECFC5F2DDCFC6F2C5C2D9FFC6C2DAFF17
:103130001200F66EF76A2C0EF722F86A000EF822DB
:1031400008001200C1C2F6FFC2C2F7FFC14BC22B7A
:10315000000EF86E0800F5CFCFF2CF511200BFC2BB
:10316000D9FFC0C2DAFFDE2A000EDD22000CF5CF47
:10317000B5F20A00F5CFB6F21200CDC2B3F2CEC25C
:10318000B4F21200DECFCDF2DDCFCEF212005992B2
:103190005990589E589683500F0B0501FF6F100EE3
:1031A0000201716F01D00400020171077129FBE176
:1031B00083500F0B0501FE6FFE51FF19ECE1FFB1CB
:1031C00017D0020151A10AD033EC8BF01C0E05017F
:1031D000E86F2C0EE96F1DECD0F015D038EC8BF0B9
:1031E000360E0501E86F2D0EE96F1DECD0F00BD007
:1031F0000001609960976085640E0501E86F2B0EF1
:10320000E96F1DECD0F002012F6B306B000160A55F
:103210000CD00301FB6B020EFA6F33ECC3F017D92D
:10322000010EFA6F33ECC3F00BD00301FB6B120EEF
:10323000FA6F33ECC3F00BD9110EFA6F33ECC3F015
:103240000501F96FFA6BFB6902012F510501FD6F52
:10325000FC6BFA51FC17FB51FD17F951FC250201DB
:103260002F6F0501000EFD210201306F436B446B8F
:103270002FC2F6F430C2F7F424EC8FF08BECCBF0D5
:10328000F6510201576F57C2F7F3D4EC8EF01CECE5
:10329000D2F002012F511EEC8FF030510AEC8FF06A
:1032A0008BECCBF0F6510201566F57C2F7F3D4EC1A
:1032B0008EF01CECD2F0F7C3F9F5F8C3FAF556C25C
:1032C000F7F330EC8FF01CECD2F00301F75105015D
:1032D000F9270301F8510501FA2302012F510501D5
:1032E000F9250401F66F020130510501FA2112ECB3
:1032F0008FF08BECCBF0F6510201556F5751180D42
:10330000F3CFF9F556519C0DF3CFFAF55551F60D63
:10331000F3500501FA25F92502012F2503018F6FCE
:10332000020157510501F96FFA6B0C0ED890F9376D
:10333000FA37E82EFBD77ED856510501FA6FF96BA4
:1033400079D855510501F96FFA6BF93BFA3BF00E4C
:10335000FA17F9510F0BFA13F00EF9176BD8030196
:103360008F51020143130F0E0501FF1B0E0EFF17B5
:10337000FF5103E1589E59820CD00C0EFF1904E155
:10338000589E5992598006D0060EFF1905E1588EB5
:1033900059925990589C07D0040EFF1906E1589E87
:1033A00059925990588C589A05D0080EFF1904E18B
:1033B00049D8588A58960ED00A0EFF1904E142D80F
:1033C000589A588607D00E0EFF1904E13BD8589A38
:1033D0005896588858A604D0620EE86F2F0E27D052
:1033E00058AA04D08C0EE86F2E0E21D058AC04D011
:1033F000BC0EE86F2D0E1BD058AE04D0F80EE86F4F
:103400002B0E15D059A204D0550EE86F2A0E0FD0FE
:1034100059A004D0D00EE86F2E0E09D058A804D0C1
:10342000180EE86F2E0E03D0030EE86F2D0EE96F15
:103430001DEFD0F0F951020143130501FA510201C9
:1034400044131200589E59925990589C1200020140
:103450002F6F306B0301FB6B1200A396769458A874
:10346000E7D090D081B402D0E38FE0D081B402D015
:10347000E38DDCD081B402D0E38BD8D081B402D00C
:10348000E389D4D081B402D0E387D0D081B402D014
:10349000E385CCD081B402D0E383C8D081B402D01C
:1034A000E381C4D081B402D0E28FC0D081B402D015
:1034B000E28DBCD081B402D0E28BB8D081B402D00E
:1034C000E289B4D081B402D0E287B0D081B402D016
:1034D000E285ACD081B402D0E283A8D081B402D01E
:1034E000E281A4D081B403D00301988F9FD081B42E
:1034F00003D00301988D9AD081B403D00301988B37
:1035000095D081B403D00301988990D081B403D0C1
:10351000030198878BD081B403D00301988586D0AE
:1035200081B403D00301988381D081B403D0030117
:1035300098817CD081B403D00301978F77D081B478
:1035400003D00301978D72D081B403D00301978B10
:103550006DD081B403D00301978968D081B403D0C2
:103560000301978763D081B403D0030197855ED0B0
:1035700081B403D00301978359D081B457D003019C
:10358000978154D00001E151130A01E16BD7060A7B
:1035900001E16CD7020A01E16DD70E0A01E16ED795
:1035A000020A01E16FD7060A01E170D7020A01E1C0
:1035B00071D73E0A01E172D7020A01E173D7060A08
:1035C00001E174D7020A01E175D70E0A01E176D74D
:1035D000020A01E177D7060A01E178D7020A01E180
:1035E00079D71E0A01E17AD7020A01E17BD7060AE0
:1035F00001E17DD7020A80E00E0A83E0020A86E03C
:10360000060A89E0020A8CE07E0A8FE0020A92E054
:10361000060A95E0020A98E00E0A9BE0020A9EE084
:10362000060AA1E0020AA4E01E0AA7E0A49612007E
:10363000090E0201716106D00001D890F137F191B5
:1036400081A4F181090E0201716508D0120E716129
:1036500005D0D8906837689181A46881110E716592
:1036600009D01A0E716106D00101D8903B373B9109
:1036700081A43B81190E0201716504D0220E716193
:1036800001D08150210E716509D02A0E716106D0DA
:103690000101D8903A373A9181A43A81290E02016A
:1036A000716509D0320E716106D00101D8903937A9
:1036B000399181A43981310E0201716509D03A0E28
:1036C000716106D00101D8903837389181A43881D2
:1036D000390E0201716508D0420E716105D0D89093
:1036E0006737679181A46781410E716509D04A0EE1
:1036F000716106D00101D8903737379181A43781A5
:10370000490E0201716504D0520E716101D08150E1
:10371000510E71658BD75A0E716188D7815086D74B
:10372000E26BE36B0CD1250EE71919E021D9DE50CD
:10373000DE10DE102EE01CD901D80BD00500FA6E89
:10374000DE50FD6EDE50FE6EDE50FF6EFA50E75129
:1037500012000501E24BE32BF2D029D9FAD7E46B32
:1037600021D0E48F2FD0F3D8DF50E76F01D9DE509E
:10377000DE10DE100EE0FCD801D8EBD70500FA6EA3
:10378000DE50FD6EDE50FE6EDE50FF6EFA50E751E9
:103790001200DAC5D9FFF3D8E7C5DFFFDED7C00EC8
:1037A000E41310D0F7D801E1CDD0580ADAE03B0A93
:1037B000DAE0070A07E00D0A05E01C0AF0E00D0A4E
:1037C000D0E0D4D7E4C5FDF4C00E0401FD170CE130
:1037D000BED800D90501E6AF2ED0030EE413E56D87
:1037E000E61FD8B0E62B27D0B2D8F4D824D0010EEB
:1037F000E76FE7516AEC98F063EC98F0F550E55DFF
:103800000900F550E6591FE3E72B050EE7191BE009
:10381000F0D7010EE76FE75170EC98F063EC98F089
:10382000F550E55D0900F550E6590DE3E72B040E70
:10383000E71909E0F0D70501E451C00BD8E0800A90
:10384000E8E0400AD4E0E4C5FDF4030E0401FD17EE
:103850001EE005018DD8DE50DE10DE1011E088D8A4
:1038600001D80AD00500FA6EDE50FD6EDE50FE6E05
:10387000DE50FF6EFA502D0C0501E24BE32B07D012
:10388000DAC5D9FF7CD82D0EDF6E91D8F5D7E7C504
:10389000E1F551D0E1516AEC98F063EC98F08FD8E3
:1038A00094D88BECCBF0F6C4D6F5F7C4D7F5050168
:1038B000D96B0A0ED86F44ECCCF00501D651300F0D
:1038C000E76F1BD082D8E15170EC98F063EC98F070
:1038D00076D88BECCBF0F6510F0B0501E06FD00ED4
:1038E000E02599EC98F0F5CFE7F507D0E451C00B4F
:1038F000D1E0800AE7E0400ACDE03AD8DE50DE10A1
:10390000DE1012E035D801D80BD00500FA6EDE507B
:10391000FD6EDE50FE6EDE50FF6EFA50E751120073
:103920000501E24BE32B07D0DAC5D9FF28D8E7C55C
:10393000DFFF3DD8F5D70501E107E129D7E12AD816
:1039400001E0F1D6E2C5DAF5E3C5DBF51200DEC52C
:10395000D9FFDFC5DAFFDFCFFDF4020EDE26DFCFB1
:10396000FEF4000EDD22FDC4D9FFFEC4DAFF000C18
:1039700020EE02F0DA51D926DB51DA221200DBC543
:10398000DAFFDECFFDF4DDCFFEF4FDC4D9FFFEC4C7
:10399000DAFF1200DCC5F6FFDDC5F7FFDC4BDD2BDF
:1039A000000EF86E0800F5CFE7F5E7511200DAC512
:1039B000D9FFDBC5DAFFDE2A000EDD22000CF5CFD1
:1039C000F8F40A00F5CFF9F41200E5C5F6F4E6C5FF
:1039D000F7F41200DECFE5F5DDCFE6F512002305A2
:1039E0007DE1010E0201DF6F110EDF251AD9640E91
:1039F000DE1823E11FD9DF5020E123D9640EB76F11
:103A000067ECC8F09A0E0201D06F2C0E31D951EC40
:103A1000D0F0FDD8350EF6D8310E25D9CCECCFF04C
:103A2000A6ECD4F02AD9CCECCFF02CD9A6ECD4F06B
:103A3000A5EC5CF014D9ACECACF0F8D8F2D85A0E86
:103A4000DF601DD0F7D85A0EDE1819E1E50ED06FF1
:103A5000270E0ED951ECD0F0DAD8350ED3D803D9D1
:103A6000CCECCFF0A6ECD4F008D9CCECCFF00AD94E
:103A7000A6ECD4F0A5EC5CF0F2D8ACECACF0D6D867
:103A8000D0D8DF5022E1D6D8DF501FE0DAD8B76BAC
:103A900067ECC8F0910E0201D06F2A0EE9D851EC04
:103AA000D0F0B5D8350EAED8320EDDD8CCECCFF094
:103AB000A6ECD4F0E2D8CCECCFF0E4D8A6ECD4F06D
:103AC000A5EC5CF0CCD8ACECACF0B0D8AAD8460EE3
:103AD000DF25BED8DF2B100EDF6586D7110E010162
:103AE00023259FD8DF5004E0110E23259AD8DF0646
:103AF0000301395107E001012351A6ECD4F0030181
:103B0000351936E00F0E0101231905E18F800301FD
:103B1000786B230E776F86863A0EAE6EADA2FED717
:103B200001012351A6ECD4F0AE6EADA2FED7540E27
:103B3000AE6EADA2FED7450EAE6EADA2FED70101B0
:103B40002351A6ECD4F02B0AA5D8A6ECD4F0AE6E87
:103B5000ADA2FED79BD8A6ECD4F0AE6EADA2FED738
:103B60000D0EAE6EADA2FED70A0EAE6EADA2FED7A2
:103B7000A50E030139193BE101012351A6ECD4F054
:103B80000301351934E186863A0EAE6EADA2FED73A
:103B900001012351A6ECD4F0AE6EADA2FED736C320
:103BA000AEFFADA2FED737C3AEFFADA2FED7010177
:103BB0002351A6ECD4F00301361937193A0A020151
:103BC00069D8A6ECD4F0AE6EADA2FED75FD8A6EC55
:103BD000D4F0AE6EADA2FED70D0EAE6EADA2FED786
:103BE0000A0EAE6EADA2FED70301396B356B010133
:103BF000232B100E231902E1010E236F020E246FF6
:103C00008696020C0201A16F330EA06F330C8F80D9
